:020000040800F2
:1000000000A00020093E0108713E01083D2E0108B4
:10001000713E0108713E0108713E010800000000B8
:10002000000000000000000000000000713E010818
:10003000713E010800000000713E01085BBA000833
:10004000713E0108713E0108713E0108713E0108D0
:10005000713E0108713E01085D880008598800085A
:10006000713E0108713E0108713E0108713E0108B0
:1000700059F20008713E0108C38A0008713E010868
:10008000713E0108713E0108713E0108713E010890
:10009000713E0108713E0108713E01085588000853
:1000A0004DFD000889FD00083DFD0008ADFD00087C
:1000B0007DFD00086DFD00085DFD0008713E010832
:1000C000713E0108713E0108713E0108713E010850
:1000D000713E0108D1FF0008C5FF0008B9FF000804
:1000E00069BA0008713E0108713E0108713E0108BD
:1000F000713E0108713E0108713E0108713E010820
:10010000000000000000000000000000713E010837
:10011000713E0108713E0108713E0108713E0108FF
:10012000713E0108713E0108713E0108713E0108EF
:10013000713E0108713E010800000000000000004F
:10014000713E0108713E0108713E01080000000087
:10015000000000000000000000000000000000009F
:100160000000000000000000713E0108713E01081F
:10017000713E0108000000000000000000000000C7
:0801800000000000713E0108BF
:100188002DE9F04F2DED028B6A4F6B4B3B60AFB002
:1001980000237B6010F065FB18B910F085FB0BF0AD
:1001A80039F90BF0F1F9654A654C137843F001030E
:1001B8001370644B4FF47002C3F88820002309932E
:1001C8000A93236843F480332360236803F40033DD
:1001D8000A93099B013309930A9B1BB9099BB3F541
:1001E800A04FF2D1236813F4003318BF01230A93F8
:1001F8000A9B012B68D0534E534BF360636ABB6074
:10020800636ADFF874B1DFF87481DFF874A143F032
:1002180080736362636943F4FC032EAD6361032357
:100228008DF86A3041F6FF7325F8503D4FF0904045
:1002380029460FF001F94FF6FF7358462946ADF8E5
:1002480068300FF0F9F8414829460FF0F5F84048B2
:1002580029460FF0F1F83F4829460FF0EDF82946F6
:100268003D480FF0E9F828460CF076FD1A9B3B4A0A
:10027800B3FBF2F33A4A3B4913603B4B00221A6046
:100288005A603A4B5960F02186F823109A60384E2C
:1002980007221A60B368CAF8003098E80300636957
:1002A80085E8030043F4802363610823CBF8183002
:1002B8001A981BA90FF0C0F8DAF8003013F0080FED
:1002C800A8F10C0829D163E02A4B12221A6063684E
:1002D800636063686360636843F480636360636852
:1002E80023F47C136360636843F4E8136360236852
:1002F80043F0807323602268114B9001FBD55A6844
:1003080022F003025A605A6842F002025A60636897
:1003180003F00C03082BFAD16DE796F89231012B04
:1003280036D8044B96F893219B6813F0805900F057
:10033800D3852DE00001002087AC000800340020A0
:100348000010024000ED00E00005FA050008004832
:10035800000C0048001000480014004840420F00FC
:10036800441F00203F190100481F002010E000E052
:10037800202C00200020024000040048CC83010803
:10038800FC270020BD4B002283F893210BF098FA3C
:1003980064200BF054FBBA4800214FF48C7215F01E
:1003A80048FEE369B74843F00703E361A36943F4F0
:1003B800E123A361636943F4C023636100F5887492
:1003C800837B416890F80FE003F00702DB0801EB3C
:1003D80083039200196A4FF00F0C0EFA02FE0CFA12
:1003E80002F221EA02021A62196A10304EEA010288
:1003F800A0421A62E4D10022A349002353540132D7
:10040800112AF9D1A14AFF2199540133072BF9D1B7
:100418009F4BDAF800409F4A1A609F4800213C220F
:1004280015F007FEC4F3801905234FF0000E9B4A10
:1004380099481EF802100C2202FB0EF21154B9F171
:10044800000F07D11E3901299FBFFF2103F1FF3398
:100458001154DBB20EF1010EBEF1050FE7D1904A3F
:1004680096F805B013708F4B8F4983F800B08F4B07
:100478007B62C0330B608E4B8E4A03EBCB03A10625
:100488005B7848BF0123936200238B4A40F2DC511A
:1004980022F813100133082BF7D113A800211C22CE
:1004A80015F0C7FD14F4007A1DBF844B199503930A
:1004B800CDF80CA0BBF10E0F03D00BF0EF03082B07
:1004C80002D101238DF85E30022007F061FA18B1DD
:1004D8004088003018BF0120C4F340038DF8523023
:1004E800C4F340338DF84C30C4F3C03300F001003E
:1004F8008DF84F3014F400638DF851008DF8549046
:1005080007D096F8863103F1FF3EDEF1000343EB96
:100518000E038DF85030C4F300438DF85530BB6A94
:10052800B6F84801ADF862001AF1000A18BF4FF09A
:10053800010A003318BF01238DF85730C4F3005364
:100548008DF85830B6F84A31ADF85C30B6F8563107
:10055800ADF85A3004F00101C4F38043C4F3C0027B
:10056800E40448BF45488DF85330B6F8543144BFC9
:10057800B0F85001ADF86200B3F5FA7FADF860301D
:1005880084BF0023ADF862304D4896F8D63187F81D
:100598002C30002387F82D3043709DF85E308DF89D
:1005A8004D10002B8DF84E208DF856A00CBF00235F
:1005B800022301B902B1013308EB83084FF00009A7
:1005C800D8F81430A3F1020A203304933AF8023F12
:1005D8004FF6FF72934200F0B1819DF85110DAB2E4
:1005E8001B0ADEB279B12748364C00EB021041688D
:1005F800A14208D10189B1F5806F00F09B81B1F566
:10060800006F00F097819DF8541031B111011D4819
:1006180040582D49884200F08D819DF8551079B1D8
:100628001101184C6018645828498C4200F08281E6
:100638004168B1F1904F03D1817B082900F07A819C
:100648009DF8521051B10F4800EB02104168B1F10A
:10065800904F03D10189102900F06C819DF84F104B
:10066800B1B30848174C00EB02104168A1422FD1E2
:100678000189042900F05E812AE000BF202C0020B7
:10068800941F002040A601080C0100201D01002035
:1006980014230020102E0020182300207BAE010810
:1006A800CD1000204009002028210020342C0020F3
:1006B80020AC01080001002038100020C083010888
:1006C8002D0100200004004800040040002C0140D7
:1006D8009DF8501051B1BE4800EB02104168B1F1CD
:1006E800904F03D10189202900F02481199C7CB105
:1006F800B74F216807EB02177868884208D1398913
:10070800A088884200F01681E088884200F01281B3
:10071800022B02D19DF84C3003E0012B04D19DF847
:100728004D30002B00F006819DF85710A84B17019B
:1007380059B19DF85E1041B9A2F10E01012904D802
:10074800D959A448814208BF04269DF85810DC19DD
:1007580031B19DF85E1019B9043A032A40F2D280EB
:10076800012E49D1DFF878820693D919FF2291F832
:100778000DE088F8742088F875204868C8F8844027
:1007880001F108020989ADF868104FF0000B022149
:100798008DF86B1088F878B01AA98DF86AE0059280
:1007A80088F830B0C8F834B0C8F838B0C8F83CB0E9
:1007B800C8F870B088F876B088F877B00EF03CFECC
:1007C800069B059AD85991785A4608F0BDFB2046F1
:1007D800594632460FF03CFB7F4BC8F888307F4BB8
:1007E800C8F88C30C8F890B0204608F1880108F1A4
:1007F8008C020FF083FB9DE0022E4BD15FFA89F348
:100808001C2101FB03FC764BCDF81CC003EB0C0B41
:1008180001238BF8783006936D4B8BF87990D919B2
:100828004FF0000891F80DE048688BF87A8001F1E4
:1008380008020989ADF868108BF882801AA9CBF8EC
:1008480084408DF86AE005928DF86B600EF0F4FD37
:100858005F4B059AD8599178424608F075FB069B7C
:1008680020461A4641460FF0F3FA5D4BDDF81CC0EE
:100878005C4ACBF8882003EB0C015B4ACBF88C2050
:100888008831CBF8908020460A1D0FF037FB09F11C
:1008980001094FE0032E33D19DF85330504E534F8A
:1008A8003BB196F82E80204608214FF6FF720023B0
:1008B8001AE0BDF8602096F82E80BDF86230B2F5D7
:1008C800FA7F0BD94A49B1FBF2F22046082192B2CD
:1008D8000EF0DBFD474B47F828000AE04649B1FB1C
:1008E800F2F22046012192B20EF0CFFD434B47F8B9
:1008F8002800C36096F82E30013386F82E3019E0B0
:10090800042E17D1364EBDF85A2096F82D703A4B62
:1009180093FBF2F22046BDF85C30012192B20EF052
:10092800B4FD96F82D3006EB87070133C7F8580158
:1009380086F82D30049B9A457FF448AE284F304BFB
:1009480097F82D2087F878212E4A1678A6F11702F5
:100958000024022A1C709E461BD87B6A2344D3EDD0
:10096800007AF5EE407AF1EE10FA03D1BB6A002B5B
:1009780050D126E0244A04EB020C0FCB8CE80F0080
:100988009EF8003010340133C02C8EF80030E4D1CA
:10099800ECE71E4B13F836808EF8008003EBC60395
:1009A800D3F80490B9F1000FE0D04445DEDA164AD6
:1009B800230103EB020C4B440FCB01348CE80F00EE
:1009C800F3E7134B1A6812F4805F984648D141E068
:1009D80040A6010800400140A1F0000881F100088C
:1009E80000010020E5F1000879F00008601F0020F0
:1009F80000127A00A1F1000840420F0091F10008AE
:100A0800901F0020400900207C08002020AC01082D
:100A1800FC2700202B4B2C4A13F83600107003EBF0
:100A2800C6035C68002CCCD000238342C9DAC3EB30
:100A3800C3016218DFF89C80D2F8009041F8089052
:100A480001EB080C9188ACF8041092798CF8062018
:100A58000133EAE706F0EF03082B1C4B20D121E015
:100A68009EF80020012AF5D9194B03EB0212103227
:100A780010339342EED053ED047AB6EE007A67EE67
:100A8800877A43ED047A53ED057A67EE877A43ED6A
:100A9800057A53ED037A67EE877A43ED037AE7E741
:100AA8000E2E08D11A7842F010021A70182E13D19F
:100AB8000BF028FA10E01A7822F010021A70192E9A
:100AC800F5E700BF40950108B42000201011002070
:100AD80084080020B52000200BF0F8F9D8F8003081
:100AE800B14CB24E580358BFB14BB2485CBF01225B
:100AF8001A70B14A137843F0040313704FF400439B
:100B0800ADF8683063694FF0020943F400234FF0F1
:100B1800010B8DF86B9029468DF86AB063610EF071
:100B28008BFCA64BA64A1A6000200AF0A7FFE369CF
:100B380043F48043E361236943F480432361636999
:100B480043F480236361736A23F470037362736AE6
:100B580043F4A0037362736A23F070637362736A69
:100B680043F0A0637362736A23F070437362736A1D
:100B780043F0A0437362736A23F470237362736A49
:100B880043F4A02373624FF460431A938DF86C907A
:100B980003234FF00009304629464FF4805A8DF858
:100BA8006D3004938DF86E908DF86F900CF046FAC6
:100BB800049B8DF86D3030462946CDF868A08DF835
:100BC8006CB08DF86E908DF86F900CF037FA236941
:100BD80043F480432361236923F480432361794BE1
:100BE8009A8822F480521204120C9A809A8892B23F
:100BF80042EA0A029A801A8802F4415242F4457283
:100C080042F003021A809A8822F470621204120CCD
:100C180042F4E0629A809A8B22F400621204120C69
:100C28009A8307221A821A8892B242F040021A80E6
:100C3800C6F818A0D8F8003003F41073B3F5107F85
:100C480000F09E80604B614E1E606369DFF85C9126
:100C580043F480236361E36943F40013E361236B86
:100C680023F010032363236B43F010032363D9F8A5
:100C7800203023F07063C9F82030D9F8203043F0D1
:100C88008063C9F82030D9F8203023F07043C9F8C0
:100C98002030D9F8203043F08043C9F820304FF095
:100CA80000084FF0020C4022484629464FF0030B3B
:100CB8008DF86CC0CDF818C01A928DF86E808DF83A
:100CC8006F808DF86DB00CF0B9F98022484629463E
:100CD8001A920CF0B3F93268DFF8089122F0010299
:100CE800326031683A4A0A4032603A4A32613268C0
:100CF80042F001023260C6F80880C6F80C80C6F8D7
:100D08000880B26842F40042B260326832607268A9
:100D180022F0784222F400427260326842F0010206
:100D28003260D9F800502C4E05F400434FF0100AF9
:100D38000493524605F4006330464146059315F086
:100D480078F94FF6FF72DDF818C00E9215F002051B
:100D58008DF83DC08DF83E808DF83F808DF83CB011
:100D680042D02EA94FF0904041F880AD0CF066F9C2
:100D780001250723357086F80180F370B57033E0DC
:100D880016490A784B4616481E561F2E02BFFF26E4
:100D98001E5402F1FF3203F10C0308BFD2B23C2B00
:100DA800F1D10A704EE700BF00100240000400486D
:100DB800A80D00200008004800340020103400204E
:100DC800DDB800080038004004100020005400403E
:100DD800FFE0CF007A25E00080230020CD1000201E
:100DE80018230020FC270020049B7BB12EA9042394
:100DF80041F8803D92480CF021F90C233371072308
:100E0800F371012375711D44B371EDB2059B83B174
:100E18002EA9202341F8803D4FF090400CF00EF9A8
:100E2800022333730723F373012375731D44B373CC
:100E3800EDB2E36A834823F4F873E362E36A43F4A8
:100E4800D873E362636943F0805343F0020363613C
:100E58000BF031FE1AA80BF003FE7B4B1A937B4B69
:100E68001B93012D4FF0000394BF1A4680221F9256
:100E78004FF48072734C20924FF4806221922022AA
:100E8800204622921AA94FF400521C931E932392D3
:100E98002493ADF874500BF0F0FD236843F0010380
:100EA80023606B4CA36823F04053A360A36843F00E
:100EB8008053A3600A200AF0C2FDA36823F0804390
:100EC800A360A368A360A36843F00043A360A2687B
:100ED8005F4B002A31DAFAE7531E092B3FF658AA6E
:100EE800D8F858002860294658460EF0A5FA4FF45D
:100EF8000063CBF818303C200AF0A1FD96F8933136
:100F08009945BFF63FAADFF838B108224FF40063CD
:100F1800CBF8182078200492ABF8283003930AF015
:100F280083FD049A039BABF828207820CBF818306F
:100F38000AF07AFD09F10109E0E79A68454922F0CB
:100F480040529A609A6842F000529A608868424A11
:100F5800024042F468328A60D968404A0A4042F442
:100F68000052DA601A6B013D22F00F0215431D632F
:100F78000021012372189078002800F084805C1CFE
:100F8800042B16F801E0D278DFF8C4C0E4B20ED81A
:100F980003EB4303DCF830505B001F20984025EA40
:100FA80000000EFA03F30343CCF8303031E0092B8C
:100FB8000ED80620053B4343DCF834501F209840E8
:100FC80025EA00000EFA03F30343CCF8343020E09E
:100FD8000E2B4FF006050ED8A3F10A006843DCF883
:100FE80038801F23834028EA03050EFA00F32B43B9
:100FF800CCF838300DE00F3B05FB03F0DCF83C8003
:101008001F23834028EA03050EFA00F32B43CCF88C
:101018003C30BEF1090F0E4822D983698569AEF1CB
:101028000A0303EB43034FF0070E0EFA03FE25EA0B
:101038000E05856185699A402A43826122E000BFD6
:10104800000400480804024040010050902300209A
:101058000001005000030050E010FCFF07C0FFFD36
:10106800436945690EF1FF3303EB43034FF0380E34
:101078000EFA03FE25EA0E054561456903339A40D9
:101088002A4342612346043110297FF473AFBB4BD6
:101098009A6842F001029A601A461168B74BC9076C
:1010A800FBD5DA6822F00202DA60DA6842F002025E
:1010B800DA60DA6842F00102DA609A6842F0040203
:1010C8009A60AF4AB2F85C319046002B41F07480C8
:1010D800B8F95E21002A41F06F80B8F96021002A32
:1010E80041F06A80D9F800309B031FD5C8200AF068
:1010F800A6FCAE2009F0B1FC08B109F0B3FCA14C84
:1011080087F87901C8200AF09AFC9F4BC7F87C3110
:1011180000210C22204614F08CFF0223E3700CF00F
:10112800A8FD0AF065FC994B0344A360984B9948C5
:101138001B68B8F86461B3F8563098F863B198F84A
:101148006B4198F86C51049300210C22B8F80C906C
:1011580098F80FA014F06DFF8F4B069318460021E6
:10116800142214F066FF8D4A0592002111708C49F3
:10117800C7F880110EF0C9FD059A8046002832D0C4
:10118800069B88491960884959608849D960B6F52D
:10119800807F87491961874B01D1002116E0BB2E5A
:1011A80001D9012112E0612E01D902210EE0292E78
:1011B80001D903210AE0132E01D9042106E0092EE2
:1011C80001D9052102E0002EE7D006211970042379
:1011D8001370794B02221A70784A136843F001039E
:1011E80013605B460EE003200AF09CFC40E24FF0DF
:1011F800010B0BFA03F140F2B2320A4042B1012B63
:101208005FD900236E490022092B0A70F9D8EEE74E
:1012180011F04D0FF3D0624A0593C7F880210EF004
:1012280074FD059B0028EAD0062168200A460DEBCC
:1012380000030EF017FA9DF86D1001EA0B029DF8F5
:101248006B1001EA0B0101FA0BF343EA82019DF8E6
:10125800692002EA0B030B430AD05BB25B4501D15C
:10126800002302E0022B0ED1012387F8843111E01C
:101278000EAB68200C215A460EF0F4F99DF8383070
:1012880013F00F0303D105200AF04CFC02E0042BF5
:10129800EAD1E5E73F4B4B4A1A604B4A5A6097F848
:1012A8008421002A0CBF6F226E221A72444B04223A
:1012B8001A70414B03225A70404A136843F00203E4
:1012C8001360042D00F2D080DFE815F00500EB0074
:1012D8009800050098000A200AF0B1FB7720A021A9
:1012E80001220EAB0EF0BEF9002800F087801E2107
:1012F800012277200EF032FA4FF42F600AF094FBA7
:101308004FF0000BABF160010025C9B202221AAB05
:1013180077208DF868508DF869500EF0A3F99DF884
:1013280068209DF86930294943EA022301F5C37210
:101338002BF802300BF1020BBBF1100FE2D1B1F820
:10134800942102F00F0E02F47F42A1F894210120AB
:101358002B462946DFF874C021F001056544B5F82D
:101368008651002D18BF002011F0010F03D0EDB2F7
:101378006B4008252CE083EA1523FAE700010050AA
:10138800202C002078240020AA2D0020404B4C005F
:1013980048100020802800202C2100204021002017
:1013A800E4830108EDFB00085DFA0008DDFA000897
:1013B80090C1793D00000020880000200C11002019
:1013C8002C34002065FC00089DFA0008000100206C
:1013D80013F4004F18BF83F4C053013D4FEA430391
:1013E800F6D101311029B5D16E4942EA0E02A1F8B1
:1013F800942118B9C3F303339E4538D0694D95F845
:1014080096B1BBF1000F40F0C68614200AF017FB16
:1014180005F297137620D02101220EF023F995F8D2
:101428009731582B3DD105F5CC73882118227620A9
:101438000EF018F931227620F4210EF08FF90123ED
:1014480085F89631584B594A9A60594A5A6045F678
:10145800D8125A80574ADA60574A1A61574AA3F88D
:1014680000B05A6100F097BE012D13D119E04E4B20
:1014780042F210721A805A80514A5A60514A9A6050
:10148800514ADA60514A1A61514A5A61B8F1000F5B
:10149800B4D003254F4B504A9D70136843F00403A2
:1014A80013604D4D2B689B0702D54C4B1B68984722
:1014B8004B4ABAF1000F25D016F0FF0F0AD12B685E
:1014C80013F0020F4FF07D0140F2712308BF4FF473
:1014D800FA7302E04FF47A731946994505DBB9F5BA
:1014E8007A6FA8BF4FF47A6900E099464B1E4B44C7
:1014F800B3FBF1F3013BDBB203FB011187F8B43115
:10150800116004E0274BC2F8009083F8B4A1354B72
:101518001B689847344A0023022C1370914604D064
:10152800032C20D0002C40F039862EAB002203F883
:10153800502D2E4AC7F8B8211E200A2101220EF08C
:1015480091F880B19DF86830482B0CD1284B294A76
:101558001A60294A5A60B8F1000F04D0042389F8A8
:10156800003002234EE02EAB002603F8506D0C200D
:10157800314601220EF076F880B19DF86830482B8C
:1015880040F042861A4B1D4A1A601D4A5A60464668
:10159800B8F1000F00F03886032333E0064600F068
:1015A80033BE00BF0001002070060020F9A100082A
:1015B800FBA10008CBA3000869A40008FB9F000852
:1015C8000BFA00084DFA000801FA00083DFA000875
:1015D80041F80008880000200C1100208028002015
:1015E800A82800202C21002028340020FC83010892
:1015F8004C060020D9A50008D5A3000841A500087D
:10160800B5A40008B84AD3702B6843F008032B60D0
:10161800B64B93F858210AB1B5490A7093F8592185
:101628000AB1B4490A7093F85A310BB189F80030FD
:101638002B68B14913F0080F00F0B685BDF910000A
:10164800DFEDAE6A642290FBF2F302FB130212B2E2
:1016580007EE902AB8EEE77A07EE903AF8EEE77AC6
:10166800E7EE267AB2EE047A67EE877AC1ED007A61
:10167800A34A137843F002031370A24B08229A611D
:101688000A24A04DAB8A9BB283F00803AB821920D1
:101698000AF0D5F901200AF0F1F919200AF0CFF97A
:1016A800013C00200AF0EAF914F0FF04E9D108230C
:1016B800AB61954B1A6812F0080F984605D0934B0A
:1016C8001B689847924B01221A70924B9FED928AA1
:1016D8001B68924C1B7B00EE103AB8EEC00A20EE55
:1016E800080A09F099FD238807EE903AF8EEE77AA0
:1016F80027EE800A14F0ACFE894B9FED8A7A188099
:101708002388894C07EE903AF8EEE77A874BC7EEC4
:10171800277A2046FF211A229FED857AC7EE877A1D
:101728009FED847AC3ED007A834BD3ED047A834B23
:1017380067EE887A67EE877AC3ED007A14F079FC51
:1017480000222270D8F800207D4B012112F0020FF0
:1017580018BF617019701FBF032119700221A17091
:10176800550748BF1978204641BF4C1C1C700324FC
:10177800445412F00A0F0CD01A7804218154511CD9
:10178800C9B205244454D11C0232D2B219700621C0
:1017980081546C4D29688C0641BF1A78541C1C7002
:1017A800072448BF84540A0608D51A7809248454A3
:1017B800941C0132D2B21C700A2484544B4E7479A2
:1017C800082C01D00E2C04D11A78571C1F700B2737
:1017D80087541A7811F4803F4FF00C0E00F802E09D
:1017E80002F101071CBFDFF858E10232FFB21F7097
:1017F8001FBF8EF800204C4A4FF00E0E02F807E08B
:101808004A0741BF1A78571C1F70102748BF8754D2
:101818001A78571CFFB24FF0120E11F4806F1F7028
:1018280000F802E00ED096F81CE2BEF1000F09D0D5
:10183800DFF80CE102328EF800203B4A4FF0130E1D
:1018480002F807E01A7811F4007F4FF0140E00F840
:1018580002E002F101071CBFDFF8E4E00232FFB248
:101868001F701FBF8EF800202F4A4FF0150E02F888
:1018780007E0182C0DD11A7816278754571CFFB289
:101888004FF0170E00F807E0D71C0232D2B21F70D3
:1018980084540C0341BF1A78511C1970192348BF8E
:1018A800835400219822284814F0C3FB0AF0B3FFA0
:1018B800264B274A27491A6000234B800B7126497B
:1018C8000A60B6F8982190B2244921F81300013330
:1018D800122BF9D12B68D8045CBFB6F89E0108809A
:1018E8001B0740F100813BE088000020202C0020ED
:1018F800402100202C340020701A00208988883C60
:1019080000340020000400480C1100204C06002080
:1019180064060020D421002035FA8E3C20000020E7
:10192800F02100200AE81C4111100020880700203F
:1019380000401C46BD3786352C210020D0210020D0
:1019480010100020FC27002070220020E40E002048
:10195800AA2D0020340E0020142C00203828002046
:1019680096F89241062C00F2B880DFE804F00407EC
:101978000E3D5878780045F2F05201E042F6F82220
:10198800804B1A800AF0E4FFA6E007EE902ADFED0C
:101998007E6A7C4BB8EEE77ADFED7C7AE7EE267A52
:1019A80042F6F82119800023FCEEE77A784A17EE10
:1019B800901A42F823100133122BF7D1754A764951
:1019C8001160764A4020137006F0BCF8002800F039
:1019D800848001234FF0070990F90000704A8DE8D0
:1019E800080240216F4B72E0664B42F6F8221A80DB
:1019F800684B6D4A1A60694B102240201A7006F035
:101A0800A1F8002869D001234FF0000C90F90000DC
:101A1800664A8DE8081040214FF4E13357E0594BEE
:101A280042F6F8221A805B4B614A1A605B4B082227
:101A380040201A7006F086F800284ED001234FF097
:101A4800000E90F900005B4A8DE8084040214FF4F1
:101A5800E13305F04DFF584BC3F8BC0139E0494B61
:101A680056485749DFF888C1DFF888E142F6F8227E
:101A78001A804A4B534A0C271F70062C4FF000035C
:101A880003700B7013700AD01B238CF800304E4B78
:101A98008EF8007005221A704FF4E13407E0212314
:101AA8008CF80030484B8EF800701C70474C394B4E
:101AB800474A1A60402006F045F870B10123002714
:101AC800444A90F9000040218DE88800234605F03B
:101AD8000FFF003018BF012028B9082009F060FC6A
:101AE8002C4B3D4A1A602B682C4A13F4804F1FBFB9
:101AF800082111702749394818BF086042F20101CE
:101B0800194003F0010003F4005479B11D4944F66B
:101B180020670F8024B1082111701E49304C0C60D9
:101B280020B10C2111701B492E4808601178180645
:101B3800A1F10401517040F196801F482A4CDFF84A
:101B4800B890C0F8C09100273946152200F5E27018
:101B5800DFF8A8A067706760A76014F06AFAA9F1B7
:101B680005033846CAF8003006F090FB1F4B0220E8
:101B78001B68E36005F0E6FF002841D1802009F0EA
:101B88000FFC68E0E8070020CDCCCC3F0000B0C4D3
:101B9800242B00203C000020B52A01080C2300203B
:101BA8005D2C0108A0860100A12A0108B12B0108BB
:101BB8008D2A0108652B010800010020102C002047
:101BC80049220020482200206C22002090D00300E7
:101BD800F9C600080DC70008152B0108E92A0108F5
:101BE800052B0108F52A0108A40700202028002059
:101BF8006B2200200F2C0020102E0020C40700208C
:101C080047796378CE490C2202FB03125278BA4214
:101C180004D00133DBB2042BF4D900236370DAF863
:101C2800003062781B7890F90000002B4FF00C030D
:101C380003FB021314BF0327012700225B780097D8
:101C48000192022105F054FEBE4B1860002895D081
:101C5800012006F01BFBBC4B1868BC4B00F5C57295
:101C68001A6006F0C1FB2B6813F4007F1AAF59D035
:101C7800B74C039B2360B74BB7485A6942F480229C
:101C88005A619A6942F001029A61039B1B88ADF878
:101C980030304FF0010902230CA98DF833308DF84C
:101CA80032900DF0C9FB2368AB485B88ADF8303043
:101CB8004FF0000A0CA98DF832A00DF0BDFB236887
:101CC8004846197A0AF070FF236858680AF0BCFE83
:101CD80023685B681A93384610238DF86D308DF8A9
:101CE8006CA08DF86E900FF095FA23685B7A8DF8EA
:101CF80038300EA803238DF839308DF83AA08DF8C6
:101D08003B900FF069FA954B954A1B683C3B136072
:101D1800D8F8003043F01003C8F80030914B4FF06A
:101D2800FF321A60904A914B1360914ADFF8608243
:101D3800803313602B680024D90388F8004040F1F1
:101D4800BC800EF0B7F9DFF84CC2DFF808A2CDF876
:101D580014C040F22A334FF001091A466046214662
:101D6800049388F8009014F064F9DAF81420DFF886
:101D780028824FF0904042F40032CAF81420426A98
:101D880022F00F024262426A032142F006024262D6
:101D98004FF4807B02228DF835100CA98DF8342081
:101DA80003928DF83640CDF830B08DF837900BF0AF
:101DB80045F9DAF81810039A41F40061CAF81810C6
:101DC800B8F8001021F45C710904090CA8F8001097
:101DD8001D21C8F82C104046A8F828200EA9A8F8FC
:101DE80030406022C8F814900E92ADF83E4010942E
:101DF800ADF84440ADF84640ADF84840ADF84A402B
:101E0800ADF83C900AF06AFFD8F8182042F00802B2
:101E1800C8F81820D8F8442042F40042C8F84420F2
:101E2800DAF8142042EA0902CAF81420AAF6E47A79
:101E380050460AF040FE38460AF012FE049B4D4A0E
:101E4800ADF874308023DDF814C01A923946102298
:101E58001F9350464FF40053CDF86CC01C92239347
:101E68001E94CDF880B02194229424940AF005FEA3
:101E7800D8F80C3043F40073C8F80C30DAF80030A6
:101E880043F00203CAF800300BA80C238DF82C305D
:101E98008DF82D908DF82E408DF82F900FF09CF92D
:101EA8002146354B1A68354B43F82120013120294A
:101EB800F7D10DF0E3F90DF0E1F92B685A0540F17F
:101EC80090802F4C2F4BD4F80495C3F80090042031
:101ED80005F038FE0421C4F8080505F00FFE2A4B6A
:101EE80084F80C050820C3F8009005F02BFE274B5A
:101EF800DFF8A8801860082105F000FE002184F8AA
:101F08000D052C22404614F094F88E2388F80130F1
:101F18004FF07C0BE0234FF07D0A88F8033088F8F7
:101F280000B088F82BA0DFF878802C2200214046EA
:101F380014F07FF88A2388F801301020A02331E0BC
:101F4800988401087424002048100020380F0020CD
:101F5800A0070020001002400004004820280020AC
:101F68009C07002068100020E01100204C2E002063
:101F7800B8240020342C014014840108AA0D002044
:101F8800000100200011002058110020A411002099
:101F9800A90D0020D9020020002C014028110020A2
:101FA8005D11002088F8033088F800B088F82BA06D
:101FB800C4F8109505F0C6FD1021C4F8140505F005
:101FC8009DFD84F818052020C4F81C9505F0BAFD7D
:101FD8002021C4F8200505F091FD84F824050BF0B4
:101FE8001FFD8D4A138823F040031B041B0C13802C
:101FF800138823F038031B041B0C138013889BB22F
:1020080043F04003138000249F2332208DF838309A
:102018008DF839408DF83A408DF83B4009F00FFDB6
:102028008DF869407D4C4FF480580422A4F828802C
:1020380038460EA90FF09AF8C4F818809DF86A205F
:102048009DF86930120242EA03429DF86B301A4348
:10205800734B9A42734B17D008D873498A420CD0F5
:1020680001F51A4102318A4209D01CE06F498A42BF
:1020780005D001318A4207D015E0202200E08022F5
:102088001A804FF4807202E04FF480721A805A80EE
:102098009A88198812029A604A43DA60644A0121D0
:1020A80082F8251504E000221A805A809A60DA60C6
:1020B800DC680CB3240CA1464FF0000AA24514DAE0
:1020C8000AEB04084FEA68084FEA0840394610222C
:1020D80008F074FC002357F82320013268D101333B
:1020E800042BF8D1C1464446E8E706F049FB504BBB
:1020F8004FEA0942C3F828252B684E4A13F40023F7
:1021080018BF0123137009F073FC4B4B18607379E7
:10211800052B02BF494B4FF4C8721A80484B4FF445
:102128007A721A80474BC8221A80474A137843F0BC
:1021380008031370454A137823F0020313702A68C2
:1021480040F6020313406BB1414B42491960424BC0
:1021580003211970414B01211970414900230B805B
:1021680040490B80930341BF3F4B04221A71DA7830
:1021780044BF42F00102DA70B3682B603B4B012286
:102188001A703B4A137863F07F0313702FB0BDECCD
:10219800028BBDE8F08F0425FFF77CB9012C7FF690
:1021A80037AA1C46FFF7B6B900230B60FFF760BAE1
:1021B80008F1010AA04696E71BB207EE903ADFED58
:1021C8002D6AB8F95E312C4AF8EEE77A07EE103A34
:1021D80067EEA67AB8F96031CDED1A7A07EE903A33
:1021E800B8EEC77AF8EEE77A002127EE267A67EE8E
:1021F800A67A11701AA821498DED1B7ACDED1C7AAB
:1022080009F012F8FEF76EBF012C7FF601AA002430
:1022180089F80060FFF789B90038004000040048D9
:1022280018BA200010000020152020001740EF00E9
:1022380000010020A42800202C0E00209C21002052
:102248002634002020340020101100202A340020D9
:10225800F81000209C2D00205C1100208000002038
:10226800D80F0020DA0F002078240020A80D0020C5
:102278000034002035FA8E3C700000205C230020DA
:10228800874A2DE9F04F1368864C03F59C432033A9
:102298002DED028B2360A3880133A380824B19683C
:1022A80089B011F4804F0592019305D110F070FDAB
:1022B80010B9237B0133237300277C4BDFF804829A
:1022C8001E78FDB2AE4230D9D8F800307748072DD5
:1022D80098BF595D764B88BF29461B689847032DE0
:1022E8001ED8D8F8002005F10E0302EB8303998865
:1022F800DA88A8B14FF47A73401A5843531A90FBFE
:10230800F3F040F6C90300F57A70984205DC40F214
:10231800EE239842B8BF184601E040F6CA0080B2E2
:1023280004EB45050137E881C7E70F23277B84F8CD
:102338003230032594F83330B7FBF5F505EB450546
:102348007D1B029394F834300393D8F800A0DFF88B
:102358007CB1EBB204930025B54255DA5549029B8E
:1023680031F815904FEA450853B910F011FD28B11E
:10237800039B002B08BF4FF0000901E0DDF808902F
:10238800BAF81400484503D8BAF8160048450ED2E2
:10239800E8B210F0D3FC032D8146DFBF94F832E099
:1023A8000120A8402EEA0000D8BF84F8320010F0BF
:1023B800EFFC18B1404828F8009021E0049B94F8FD
:1023C8007E002BF8139028B9022F15D93549012022
:1023D80081F87E00BBF80210BBF800000844BBF887
:1023E80004100844354980B228F8010000B20321DE
:1023F80090FBF1F080B200E048462F4928F8010030
:1024080001350BF1060BA7E794F83250254BA5F1DF
:102418000F0EDEF1000545EB0E0584F898503DB12E
:102428009A8811B21429CCBF143A00229A800BE082
:1024380083F83350B54207DAE8B210F07FFC1E4B40
:1024480023F815000135F5E7019B1B68DF0405D566
:102458001B4B1B68DE0701D40FF012FF059B1968A0
:10246800184B1868837A9BB3013B134D027B35F8F0
:1024780013301AB1C3F53B6308339BB21BB2A3F503
:102488007A73B3F57A7FA8BF4FF47A7323EAE373BC
:1024980007EE903A9FED0C7AF8EEE77A51E000BF2C
:1024A80008340020300E0020FC2700200C230020D8
:1024B8003C0000203E0E002038280020B00E0020EE
:1024C8000C100020142C002000007A44660E002016
:1024D800019A1268150440D5D4F89C20AD4E8A1A8A
:1024E800002A3ADB01F59C422032C6F89C20AA4A11
:1024F800C07A5579A94A32F8152096F8A0500135C6
:1025080092B292FBF0F205F00F0086F8A00030447A
:1025180080F8A1201A46A248185C01330244102B07
:1025280092B2F8D112B292FBF3F31BB2642BA8BF9C
:10253800642323EAE37307EE903A9FED9A7AF8EE64
:10254800E77AC7EE877A984A9FED987A67EE877A96
:10255800FCEEE77A17EE903A1380019B944D1B68C6
:10256800DFF8708213F4807F7AD0924B994204D9B5
:10257800237A13B9874B01221A72B4F904E098F848
:102588000060844BBEF1140FCCBF4FF0000E4FF02B
:10259800010EC6F38006BEF1000F03D000279F721C
:1025A8005F7200E00327A07AD4F8B4B0D4F8B8C0BA
:1025B800B4F90490617AE3882A88032848D8DFE8C8
:1025C80000F0020E1B35BEF1000F02D02A80002257
:1025D8002AE0002E40F05A862A80A6723AE09CF83B
:1025E800000000EB8000814502DC2A8001221BE00C
:1025F80001206EB300F0D8BE3EB1BBF80E206A8051
:10260800AA80BCF80200E88002279CF800A09CF889
:102618000100504400EB8000814500F33A86002E0B
:1026280000F037862A800222A27213E02A80032251
:10263800A2726172E3807EB198F8003043F0020321
:1026480088F80030534B00225A720FF019FE03E04D
:102658002A80A0726172E38017B1384609F028FA1F
:10266800554EB6F8520110F0C5FB834668B910F014
:10267800E7F9524BC3F800B0C3F804B0C3F808B088
:102688004F4B00221A605A609A6098F800305A0737
:1026980036D5019B1B68DB0632D54A4B1B78DF0613
:1026A8002ED4494B1B7893B196F8DE31BBF1000F5D
:1026B80015D17BB1454B1A68D4F8BC309B1A002B56
:1026C80008DA0FF0DDFD334B83F8C0B018E0BBF13A
:1026D800000F0DD1102009F0EBF901230EE03BB1FA
:1026E8003A4A12684FF47A7101FB0323C4F8BC30EC
:1026F80094F8C03023B109F0C7F9002384F8C0303A
:10270800002296F8DCA196F8DD11B6F89A71B6F8B1
:102718009CE1134635F912009B08B842C4BF63F028
:102728007F03DBB201327045B8BF43F04003042A8F
:10273800F0D194F8C12017489A4205D190F8C220E8
:10274800F92A04D8013200E0002280F8C22084F877
:10275800C1301D4B0F4A18781D4F994600283ED1AD
:102768003B68D80709D5BBF1000F38D198F800307D
:10277800DB0734D50FF0E6FB31E098F80030580756
:102788002DD592F8333053B3537A43BB21B30FF0AE
:1027980077FD24E0300E00208023002090230020C5
:1027A800D10E00200000C8426C10002000C07F44F9
:1027B80038280020404B4C00202C0020A019002075
:1027C8005C1A0020101100200C0000202028002096
:1027D8000C1000202A340020BBF1000FD7D094F849
:1027E800C2307C4ADFF818B2142B40F0928099F876
:1027F80000301AF1000A18BF4FF0010A7BB392F8B3
:10280800C1305F2B12D198F8003003F0040303F0B5
:10281800FF0113B10FF034FD08E00B200391029281
:1028280009F046F9029A039982F8C210BAF1000F2A
:1028380015D094F8C1307D2B11D198F8003003F0F1
:10284800040303F0FF0213B10FF01AFD07E00B2099
:10285800029209F02DF95F4B029A83F8C22098F88A
:10286800003003F0040303F0FF01002B51D194F86A
:10287800C130584A572B16D1574B4FF47A721A80E9
:10288800019B1B68190601D505F010FE534B1B6808
:102898005A0742BF524A0A21118013F0080338D15F
:1028A800504A138035E001980068400716D55A2B26
:1028B80014D14D4B187820B119704C4B01221A7065
:1028C80027E092F8C33083F0010382F8C3300BB1DC
:1028D8000C2000E00D2009F0EBF81AE05D2B00F069
:1028E800DB845B2B00F0F8845E2B02D1032000F020
:1028F800F4BC562B01D108F0E3FF99F80030002B07
:1029080000F0008594F8C1306F2B40F0F5840FF08B
:1029180019FB019B1B68580733D594F8C330A3B142
:1029280098F80030590710D5B5F90620B6F89A314D
:102938009A420ADD3B6813F0010301BF2C4A322199
:102948001180244A08BF82F8C3303B68DA030AD5ED
:10295800284B1A782AB9244A127812B9244A322103
:10296800118001220CE0204A137853B198F8003006
:1029780003F0040303F0FF011BB91C4B1170012283
:102988001A70DBF8009000233B6009F17B0609F11F
:10299800CB0A3278737816F8010C9A420BD231467A
:1029A80008F0C6FF38B116F8022C012303FA02F228
:1029B8003B6813433B6004365645EAD10E4B1B78FF
:1029C80003B30E4E054F336813F0020F40F04183F6
:1029D80039E300BF300E0020263400200C110020FF
:1029E80020340020E8100020C9210020CA2100203E
:1029F800B0210020C82100202D3400200C10002018
:102A08004810002009F1CA0609F5897732787378E9
:102A180016F8010C9A4225D2314608F089FF08B30E
:102A2800B37896F804E0C04A96F80390BF480C21A2
:102A3800013B01FB0E4103EB43031344D1F8C820CB
:102A48009A420FD0C1F8C830002390F8F420C1F89A
:102A5800CC30012303FA0EF322EA030381F8C49071
:102A680080F8F4300636BE42D0D1B14BDFF8CCB294
:102A78001E68B04B1B68039394F83330049300230B
:102A88000293DBF80030002B00F0D48293F800901A
:102A9800B9F1000F00F0CE82DBF8042003998A1AFE
:102AA800002A0CDB01F5FA720299CBF80420012206
:102AB8008A4094F8F41021EA020284F8F420049A77
:102AC800002A00F0B7821BF8042C59780432D2B2DD
:102AD800002940F0718235F91210974A934FB2F8E5
:102AE800982102F1C800814202DD93F802A015E0A6
:102AF800C83A914203DA9978C1F1000A0EE0029AC5
:102B08000123934097F8F42022EA030387F8F4306E
:102B1800039B03F5FA73CBF804308BE297F8F43093
:102B2800029A1341DB0700F18582BAF1000FCCBF8E
:102B38000220012008F0DEFF09F1FF33132B00F219
:102B48007082DFE813F0140021002F0043005C00BE
:102B58006300CA004001A701D70107026E024300C3
:102B680052006300CA0040019A00120177013778C9
:102B78005744FA2FA8BFFA2727EAE7773046377075
:102B880008F0BCFE01200BE077785744642FA8BFFB
:102B9800642727EAE7773046777008F0AFFE02200F
:102BA8003946D4E196F80390D144B9F1640FA8BF2F
:102BB8004FF0640929EAE97986F803903046D7F896
:102BC800F81004F0C5FF03204946C0E1717951446B
:102BD8006429A8BF642121EAE17171710D2008F010
:102BE800F3FEB9F10D0F00F01C82317951446429CC
:102BF800A8BF642121EAE17131710E20A7E1B17902
:102C0800514481F30801B1710520A0E1D7F8FC30E7
:102C18001A78022A22D107EE90AAF8EEE77AB2EEE5
:102C2800040A87EE800AD3ED097A30EE270AB5EE5A
:102C3800C00AF1EE10FA09D4DFED427AB4EE670A61
:102C4800F1EE10FAC8BFB0EE670A01E09FED3E0A48
:102C580083ED090A0F2008F0A2FE0AE09978514492
:102C6800C829A8BFC82121EAE17199700F2008F08E
:102C7800ABFEB9F10F0F00F0D481D7F8FC301A7809
:102C8800022A20D107EE90AAB8EEE78AB2EE040A2B
:102C980088EE008A93ED080A38EE000AB5EEC00AFD
:102CA800F1EE10FA09D4DFED277AB4EE670AF1EEF7
:102CB80010FAC8BFB0EE670A01E09FED230A83ED62
:102CC800080A12206BE159785144C829A8BFC821C5
:102CD80021EAE1715970122039E1D7F8FC301A78ED
:102CE800022A33D107EE90AAB8EEE70ADFED157A8B
:102CF80093ED0C7A80EE270A30EE070AB5EEC00A8B
:102D0800F1EE10FA07D4B4EE670AF1EE10FAC8BF74
:102D1800B0EE670A01E09FED0C0A83ED0C0A102063
:102D280008F03DFE1DE000BF90880108300E00202D
:102D38007010002020280020202C0020F80E0020F1
:102D480000007A440000C84200000000197B51448A
:102D5800C829A8BFC82121EAE1711973102008F019
:102D680033FEB9F1100F00F05C81D7F8FC301A7807
:102D7800022A1ED107EE90AAB8EEE78A5FED0F7A15
:102D880093ED0B0A88EE278A38EE000AB5EEC00AE2
:102D9800F1EE10FA07D4B4EE670AF1EE10FAC8BFE4
:102DA800B0EE670A01E01FED180A83ED0B0A132045
:102DB800F5E0D97A5144C829A8BFC82121EAE171B0
:102DC800D9721320C3E0D7F8FC301A78022A22D12E
:102DD80007EE90AA1FED260AF8EEE77A87EE800A3A
:102DE800D3ED0F7A30EE270AB5EEC00AF1EE10FAED
:102DF80009D45FED2C7AB4EE670AF1EE10FAC8BF79
:102E0800B0EE670A01E01FED300A83ED0F0A1120CA
:102E180008F0C5FD0AE0997D5144C829A8BFC8211A
:102E280021EAE1719975112008F0CEFDB9F1110F71
:102E380000F0F780D7F8FC301A78022A20D107EE84
:102E480090AA1FED410AB8EEE78A88EE008A93ED52
:102E58000E0A38EE000AB5EEC00AF1EE10FA09D4EF
:102E68005FED487AB4EE670AF1EE10FAC8BFB0EE2B
:102E7800670A01E01FED4C0A83ED0E0A14208EE06C
:102E8800597D5144C829A8BFC82121EAE171597563
:102E980014205CE0D7F8FC301A78022A20D107EE1B
:102EA80090AAB8EEE78AB2EE040A88EE008A93ED9B
:102EB8000A0A38EE000AB5EEC00AF1EE10FA09D493
:102EC8005FED607AB4EE670AF1EE10FAC8BFB0EEB3
:102ED800670A01E01FED640A83ED0A0A09205EE033
:102EE800D9785144C829A8BFC82121EAE171D9700D
:102EF80009202CE0D7F8FC301A78022A1ED107EEF8
:102F080090AAB8EEE78A5FED717A93ED0D0A88EE24
:102F1800278A38EE000AB5EEC00AF1EE10FA07D497
:102F2800B4EE670AF1EE10FAC8BFB0EE670A01E026
:102F38001FED7B0A83ED0D0A0A2030E0597B5144CE
:102F4800C829A8BFC82121EAE17159730A2008F0ED
:102F58003BFD66E0D7F8FC301A78022A22D107EE4A
:102F680090AA1FED890AB8EEE78A88EE008A93EDE9
:102F7800100A38EE000AB5EEC00AF1EE10FA09D4CC
:102F88005FED907AB4EE670AF1EE10FAC8BFB0EEC2
:102F9800670A01E01FED940A83ED100A0B2008F080
:102FA800FEFC3EE0D97D5144C829A8BFC82121EACA
:102FB800E171D9750B20CAE7012932D1987835F922
:102FC8001230B3F5617F05DB40F633029342A8BFA8
:102FD800134601E04FF46173B9F10C0F21D14FF49E
:102FE800966292FBF0F0AD4AA3F5617393FBF0F3A0
:102FF800DFB21378BB4214D0042F34BF3B46022300
:103008001370A74A09FB0323A64A0633136008F086
:1030180097FA4846394608F0D7FC781CC0B208F041
:1030280069FDA149029A0123934091F8F4201343C2
:1030380081F8F430029B0133042B02930BF10C0B43
:103048007FF41FADBDE4019B1B68DD050FD5637AD6
:103058006BB13B6898070AD5944B1B8813F00105A0
:103068000AD10FF0EDFC012008F08AF904E00120F4
:1030780008F075F9012300E00023326851070DD5E7
:1030880063B1012008F06BF9884B1B889A0708D4B4
:103098000FF0D6FC022008F073F902E0022008F0D5
:1030A8005EF93B6813F00A0F26D03368DB060BD5B0
:1030B8007E4B1B885D070AD4042008F061F97C4B1D
:1030C8001B88A4F8003102E0042008F048F93368AE
:1030D800980607D5754B1B88590606D4402008F07A
:1030E8004FF902E0402008F03AF933685A0642BF27
:1030F8006F4B1B88A4F802313B689B0608D43368E1
:103108001F0540F18F804FF4807008F039F98DE089
:10311800684B664F1B7813F0020F50D0664B1B7834
:10312800042B4CD93368DFF8809113F4007A0ED061
:103138003B88DD0637D4102008F022F9202008F05B
:103148000EF95E48011D05F005F9022327E03D88C8
:1031580005F01005ADB22DB1102008F000F90125D9
:1031680089F804A13368580512D5D9F808315449AB
:103178005A89B1F90030002BB8BF5B42934207DA95
:10318800B1F90230002BB8BF5B429342C0F2128102
:103198003B88990608D5202008F0E1F8002389F833
:1031A8000431012500E0002594F80C31B3B90E2054
:1031B80008F07EFC3C4B012283F80C210EE03B8892
:1031C80003F03003002B9AD0102008F0C8F8202014
:1031D80008F0C5F8002384F8043101E0002D8ED0F2
:1031E800384B002003F1280503F15004364A00212A
:1031F80022F81010354A596022F81010043269601C
:1032080022F8101000221A609A602A60AA602260D0
:103218006160A26014331435143400287FF46FAF52
:103228000120E3E74FF4807008F099F8284B5A79A9
:10323800082A1C4601D00E2A02D1402008F08FF837
:10324800019B1B685A0540F1CA8094F81C3223B9C7
:1032580098F8003013F0040F02E0336813F4002FDD
:103268000BD01C4B00221A703C2009F0B9FB002837
:1032780000F0B5800EF088FBF6E70AF0D1FB09B044
:10328800BDEC028BBDE8F04F09F0C5BA0120FFF78D
:1032980094B90320FFF791B901201EE060280020AF
:1032A800D033002070100020300E0020D4110020F0
:1032B800E8100020101100201611002078100020BE
:1032C800F0100020400F002022340020B80F00200A
:1032D800202C00201123002002205FFA80F909F138
:1032E800FF3386F8B43708F095F808F04DF94846EA
:1032F80008F000FCFFF70DBBBAF1000F02D07E2BDF
:103308003FF405AB94F8C130972B05D1364B4FF4F9
:10331800C8721A80FFF7FDBAA72B06D1334A137873
:1033280043F004031370FFF7F4BA0022BB2B079293
:1033380001D1022303E0B72B04D14FF6FE73ADF899
:103348001E3009E0BE2B01D1022303E0BD2B1AD1A8
:103358004FF6FE73ADF81C30DBF80030BDF81C10DA
:10336800B3F858200A44A3F85820BDF81E10B3F843
:103378005A200A44A3F85A2008F0A2FA002384F835
:10338800C230FFF7C6BA792B04D1194AD37823F093
:10339800010306E07A2B7FF4BCAA154AD37843F0E0
:1033A8000103D370FFF7B5BA013301469BB202207F
:1033B800FFF703B93B889B063FF5F6AE202007F0E0
:1033C800DFFF0C480C4B011D1A685B684360026004
:1033D80004F0C0FF094B012583F80451E4E609B065
:1033E800BDEC028BBDE8F08F9C210020101100205D
:1033F800782400208010002018110020300E0020B2
:103408002DE9F04FC14BB3F90610C14B2DED028BDE
:103418001F687A8989B0914201930EDBB1F5FA6F82
:10342800FC79BDBF8B1A6343A2F5FA64C4F1640446
:10343800BCBF93FBF4F4643400E06424B54AB64B93
:10344800B2F898A192F962211868049092B2059294
:10345800054600220293AD4B33F912300393CAEBB1
:10346800030303F2F31640F2E63086424FEA420BBA
:1034780003D8002BB8BF5B4201E04FF4FA73022A6D
:10348800049E4FF064002FD096F811E1BEF1000FB2
:1034980004D07345CCBFCEEB03030023DFF8C0E2B2
:1034A80093FBF0FC6FF063093EF81C809B4E09FB10
:1034B8000C390CF1010C3EF91CE00FFA88FCCCEB3E
:1034C8000E0E0EFB09FE9EFBF0FEC64426F80BE02E
:1034D800BE1836797343924E93FBF6F364339BB26E
:1034E800634393FBF0F02EE096F812E1BEF1000F73
:1034F80004D07345CCBFCEEB03030023DFF84C8226
:1035080093FBF0F06FF0630C0CFB003938F910E016
:103518000130002B38F91000CEEB000000FB09F950
:10352800BDF8140099FBFCF9CEEB090919FB00F969
:103538007A48A0F80490B879B8BF5B42434378480A
:1035480093FBF0F064306B78764E4FF0640E434393
:1035580093FBFEF3B354744EEB7A434393FBFEF3B1
:10356800B3546B7D6D4E5843704B90FBFEF0022AAE
:1035780098546F4B0FD183F802E0039B53450EDB41
:10358800644CB4F89A21914215DBB1F5FA6FA8BFE3
:103598004FF4FA6110E09C54039B534504DA36F863
:1035A8000B305B4226F80B300132032A05F1010586
:1035B8007FF451AFE4E71146891A4FF47A73DFF8C4
:1035C800A4E1564D59436FF06303C2F5FA626427CC
:1035D800B1FBF2F191FBF7F23EF8120003FB021186
:1035E800013203B23EF91220D21A514391FBF7F38C
:1035F8000344F3804F4B1B88580635D54E4B4F4A32
:103608001B881288DFED4E7A9B1A1BB208EE103A1F
:10361800B8EEC88A28EE278AB0EE480A07F0FCFD03
:10362800F0EE408AB0EE480A07F093FDB5F9023093
:1036380006EE903AB5F90030F8EEE66A07EE903AF1
:1036480020EE667AF8EEE77AA7EEA87A67EE807A37
:10365800BDEEC77AE6EEA87A17EE103AFDEEE77AE5
:103668002B8017EE903A6B80364D2B68990740F106
:10367800A180354B354F1A687B6945F20721D31A6B
:103688008B4240F397807A6109F0EEFD304BDFF80A
:10369800D8901A78032A9846B9F8003022D10A2B14
:1036A8002AD90023282088F8003008F0C8F909F042
:1036B800DBFD284B188809F0C1FD274B1A68D37821
:1036C80090FBF3F001300828244BA8BF082018709D
:1036D800537980B213FB00F33B83137913FB00F09B
:1036E800788309E00A2B07D803231C4A88F800309E
:1036F800002313703B837B8398F80030144A012B16
:103708003DD033D3022B4CD054E000BF38280020E2
:1037180070100020202C002048100020F0100020FD
:103728000CFEFFFF1C1A0020CE0F0020341A0020C8
:1037380080190020D4110020E8100020320F00204A
:1037480035FA8E3CFC27002008340020C00F0020EA
:103758005C11002098230020F81000208000002031
:10376800341F0020E6110020FC1000203A8BB9F825
:1037780000309A421EDD012388F800300FE0B9F8C6
:1037880000107B8B8B4202DD022313700FE0A34BEA
:103798001B8B0133994202DD002313700AE00820D5
:1037A80006E07B8BB9F8002001339A42E3DC07205E
:1037B80008F07EF92D682A0576D5994B974F1A6837
:1037C800FB69C3EB020845F2072398456CDD954B6E
:1037D800B6F906B0D3F80090FA6199F80A30B4F84F
:1037E8005201914E012B4FF47A71ABF57A7B98FB1D
:1037F800F1F803D041D3022B20D040E08B4B386A3C
:103808005A7B8B4B33F812204FF0080E92B290FB84
:10381800FEF3C01A8318BA843B6240F6E44293FB75
:10382800FEF39BB25343B9F80820C2EB1333594354
:10383800B9F9063091FBF3F1316020E07D4BB9F81E
:1038480008A01B78C6F800A05B0718D50FF0D2FABD
:1038580020B915F0100F18BF4FF0000B32220BFBE8
:103868000BF393FBF2F3B9F906205B445A434FF488
:103878007A7392FBF3F3534400E000233360D7E9F3
:103888000A0133686C4A03FB08F84FF47A7398FB13
:10389800F3F810EB080041EBE8710023C7E90A01CF
:1038A8000FF0E2FA654B1860654E3368D90427D5E6
:1038B8002A0622D5634B1B789B071ED5624B1878C6
:1038C80004281AD90022614BD7180521951C4FF0FE
:1038D8000A0E122AD154E9B287F801E004D0B0EBFD
:1038E800510F2A46EFD800E014215A18322002F866
:1038F800010CFF225A540F2000E00A2008F0D8F8E3
:10390800534D2A68002A50D0524B534F18683968D3
:103918008142984649D8514BDFF84C911978526842
:10392800E1B94FF0010A83F800A0B9F80030D35C80
:1039380023B3504608F0A2F8494B83F800A00FF0D3
:1039480033FAB9F80030CBB92B681B78053B5345DF
:1039580014D808F04DF8434B18600FE04FF0000AF8
:1039680083F800A0B9F80030D35C3BB1504608F0AA
:1039780085F83B4B83F800A00FF016FA2A68B9F8CF
:10398800003052683848D25CFE2A01D100230BE08F
:10399800FF2A02D108F078F807E0D8F800500A2189
:1039A80011FB02523A6001330380224D2B785F07E6
:1039B80003D52E4B08221A8570E03268D0075CBF09
:1039C80043F001032B701F4B1B7819075EBF2B7840
:1039D80023F001032B70D30248BF2B78204A44BF41
:1039E80023F001032B70224B1B6813F0040F02D045
:1039F8002049098851B92049098809B19F0705D488
:103A08001E4B1B88003318BF0123CBB3022313704E
:103A18002B7823F001032B7037E000BFC00F002084
:103A280008340020F8100020041100208023002012
:103A3800902300202A340020407E05000811002031
:103A48000C10002010110020161100208C280020D6
:103A58005C1F002020280020541F0020501F002039
:103A6800182C0020602A0020581F0020000400485D
:103A78000C110020203400209C2100202634002036
:103A88002978CE0758BF0223137007F0B1FFB34B54
:103A98001B68C01A002801DB0FF086F909F0C0FF87
:103AA800AF4B03931E78002E00F0A880AD4F3B6803
:103AB800002B00F01D87386808F082F8002800F015
:103AC8001787A84BA84C186808F077F8092801D080
:103AD8003F2852D14FF000092668DFF8C8824D46CA
:103AE80036B1A248D8F80010324612F0EFFA10B9F1
:103AF800C14605B945469E4B08F110089845EFD3D5
:103B0800EDB1D5F800C0D9F8008023681CF803E0AF
:103B180018F80300704512D15A1C944958B92D2B36
:103B280009D8DFF844E2CEF800204FF0200E01F863
:103B380003E0885403E001F803E02260E5E7236826
:103B48000BB14D4510D08B480EF018F84D4507D8ED
:103B580055F8100B0EF012F809200EF007F8F5E7EB
:103B680085480EF00BF8002623689E42A3D27F4BAF
:103B7800985D0DF0FBFF0136F6E72368002B40F057
:103B88009C86042840F0D38678480AF0ABFD00F004
:103B9800AFBED8F80000DFF8F0A108F011F818B3AC
:103BA800DAF8000008F009F8D9F8003093F848204E
:103BB80083468ABB242868D1012283F84820D9F893
:103BC8000030DFF8C0A193F848B0BBF1060FE0D190
:103BD80093F8490000F03AFF002877D00DF022FF53
:103BE8003B68002283F84820644B93F83530002B5B
:103BF80040F051864C36982E00F07A86604BF218C9
:103C080092F84A100129F5D15E4FF3583A605E4A9E
:103C1800B94613609046BCE7012A04D14D2814BF69
:103C280000220222C9E7022A04D13C2814BF00223C
:103C38000322C2E7032A0AD140284FF000029FBF9F
:103C48001A71DA715871987198BF0422B5E7042A7D
:103C580008D19A7983F8490080EA020B83F806B004
:103C68000522AAE7052AAAD159791A7991429979A0
:103C780006D941409971511C1971134418729EE775
:103C880081420CBF0622002297E72B78590796D469
:103C98002328DAF800300CD103993C4801220A7035
:103CA800304A1360354A13630DF068FF32480DF04F
:103CB80065FF374B1B681B785B4501BF354B364AA0
:103CC8001A60364B04BF364ADA6078E7DAF8002023
:103CD80092F849304C2B00F0B58400F2B780352BB0
:103CE80000F08B8260D82B2B00F0848420D8252B01
:103CF80000F05C8404D8232B00F0448200F013BE4B
:103D0800272B00F05984292B40F00D860DF066FE14
:103D1800A4F882010DF062FEA4F884010DF054FEAF
:103D280084F886010DF05AFEA4F8880100F0AEBDB3
:103D38002F2B00F0278504D82D2B00F05F8400F08E
:103D4800F2BD312B00F03385332B40F0EC850DF0BC
:103D58003BFE84F8940100F099BD00BF1C2C0020A4
:103D68002D3400207C280020B42400208424002046
:103D78008094010877AA01087CAA0108C00F0020D6
:103D880070220020B4110020B8110020ACAA01084C
:103D980014230020FC9F0020EFBEADDE00ED00E004
:103DA8000400FA05A0920108412B00F0A58418D858
:103DB800392B00F00E8404D8372B00F0AA8400F0C9
:103DC800B2BD3C2B00F0CC803E2B40F0AC850DF012
:103DD800FBFD84F8DE010DF0F7FD84F8DD0100F04D
:103DE80055BD442B00F0178525D8432B40F09B8503
:103DF8000DF0EAFD0023A36060710DF0F9FD07F0F6
:103E0800D7FA0DF0E1FD84F892010DF0E7FDA4F872
:103E18005C010DF0E3FDA4F85E010DF0DFFDA4F8F0
:103E280060010DF0DBFDA4F882010DF0D7FDA4F8C8
:103E3800840100F02BBD482B00F04D834A2B40F045
:103E480072850DF0CBFDA08100F020BDD12B00F0D4
:103E58006C8320D8CC2B00F00F820FD8C82B62D0EF
:103E680004D84E2B00F01A8400F05DBDC92B00F079
:103E78003583CA2B00F0838000F055BDCE2B00F0AF
:103E88001D83C0F01283CF2B00F04A82D02B00F0A4
:103E9800018300F048BDD82B00F005810BD8D32B47
:103EA8003BD027D3D42B00F07F82D62B40F03B8524
:103EB8004FF000086DE2F22B00F0C48212D8EF2B0D
:103EC80040F03185DFF89083D8F800900DF086FD3A
:103ED800A9F85A00D8F800800DF080FDA8F858001D
:103EE80000F0D4BCF32B00F09B84FA2B00F0EF8297
:103EF80000F019BD2B7803F0040303F0FF08002B32
:103F080040F0C4840DF060FD022884F8B40740F244
:103F1800C782CD4B83F8B487C2E20DF05FFDCB4B6F
:103F2800188000F0B3BC92F805804FEA5808B8F141
:103F3800120F03D908F050FD00F0A8BC4FF000099B
:103F4800C14507D20DF04AFDC14B23F8190009F10C
:103F58000109F5E7BF4B012283F8342000F096BC35
:103F6800DFF8F482D8F800900DF02EFD89F80000F3
:103F7800D8F80030187805F0E5FF00F087BCB64B9C
:103F88001A681278022A4FF00009984670D1D8F8BA
:103F980000A00DF019FD07EE900AF8EE677AB2EE70
:103FA800048AC7EE887A0AEB890ACAED087AD8F833
:103FB80000A00DF009FD07EE900A9FEDA87AF8EE33
:103FC800677A0AEB890AC7EE877ACAED0B7AD8F8BE
:103FD80000A00DF0F9FC07EE900A9FEDA17AF8EE2B
:103FE800677A0AEB890AC7EE877A09F10109B9F1FC
:103FF800030FCAED0E7ACAD1B9F1070FD8F800A09D
:104008001CD10DF0E1FC07EE900AF8EE677AC7EED6
:10401800887ACAED117AD8F800A00DF0D5FC07EE21
:10402800900AF8EE677AC7EE887ACAED127AD8F85D
:1040380000A00DF0C9FC8AF84C0012E00DF0C4FC99
:10404800CA448AF80100D8F800A00DF0BDFCCA44A3
:104058008AF80B00D8F800A00DF0B6FCCA448AF81C
:10406800150009F10109B9F10A0FC5D100F00EBC1C
:10407800D8F800A00DF0A8FCCA448AF80100D8F8C6
:1040880000A00DF0A1FCCA448AF80B00D8F800A0E3
:104098000DF09AFCCA4409F10109B9F10A0F8AF82E
:1040A8001500E5D1F2E38146DFF8AC819FED6C8A1B
:1040B800D8F800A00DF092FC07EE900AF8EE677AA7
:1040C8000AEB890AC7EE887ACAED087AD8F800A000
:1040D8000DF084FC07EE900AF8EE677A0AEB890A7D
:1040E800C7EE887ACAED0B7AD8F800A00DF076FCF6
:1040F80007EE900AF8EE677A0AEB890AC7EE887A23
:1041080009F10109B9F1030FCAED0E7ACCD1B9F161
:10411800070FD8F800A01CD10DF060FC07EE900A3C
:10412800F8EE677AC7EE887ACAED117AD8F800A057
:104138000DF054FC07EE900AF8EE677AC7EE887A1D
:10414800CAED127AD8F800A00DF048FC8AF84C00A5
:1041580012E00DF043FCCA448AF80100D8F800A028
:104168000DF03CFCCA448AF80B00D8F800A00DF00A
:1041780035FCCA448AF8150009F10109B9F10A0F9A
:10418800C5D183E30DF020FC132882463FF6D2AE5A
:10419800DFF8C490D9F800B00DF016FC0023314ABE
:1041A8000C2101FB0322117A814222D10FFA8AF8ED
:1041B8000BEB8808137888F879300DF005FC88F83F
:1041C8007A000DF001FC88F87B000DF0FDFB264B12
:1041D800264A1A6088F87C00254BD9F80000186038
:1041E8000021793007F0CAFB224B80F001001870DB
:1041F8004CE301331B2BD2D19CE60DF0E5FB0B28D9
:1042080080463FF697AE144BD3F800900DF0DCFBD8
:1042180003283FF68FAE0BFB089B8BF8CE000DF002
:10422800D3FB8BF8C9000DF0CFFB8BF8CA000DF05B
:10423800CBFB8BF8CB000DF0C7FB8BF8CC000DF057
:10424800C3FB8BF8CD0021E3202C0020300F002089
:1042580038280020C00F0020481000200000C84265
:1042680000007A44FC880108280F0020642D0020F3
:104278002C0F00200C0000205379092B7FF65AAE32
:10428800019BD3F800800DF09FFB019B88F800008C
:10429800D3F800800DF098FB88F801000DF094FB2E
:1042A800019B64281B68A8BF642018710DF08CFB63
:1042B800019B64281B68A8BF642058710DF084FB1B
:1042C800019BFF281B68A8BFFF2098710DF07CFB9D
:1042D800019B6428D3F8008028BF642088F8070071
:1042E8000DF072FB019B88F80200D3F800800DF0F6
:1042F8006BFB019B88F80300D3F800800DF06EFB80
:10430800DAF80030A8F80A005B790A2B40F2BE827E
:10431800D34BD3F800800DF057FB88F80800B5E2BE
:104328000DF05CFB6FF4AF6283189BB2C62B98BF8D
:10433800A4F898010DF052FBA4F844010DF04EFBCF
:10434800A4F846010DF04AFBA4F848010DF046FB1D
:10435800A4F8DA010DF038FB84F8EB010DF034FB1A
:104368000DF032FB84F8EC010DF02EFB84F8870188
:104378000DF02AFB84F894010DF026FBB94BD3F815
:1043880000800DF02BFB00EB80004000A8F85600E1
:104398001FE10DF023FBB44B23F8180008F10108C6
:1043A800B8F1080FF5D171E253790F2B7FF4C2AD44
:1043B8000DF00AFB072880463FF6BCAD029BD3F8F8
:1043C80000900DF00BFB0E2303FB08F8C144029B81
:1043D800A9F81901D3F800900DF000FBC144029B25
:1043E800A9F81B01D3F800900DF0F8FAC144029B1C
:1043F800A9F81D01D3F800900DF0E6FAC144029B1C
:1044080089F81F01D3F800900DF0DEFAC144029B31
:1044180089F82001D3F800900DF0D6FAC144029B28
:1044280089F82101D3F800900DF0CEFAC144029B1F
:1044380089F82201D3F800900DF0DAFAC844C8F8D8
:10444800230123E20DF0C0FA0F2880463FF672AD33
:104458000DF0BAFAC8EBC808A04488F8D4000DF0EB
:10446800B3FA88F8D5000DF0AFFA88F8D6000DF049
:10447800ABFA88F8D7000DF0A7FA88F8D8000DF045
:10448800A3FA88F8D9000DF09FFA88F8DA0007F047
:1044980039FDFBE12B785B0700F1F8810CF004FA99
:1044A80006F0B8FF07F070F8F0E12B78580700F134
:1044B800ED816E4B4FF4C8721A80E7E12B785907EB
:1044C80000F1E4816A4A137843F004032BE02B7867
:1044D8005A07E5D527E204F091F9D7E10DF074FA0F
:1044E800634B1A7810B142F0020201E022F0020296
:1044F8001A700DF069FA5F4BDFF8988118700DF0AB
:1045080077FAC8F800000DF073FAC8F804000DF047
:1045180065FA594B18800DF061FA584B584A1880C3
:10452800137843F002031370B0E10DF04DFA83469F
:104538000DF05EFA82460DF05BFA81460DF058FAEE
:1045480080460DF04BFA0DF049FA0DF03DFABBF13B
:10455800000F14D14B4B1020C3F800A0C3F80490EF
:1045680006F0FDFE424A137843F001031370B8F1D8
:10457800000F00F08B81444BC3F8008086E1BBF14B
:10458800100F40F08381414BC3F800A0C3F804909A
:10459800B8F1000F02D03C4BC3F800803B483C4BBD
:1045A8000222011D1A7003F0D5FE6FE1A0600DF024
:1045B8001FFA06F0FDFE69E10DF010FAA4F85C019F
:1045C8000DF00CFAA4F85E010DF008FAA4F86001E9
:1045D8005CE10DF0F9F984F87C010DF0F5F984F847
:1045E80080010DF0F1F984F87F010DF0EDF984F800
:1045F80081014BE10DF0E8F9607147E10DF0E4F954
:1046080084F892010DF0EAF9A4F89C010DF0E6F99E
:10461800A4F898010DF0E2F9A4F89A010DF0D4F984
:104628003B6884F893015B79DFF86C80082B40F2D3
:104638002D810DF0D3F9A8F89E010DF0CFF9A8F857
:10464800A00123E10DF0C0F984F8D8010DF0BCF900
:1046580084F8D9010DF0C2F9A4F8DA0116E100BF17
:104668007010002048100020622800209C210020A3
:104678001011002016110020141100201211002022
:10468800761000207810002088100020801000206C
:10469800340F002018110020202C002092F80580EB
:1046A8000323B8FBF3F8B8F1120F3FF643ACDFF879
:1046B80098934FF0000AC24580F0E8800DF084F925
:1046C80089F8A2010DF08AF940F2ED23984205DD40
:1046D80040F6CA039842A8BF184601E040F2EE200F
:1046E800A0F2EE2019230AF1010A90FBF3F009F178
:1046F800020989F8A101DEE781460DF065F904EBAE
:10470800090309F10109B9F1080F83F88A01F4D105
:10471800BCE053794FF00709B3FBF9F9C9EBC902BB
:104728009B1A13F0FF0F7FF405AC5FFA89F909F1C2
:10473800FF395FFA89F9B9F1FF0F00F0A7800DF092
:1047480043F95FFA80FA4FFA8AF003F021F98046BC
:1047580000283FF4EFAB80F800A00DF03FF9A8F86F
:1047680002000DF031F988F804000DF02DF988F8F1
:1047780005000DF029F988F807000DF025F988F8EB
:104788000600D4E7DFF8C08208F140090DF026F9E9
:10479800A8F8AC020DF018F988F8AE020DF014F97B
:1047A80008F1040888F8AB02C845EFD16EE00DF0B7
:1047B8000BF91F2880463FF6BDAB3B685B79082B99
:1047C8007FF4B8AB0DF00AF908F18A0804EB880801
:1047D80000F03F00A8F806000DF000F9B8F8063020
:1047E800800100F4FE501843A8F806000DF0ECF81C
:1047F800000188F804000DF0E7F898F8043000F09C
:104808000F00184388F804000DF0DEF888F805005A
:104818000BF050FC3AE0794B012283F8352035E063
:104828000DF0D2F8FF2881461BD100238DF81F30E8
:104838009DF81F30072B29D89DF81F00704A9DF856
:104848001F3052F8300002EBC30301215B68994026
:1048580089B2042202F0AEFF9DF81F300133DBB2AB
:10486800E4E707283FF666AB00200DF0FFF80DF0EF
:10487800D9F8D8F8000007F09AF918B9322007F0EB
:10488800DEF8F6E74FFA89F002F0A2FF00200DF0FB
:10489800EDF8FFF7A3B95B4B985907F088F918B9F9
:1048A800322007F0CCF8F6E707F0ECFA06F088FDBE
:1048B800554B564ADA60FFF79DB90C2839D00A28BB
:1048C80040D1534D53480DF059F92846232111F092
:1048D800E6FB08B1401B20602368002B55D14C48EB
:1048E80023600021302211F0A4FB039B1B781BBB23
:1048F800494B1B689B060FD5484B40491B688A6B80
:104908009A1A002A08DB464A1278042A82BF03F55D
:10491800123303F5F8738B63424B9B68002B67D007
:104928004148984764E008F057F8FFF757B90C2852
:1049380004D13E480DF022F93D480DE07F2812D100
:10494800FFF7B9B80D28BCD07F2809D1013B304A00
:10495800384823600021D1540DF010F9FFF7ABB8A7
:104968002F2B3FF6A8A8A0F12002D2B25E2A3FF66C
:10497800A2A813B920283FF49EA85A1C2260244AF2
:10498800D0540DF0F3F8FFF796B85A1EA95C202909
:1049980001D11346A1E71E4A23600021D154264BBA
:1049A800264DD3F80090D5F800A0DFF86480504673
:1049B80011F083FB064632464046514611F086FB0D
:1049C8001F4A28B918F806304B445B78580703D0BB
:1049D80010359542E7D306E0954204D2701CEB6887
:1049E8004044984702E017480DF0C8F8002376E7DE
:1049F80009B0BDEC028BBDE8F08F00BFC00F0020EE
:104A080014AE01087022002000ED00E00400FA0551
:104A180084240020E8B901080C1100200834002083
:104A2800161100202C210020FC0F002081AA01086B
:104A38007CAA0108A8AA010890000020A0920108F9
:104A4800809401088CAA0108202C00202DE9F04749
:104A58002DED028B4B28A0B0044600F0438600F2EF
:104A6800B480302800F0CE8651D8222800F08D84FA
:104A780023D8032800F0608114D8012800F0508161
:104A8800022840F02A8704200CF0F0FF43200CF0A5
:104A9800B8FF4C200CF0B5FF46200CF0B2FF4C20BC
:104AA80000F055BE042800F05181052840F0158714
:104AB8001A200CF0DBFF002459E1282800F0E085DB
:104AC80015D8242800F0C785262840F00687B44C5E
:104AD80006200CF0CBFFB4F85C010CF0CAFFB4F868
:104AE8005E010CF0C6FFB4F8600100F0B1BD2C28DF
:104AF80000F0D9852E2800F055862A2840F0ED864A
:104B080001200CF0B3FFA64B587900F020BE3D28D9
:104B180000F016831ED8362800F02A860BD83228D3
:104B280000F00F86342840F0D88648200CF09EFF0D
:104B3800002500F04CBC3A2800F0B3823B2800F076
:104B48001D84382840F0C98604200CF08FFF944C4F
:104B580000F087BD452800F0AD8627D8402800F032
:104B6800F985422840F0B9868D4C10200CF07EFF64
:104B780060790CF046FFA0680CF084FF94F892016D
:104B88000CF03FFFB4F85C010CF073FFB4F85E0161
:104B98000CF06FFFB4F860010CF06BFFB4F8820101
:104BA8000CF067FFB4F8840100F052BD472800F00C
:104BB8005F86C0F04C86492840F08F8602200CF0B2
:104BC80055FF774B988900F043BD702800F0EB82C1
:104BD80058D8692800F045822AD8652800F0FA805C
:104BE80015D84D2800F08D85642840F0768607207A
:104BF8000CF03CFFE7200CF004FF694B58790CF0EF
:104C080000FF00200CF0FDFE042000F062BE6728C3
:104C180000F0AA8100F2188212200CF027FF614BE5
:104C28001B88B3F5806F8CBF0825012500247EE121
:104C38006C2800F0298217D86A2800F08D846B2828
:104C480040F04B8605200CF011FF574B18880CF0EC
:104C580010FF564B18880CF00CFF554B93F8760054
:104C680000F0010000F073BD6E28514D00F0208265
:104C780000F2718206200CF0F9FE686E0CF002FF5B
:104C88004C4B0CE2782800F07C8119D8742800F08D
:104C9800BF830BD8722800F01F84732840F01D864C
:104CA80008200CF0E3FE012400F04FBC762800F049
:104CB800738400F2F1832F200CF0D8FE3E4C55E3AC
:104CC800A42800F0918414D87B2800F0F582A0284D
:104CD80040F003860C200CF0C9FE384B18680CF025
:104CE800D1FE374B18680CF0CDFE364B186800F033
:104CF800F0BDF12800F08181FE2800F09C84F028A6
:104D080040F0EB852A4C04200CF0B0FEA36CB3F8FD
:104D18005A000CF0AEFEA36CB3F8580000F098BC33
:104D280003200CF0A3FE00200CF06BFE20460CF0D4
:104D380068FE0C2000F00BBD0CF098FE01200CF072
:104D480060FE0A200CF05DFE00F04CBC06200CF062
:104D58008DFE53200CF055FE52200CF052FE4620DA
:104D68000CF04FFE33200CF04CFE00F070BC164BDC
:104D7800185D01340CF045FE0B2CF8D10024134BC0
:104D8800185D01340CF03DFE082CF8D10024104BBE
:104D9800185D01340CF035FE072CF8D100F09BBDEE
:104DA800202C0020200000208A1100208C110020D7
:104DB80000100020E0100020CB880108ACF7FF1F8E
:104DC800B0F7FF1FB4F7FF1FA8A70108B4A7010891
:104DD80089A70108C94C0B200CF048FE20880CF06C
:104DE80048FE6268C64B9A420CBF2089608980B22F
:104DF8000CF03FFEC34B1B68C3F3C000C3F3800233
:104E0800800040EA4200C3F340021043C3F340125B
:104E180040EAC20003F0100318430CF02AFEBA4B14
:104E28001A88E36812F0010F14BF4FF0020C4FF01C
:104E3800000C12F0020F02F0080814BF4FF0040E25
:104E48004FF0000E03F4475912F0040F14BF102757
:104E5800002749EA080912F0400F03F4804814BFFC
:104E68002026002649EA080912F0100F03F400482A
:104E780014BF4FF40075002549EA080912F0200F05
:104E880003F4803814BF4FF48060002049EA080911
:104E980012F4807F03F4003814BF4FF4006100213E
:104EA80049EA080912F4007F03F48028974A49EA7E
:104EB800080903F4002849EA0809127803F480185D
:104EC80049EA080903F0007349EA0303C2F38002C0
:104ED80043EA020343EA0C0343EA0E0E4EEA0707CD
:104EE80046EA070645EA060540EA050041EA0001E8
:104EF80014BF4FF400184FF0000841EA08080020DA
:104F0800217C03468B420BD2814A9C5C012202FA27
:104F180004F414EA080F1CBF9A4010430133F1E768
:104F28000CF0B0FD7B4B93F8B40700F010BC7A4B43
:104F380033F9140090FBF5F0013480B20CF099FDC0
:104F4800032CF4D16D4CA08D0CF093FDE08D0CF08A
:104F580090FD208E0CF08DFD608E0CF08AFDA08EE9
:104F68000CF087FDE08E73E310200CF07FFD002429
:104F78006A4B185D01340CF044FD102CF8D100F098
:104F8800AABC70200CF072FD00265C4D0E24AB6CA0
:104F9800744323440136B3F819010CF06AFDAB6C75
:104FA8002344B3F81B010CF064FDAB6C2344B3F845
:104FB8001D010CF05EFDAB6C234493F81F010CF04F
:104FC80020FDAB6C234493F820010CF01AFDAB6C68
:104FD800234493F821010CF014FDAB6C234493F89F
:104FE80022010CF00EFDAB6C1C44D4F823010CF02C
:104FF80049FD082EC9D100F06EBC7020454C0CF05C
:1050080035FD04F1700594F8D4000CF0FAFC94F81E
:10501800D5000CF0F6FC94F8D6000CF0F2FC94F8ED
:10502800D7000CF0EEFC94F8D8000CF0EAFC94F8E9
:10503800D9000CF0E6FC073494F8D3000CF0E1FC3E
:10504800AC42E0D100F047BC10200CF00FFD00246A
:10505800334B185D01340CF0D4FC102CF8D100F05F
:105068003ABC304D2878400000F0FE000CF0FEFC01
:1050780000242B789C4280F02E842B4B33F81400AC
:105088000CF0F7FC0134F4E7284C06200CF0EEFC99
:1050980020880CF0EEFC60880CF0EBFC244B1888A0
:1050A800D6E204200CF0E2FC144B986E00F011BC20
:1050B80007200CF0DBFC1F4B1888FF28A8BFFF2037
:1050C800C0B20CF09EFC1C4B186880F3100080B234
:1050D8000CF0CFFCB5F86C000CF0CBFC0D4B93F842
:1050E8008721164B186822B10A23584380F3100011
:1050F80001E000F30F0080B2AAE200BF0010002018
:10510800005400400C110020D41100202A34002043
:1051180011100020202C0020DA1000203810002068
:105128004C1000200C23002038280020F4270020F1
:10513800E8100020FC1000200811002004110020B5
:10514800C44C02200CF092FC94F8DE010CF059FCDF
:1051580094F8DD01FBE20B200CF088FC2B6F18782B
:105168000CF04FFC2B6F58780CF04BFC00262B6F83
:10517800B94C3344013618790CF043FC032EF6D1B0
:10518800236FD8790CF03DFC236F98780CF039FC2C
:10519800236FD8780CF035FC236F58890CF069FC24
:1051A800236F187AD3E2AC4C1E200CF05FFCA36C82
:1051B8001B78022B4FF000056BD1A36C03EB850322
:1051C80093ED080AB2EE048A20EE080A11F040F9BD
:1051D80080F30800C0B20CF014FCA36CDFED9F7ADA
:1051E80003EB850393ED0B0A20EE270A11F030F943
:1051F80080F30800C0B20CF004FCA36CDFED987AD1
:1052080003EB850393ED0E0A20EE270A11F020F92F
:1052180080F30800C0B201350CF0F3FB032DCCD1AC
:10522800072DA36C23D193ED110A20EE080A11F083
:105238000FF980F30800C0B20CF0E3FBA36C93ED08
:10524800120A20EE080A11F003F980F30800C0B230
:105258000CF0D7FBA36C93F84C3000EE103AB8EE84
:10526800400A11F0F5F880F30800C0B20BE02B44B7
:1052780058780CF0C6FBA36C2B44D87A0CF0C1FB11
:10528800A36C2B44587D01350CF0BBFB0A2DC7D10C
:1052980021E3A36C2B4458780CF0B3FBA36C2B448C
:1052A800D87A0CF0AEFBA36C2B440135587D0CF07A
:1052B800A8FB0A2DEDD10EE33C200CF0D7FB00240F
:1052C800654D9FED678AAB6C03EB840393ED080A89
:1052D80020EE080A11F0BCF880B20CF0CAFBAB6CE7
:1052E80003EB840393ED0B0A20EE080A11F0B0F8E3
:1052F80080B20CF0BEFBAB6C03EB840393ED0E0A9B
:1053080020EE080A11F0A4F8013480B20CF0B1FBC9
:10531800032CD5D1072CAB6C16D193ED110A20EED6
:10532800080A11F095F880B20CF0A3FBAB6C93ED72
:10533800120A20EE080A11F08BF880B20CF099FBE3
:10534800AB6C93F84C000BE0234458780CF091FBBD
:10535800AB6C2344D87A0CF08CFBAB6C2344587D9F
:1053680001340CF086FB0A2CD4D1B4E214F8010FF6
:10537800002800F0B0820CF044FBF7E701200CF0A5
:1053880075FB354B9B6C1878E1E150200CF06EFBF7
:105398000025314B9C6C334B04EB85040C2194F8AD
:1053A800792001FB0233013593F838000CF029FB12
:1053B80094F87A000CF025FB94F87B000CF021FBA4
:1053C80094F87C000CF01DFB142DE2D183E2224BF3
:1053D8009C6C062303FB0544013594F8CE000CF0C1
:1053E80010FB94F8C9000CF00CFB94F8CA000CF000
:1053F80008FB94F8CB000CF004FB94F8CC000CF0FC
:1054080000FB94F8CD000CF0FCFA0C2DDFD162E221
:105418004FF00008012600270F4B1A7C974232DA1A
:1054280011330024FA5C0F4D0C2305F1300163435E
:10543800595C914207D12B44586B10F03EFE8246CE
:105448002EB9B14610E001341B2CECD119E0804490
:1054580017E000BF202C0020001000200000C842E8
:1054680000007A44CC880108D1450ADA0C2303FBF2
:1054780004535B6B13F809000CF0C3FA09F1010936
:10548800F2E70137C8E7002E00F025825FFA88F0BE
:105498000CF0ECFA0026BEE7CD4D287C0CF0E6FABD
:1054A80000242B7C9C4280F01682CA4BE65C0021CB
:1054B800C9480C2200F1300702FB01F3DA5DB24261
:1054C80005D1034493F838000CF09BFA02E001314F
:1054D8001B29EDD10134E4E7C04C16200CF0C6FAC4
:1054E800B4F898010CF0C5FAB4F844010CF0C1FA0C
:1054F800B4F846010CF0BDFAB4F848010CF0B9FA5A
:10550800B4F8DA010CF0B5FA94F8EB010CF079FA7A
:1055180000200CF076FA94F8EC010CF072FA94F88A
:1055280087010CF06EFA94F894010CF06AFA0020E6
:105538000CF067FAA64B9B6C0A20B3F9563093FB24
:10554800F0F080B20CF095FA8BE0E0B201340CF088
:1055580058FA092CF9D1BEE110200CF087FAA04BBB
:10556800A04C187800F002000CF04BFA9E4B18780B
:105578000CF047FA20680CF085FA60680CF082FAA3
:105588009A4B18880CF075FA994B18880CF071FA38
:105598008F4BB3F874005BE00CF016FA0746122044
:1055A8000CF064FA8A4C17B9A66FE56F07E0102F64
:1055B80013BF0025D4F88060D4F884502E463846AE
:1055C8000CF01FFA30460CF05DFA28460CF05AFA37
:1055D800D4F888000CF056FA00200CF04AFA0020A3
:1055E8000CF047FA0020B2E0794D95F88C00800065
:1055F8000130C0B20CF03AFA95F88C000CF001FAC0
:1056080000242E4696F88C309C4280F06481794DB7
:10561800285D0CF0F6F905F11003185D0CF0F1F9AE
:1056280005F120033035185D0CF0EBF9285D0CF01E
:10563800E8F90134E6E708200CF018FA00200CF02D
:1056480018FA00200CF015FA00200CF012FA0020CD
:105658000CF00FFA3FE104200CF008FA5F4B986851
:1056680037E194F87C010CF0CCF994F880010CF047
:10567800C8F994F87F010CF0C4F994F8810166E048
:10568800564C07200CF0F2F9B4F882010CF0F1F94D
:10569800B4F884010CF0EDF994F886010CF0B1F936
:1056A800B4F88801D4E74D4C0C200CF0DFF994F8DD
:1056B80092010CF0A6F9B4F89C010CF0DAF9B4F8F0
:1056C80098010CF0D6F9B4F89A010CF0D2F994F8D4
:1056D80093010CF096F9B4F89E010CF0CAF9B4F8ED
:1056E800A001B5E73D4C04200CF0C0F994F8D801AE
:1056F8000CF087F994F8D9010CF083F9B4F8DA01C1
:10570800A6E73D4C3D4D207800EB4000C0B20CF0C0
:10571800ADF9002623789E4205F1020580F0DB8072
:1057280015F8020C0CF06DF915F8010C00EB80006F
:1057380000EB800000F2EE2080B20CF09AF90136FE
:10574800E8E701200CF092F9244B93F894010CF04F
:1057580058F9C0E008200CF089F900241F4B2344B5
:10576800013493F88A010CF04CF9082CF6D1B2E018
:10577800174B1A4C93F8CD00C0EBC000C0B20CF028
:1057880075F904F1280594F8F20100231C4AD25C4B
:10579800904200F0A4800C333C2BF7D10834AC4283
:1057A800F1D198E040200D4C0CF060F904F140056F
:1057B800B4F8AC020CF05DF994F8AE020CF021F9E3
:1057C800043494F8AB020CF01CF9AC42F0D182E03E
:1057D8000010002011100020CC880108202C002087
:1057E800101100201811002016110020141100209B
:1057F800121100208D1000200C230020C22D002043
:1058080018230020E020444C0CF030F904F1800506
:10581800B4F82E0200F03F000CF02BF9B4F82E0279
:10582800C0F386100CF025F994F82C0200090CF04E
:10583800E8F894F82C0200F00F000CF0E2F80434B9
:1058480094F829020CF0DDF8AC42E1D143E0334C86
:105858000D200CF00BF905F07DF80CF0D2F820883B
:105868000CF010F9E0680CF00DF902F0D1FE30E010
:105878000CF0BEF8054684200CF0F8F828460CF029
:1058880001F9264BDC6805F18003A3428CBF641B39
:10589800802402F075FF28462246694605F08EF8F6
:1058A80000240546AC4216DA1DF804000CF0A9F8ED
:1058B8000134F7E713200CF0D9F80024184B185DD1
:1058C80001340CF09EF80B2CF8D100200CF0DAF81B
:1058D80000200CF0D7F8012018E0002016E00CF0AA
:1058E80090F8B4F8F4010CF0C4F894F8F6010CF050
:1058F80088F894F8F7010CF084F894F8F9010CF0A2
:1059080080F894F8F8010CF07CF847E720B0BDEC7B
:10591800028BBDE8F08700BF202C0020100000207B
:10592800A8A701082DE9F047CB4CCC4F237886B0C7
:105938000646002B00F0EB813A686368D31A7C2B8B
:1059480040F2E581237A6260013323724FF0000848
:1059580008F12400C04DC0B208F016F805F10A039A
:1059680033F9183007EE903ABD4B1B88B8EEE77A4A
:1059780007EE903AF8EEE77A08F10108C7EE277AC1
:105988009FEDB87A67EE877AFDEEE77ACDED037A78
:10599800BDF90C0007F0E6FFB8F1030FD8D13020AD
:1059A80007F0F2FFB5F9100007F0DCFF07F0E4FF9D
:1059B8002B7A9A072CD16A6841F288339A4218D90F
:1059C800102007F0E1FF4FF06408686990FBF8F0D9
:1059D80000B207F0C7FF212007F0D6FF686990FBE7
:1059E800F8F308FB13000028B8BF404200B207F0E4
:1059F800B9FF142007F0C8FFB4F9180007F0B2FF88
:105A08001C2007F0C1FF002007F0ACFF07F0B4FF2F
:105A1800237ADFF844825B0740F05681022007F0C2
:105A2800B3FFD8F81C00DFF854926423323090FB9F
:105A3800F3F000B207F096FF0320B8F9265007F0FC
:105A4800A3FF894B1B7813F0040F4FF0050A95FB51
:105A5800FAF5ADB20BD030460DF0CCF928B9D9F82B
:105A6800003013F0100F18BF002528B205E0D8F851
:105A780028309889B0FBFAF000B207F073FFD9F824
:105A880000309E0765D5DFF8F891E68D99F800306B
:105A9800A28D714D36014FF06408B6B208FB023290
:105AA8005B00B2FBF3F346EA0326B6B2C3F3032363
:105AB8001E43062007F068FF30B207F053FFE38D5E
:105AC80099F8001001339BB293FBF1F201FB1233FA
:105AD800E385236B9B7B012B05D1392007F054FF0D
:105AE800B5F92C0019E0AD8D6E233A205D431526DB
:105AF80007F04AFF95FBF6F5AEB2B6FBF8F528B20B
:105B080007F030FF08FB15653B2007F03DFFA8B202
:105B1800451D0A2095FBF0F000B207F023FF28206E
:105B280007F032FF636B0A2093FBF0F000B207F036
:105B380019FF042007F028FFA36A9B8913B107F017
:105B480055FB03E0444B986B80F3100000B207F05C
:105B580009FFE36B404E9D0640F1AB8096F840305C
:105B680098071DD5112007F00FFFB6F842003F4BEC
:105B78004FF4F365684390FBF3F000B207F0F2FED0
:105B8800192007F001FFB6F842004543642095FB51
:105B9800F0F595FBF0F300FB135000B207F0E2FEBE
:105BA80094F84030B4F8445013F0020F08BF0025B1
:105BB800012007F0E9FE28B207F0D4FE092007F01B
:105BC800E3FE002007F0CEFE294B94F846501A88D1
:105BD800B2F5967F0AD9204B1B7A03F00F03072BE7
:105BE80004D842F20F75954228BF1546052007F0E4
:105BF800CBFE236B5B7B0BB928B21CE0A5F120031D
:105C080007EE903A9FED1B7AF8EEE77AF6EE006A17
:105C1800C7EE877ABEEE007AF5EEC07AF1EE10FA9A
:105C280058BFB0EE667A77EE877AFDEEE77ACDED6B
:105C3800037ABDF90C0007F095FE94F84020064B56
:105C4800910703D493F84720012A1DD1012384F832
:105C58004730094834E000BFD01000202028002039
:105C68002000002000007A442A340020A086010089
:105C7800820000206666E63F18110020FC270020FD
:105C8800800000208096184B1B6B5FED026A93ED35
:105C9800017AD3ED027A27EE267A67EEA67ABDEE70
:105CA800C77AFDEEE77A8DED047ACDED057A04A882
:105CB80006E0B54A92E8030004AB83E803001846FF
:105CC80007F072FE07F058FE237A282B1FD1AF4B3E
:105CD80000221A723C263B684FF47A70B3FBF0F846
:105CE800172007F051FEB8FBF6F5B5FBF6F006FBFA
:105CF8001050000200B207F035FE182007F044FEED
:105D080006FB158000B207F02DFE07F035FE94F86B
:105D180050309E4D002B00F0588105F069FE6B6DE8
:105D28009B4AC31A9342064640F2C180002385F875
:105D38005A3085F85C30AB8DDAB21B0A85F87620CC
:105D480085F8773085F86C2085F86D30D5F8842093
:105D58003B689A1AD5F88830D97B4FF47A734B434D
:105D68009A420ED38B4B1B68C5F8843095F88C305B
:105D7800013B012B9FBF102385F85A30022385F879
:105D88005C300A20626B92FBF0F284F874201212E5
:105D980084F8752094F84020A36B93FBF0F384F803
:105DA80078301B1284F87930920794F84630774996
:105DB80084F8A73003D42D2381F8A83076E0042B8B
:105DC800D4F84890E76CDFF8DC81734A8CBF332342
:105DD800322381F8A8304FF0060C704B99FBF3F092
:105DE80097FBF3F308FB009108FB037803EB8303AD
:105DF8000CFB01F103EB830391FBF2FE642502FB2C
:105E08001E119B0091FBF5F184F8991009120CFB07
:105E180008FC84F89A109CFBF2F143FA81F39BB2D8
:105E280002FB11C292FBF5F284F89E20121284F84C
:105E38009C3084F89F201B0AB4F8422084F89D30D7
:105E48002423534393FBF5F5B4F8BA3084F8A03013
:105E580000EB80001B0A00EB8000800084F8A13072
:105E68000A22B4F84430B3FBF2F303F5FA739BB299
:105E780040FA8EF080B284F8A2301B0A4FEAD97932
:105E880084F89700FF0F000A84F8945084F8A33030
:105E9800C5F30725B4F8BC3084F8969084F89800C8
:105EA80084F89B7084F8955084F8A930666594F856
:105EB800BE80364DB8F1000F0DD1D5F8C40005F0FD
:105EC8007FFE012807D90228354F00F0508207F0DD
:105ED8003BFD0123BB70D4F8C8202C4D002A74D098
:105EE80095F8BE703FB1D5F8D03040F6B731F31A07
:105EF8008B4219D869E00123D5F8C40085F8BE3073
:105F080001F0E3FCD5F8D43093F9000002238DE8C2
:105F1800880008213A464FF4964301F0E9FC85F8D9
:105F2800D870C5F8C4004EE095F8CC70CFB9D5F854
:105F3800C400C5F8C87085F8BE7001F0C6FCD5F875
:105F4800D43093F9000001238DE8880008213A46EF
:105F58004FF4964301F0CCFCC5F8C40007F0F4FCFC
:105F680031E0013FFFB285F8CC7095F8D81095F86C
:105F7800D930CFB94A1C013385F8D82085F8D930F3
:105F8800D5F8C4001DE000BF4C8A0108D0100020DD
:105F98003F0D03002028002040420F008096980003
:105FA80020000020806967FF12F8017BC5F8C8202F
:105FB800781885F8D8000133D5F8C40085F8D930A9
:105FC800394605F000FEC4F8D06094F8DA309C4DEC
:105FD800DBB1D5F8DC30C3B1D5F8E030ABB1C5F8EA
:105FE800E4301B68974AC5F8E830D5F8EC3013441C
:105FF800187AFEF72BFD0BF015FDD5F8EC300133C0
:10600800092B88BF0023C5F8EC308F4D94F8F02099
:106018002E688B4B002A00F0E481D3F8F420002A84
:1060280000F0DF8193F8F830013B012B00F2D981B1
:10603800D4F8F400824F05F0C3FDE0B1D7F8F400BE
:1060480005F0BBFD97F8F930D5F800907E2B804617
:106058000ED102231B2887F8F83009D1D7F8F400AD
:1060680005F0AEFD20B90123C7F8FC9087F8003190
:1060780084F8F980DCE7D7F8FC202B689B1A41F6F6
:10608800583293421DD9032387F8F830A9E16F4AA3
:1060980032F8130010B903464FF403600133B0F52A
:1060A800C06FDBB275D01DD9B0F5006F7AD031D989
:1060B800B0F5036F3ED184F80131E36B604F990668
:1060C8003FD494F8001194F80131002900F04C8174
:1060D8002A68921B012ADAD984F80131002384F84E
:1060E80000317EE1B0F5007F42D007D8B0F5807F5F
:1060F80047D0B0F5887F00F08580E6E7B0F5806F7F
:1061080000F0A880B0F5826F00F0ED80B0F5047F54
:10611800DBD123E0B0F5E26F00F08480B0F5E46FE6
:1061280000F08580B0F5E06FCFD184F80131B4F983
:106138000A1080E0B0F5046F6DD0B0F5026FC4D1DD
:10614800FCE097F840309A07BBD5B7F842102423F3
:106158004B431233642193FBF1F1FFE084F80131E2
:106168003B4B374F1B689B07ABD5BB8D0A21F4E02F
:1061780084F80131364B324F1B681905A1D5796B6C
:10618800ECE084F80131E36B2D4F5A0799D5796912
:10619800E4E084F801312E4B294F1B681B0590D58C
:1061A800B96BDBE0E16B264A84F801318F0688D5AC
:1061B80092F84010880784D5D90711D5D36C83EAA3
:1061C800E371002BA1EBE37101EB51014FF01902D0
:1061D800B1FBF2F1ACBF41F0004141F040410EE0AB
:1061E800936C83EAE371A1EBE371002B01EB51019E
:1061F8004FF01902B1FBF2F1B8BF41F080414FF402
:1062080000608AE084F80131E36B0D4F5B077FF58E
:1062180058AF3969A2E0B4F9181084F80131642341
:1062280059437AE084F80131B4F90C1003E0B4F969
:106238000E1084F801312C2391FBF3F16DE000BFBF
:10624800D01000204C8A010820280020C0AB01088B
:10625800FC27002084F8013194F80231624A0133A6
:10626800DBB2032B88BF012382F8023194F80211B4
:1062780042F2107359435D4B1B78D80748BF013170
:106288009A0748BF02315F07B4F8043148BF0431A8
:10629800D80748BF0A319A0748BF14311F0648BFBC
:1062A8002831D80548BF28315A0748BF64311F072D
:1062B80048BFC831980548BF01F5C8719A0648BF5C
:1062C80001F57A71DF0648BF01F5FA61580648BF43
:1062D80001F57A614FF4806000F0CCFD424B00225A
:1062E80083F80021EDE6E16BDFF8FC8084F80131EA
:1062F80011F0200717D098F8402012F0020F14BFB1
:106308004FF47A71002112F0010F14BF4FF4FA63B1
:1063180000230B4494F84610194400F0ABFD002309
:1063280084F80031CDE6324B1B6819067FF5C9AEFB
:10633800394600F09FFD88F80071C2E684F8013103
:10634800E36B294F9A067FF5BCAE97F840309B0760
:106358007FF5B7AEB7F844306421594300F08AFDA1
:10636800002387F80031ACE684F8013139E0BB78C6
:1063780023B1C5F8C06087F80280ACE5D5F8C03015
:10638800F31AB3F57A6FFFF4A6AD0123D5F8C4006C
:10639800BB7005F012FC0746D5F8C40005F00DFCEB
:1063A8007F067FF498AD8A2802D08E280CD092E51B
:1063B800EB6B98067FF58FAD95F8BE30002B7FF418
:1063C8008AAD05F18D0306E095F8BE30002B7FF409
:1063D80082AD05F15803C5F8C8302D2385F8CC30B7
:1063E80079E506B0BDE8F087D01000202A340020F7
:1063F800FC270020344B354A1B68126810B51A6018
:10640800334A1168596051689268DA60314A996074
:1064180011681961516892689A612F4A5961116827
:10642800D961516892685A622C4A19621188198593
:10643800518859859188D288DA85294A99851188A1
:1064480019865188598692889A86264A1188D9864B
:10645800518819871946928821F83A2F224A1078CC
:106468000022824206DA214C34F8124021F8024F09
:106478000132F6E71E4A1288A3F864201D4A1288E2
:10648800A3F866201C4A1188A3F86C1051889288DA
:10649800A3F87020194AA3F86E1012689A66184A71
:1064A8003B21126892FBF1F2B2F5967FC8BF4FF01C
:1064B800FF325A67134A1288A3F87820124A528981
:1064C800A3F85E2010BD00BFC828002008340020B3
:1064D800F0190020FC190020081A0020F0100020F4
:1064E8002C100020DA100020901F00204C100020F3
:1064F80098230020E40F002032100020E410002030
:10650800040000206C100020381000202DE9F8430A
:106518000E4B93E8800305460E460024B44213DA76
:106528007B1933F9140008EB050333F9142009EB40
:10653800050333F914301344022293FBF2F3C01A13
:106548000AF06CFD0134E9E7BDE8F883C8280020AB
:1065580010B5134B93F8DC37012B014619D1114BB9
:10656800114C1878421CD2B21A70120644BF00228D
:106578001A700E4A1B7812782154934236BFC2F122
:1065880080029B1A9B183F2B09D9BDE8104002F0E6
:1065980013B9074BBDE81040186805F014BB10BDCF
:1065A800202C0020682700206A2700206927002067
:1065B800B028002070B54720FFF7CAFF174B1B68AB
:1065C8001B0307D5164B174A5B6810681B68C01A6F
:1065D8000AF014FD144E154C154D30780AF00EFDD6
:1065E80023682868C01A0AF019FD63686868C01A29
:1065F8000AF014FD0F4B18880AF000FD0E4B18889E
:106608000AF0FCFC0D4B18880AF0F8FC3378237468
:106618002B68A3606B68E36070BD00BF4C2A002044
:10662800C82800200834002016110020B4280020B3
:1066380018110020141100201211002074100020DD
:106648007FB5254C254E264D2649274A274B20B194
:1066580027480088B0F5805F30D23088ADF8040054
:1066680028781D4D897912788DF806008DF8071065
:106678008DF808201B788DF8093001A829460622D4
:106688000FF0BCFC28B30198BDF808302860AB8037
:106698005320FFF75DFF20880AF0B0FCA0780AF0CD
:1066A800ADFCE37801932379029301A863790393FE
:1066B8000AF008FC0E4B00221A800AE0308820807D
:1066C8008979287812781B78A070E170227163713B
:1066D800DEE704B070BD00BFD8110020D41100203F
:1066E80010110020340E0020630E0020C80E002078
:1066F8006C2A00200A4A138801331380094A136858
:1067080001331360084A138801339BB2202B01BF61
:1067180000231380054A138808BF0133138070478C
:106728006C2A0020542A0020582A00205A2A0020C7
:1067380038B5394B1B78083B012B05460C466AD8FF
:106748004520FFF705FF2846FFF702FF0C2D23D051
:1067580004D80A2D0AD014D835B138BD0E2D4BD027
:106768002ED3FF2D50D038BD206849E02078FFF7A0
:10677800EFFE62796378002A14BF80200020184356
:1067880000E02078FFF7E4FEA078FFF7E1FEE0786C
:10679800FFF7DEFE20793BE0B4F900000AF023FCA5
:1067A800A078FFF7D5FEE078FFF7D2FEB4F9040031
:1067B8000AF019FCB4F90600BDE838400AF013BC29
:1067C800637820788BB180F08000FFF7C1FEA46861
:1067D800E0B2FFF7BDFEC4F30720FFF7B9FEC4F32C
:1067E8000740FFF7B5FE200E12E0FFF7B1FE606824
:1067F800BDE838400AF012BC20680AF0FFFB606868
:10680800BDE838400AF0FABB04480AF00BFC002047
:10681800BDE838409CE638BDA4280020E0AB01085C
:106828002DE9F04FBE4BBF4F1A888BB00193002A59
:1068380040F0A980B7F8DA07BB4E42F20103C21A4A
:1068480050425041FFF7FCFEFFF7D4FD3468492061
:10685800FFF77EFEB54B254618680AF0CFFB55F8C2
:10686800040B0AF0CBFB284605F0C8FF04F1100022
:1068780005F0C4FF04F11C094FF01008AC4D0123CA
:106888002A6803FA08F3134203D0D9F800000AF083
:10689800C5FB08F10108B8F1130F09F10409EDD19E
:1068A80004F1280005F09AFFB7F84431B4F92E0036
:1068B800C01A0AF0A3FB2B68DB0408D59D4BB4F87B
:1068C80064001B88181AC0F30D000AF097FB2B68A8
:1068D800980403D5B4F866000AF090FB2B685905B4
:1068E80003D504F16C0005F079FF2B681A0502D571
:1068F800A06E0AF093FB2B685B0402D5606F0AF068
:106908008DFB2B68180403D5B4F878000AF076FBE1
:1069180004F13000A04605F061FF04F1360005F0EF
:106928005DFFB7F8443138F93C0FC01A0AF066FB2E
:106938000127814B1B789F4208DA38F9020FB4F916
:106948003C30C01A0AF06AFB0137F2E72B68990558
:1069580005D5B4F95E00A0F2DC500AF05FFB32689E
:1069680076487260B260121A9110754A4A43531CF5
:10697800032293FBF2F202EB42029A1A7C2303FBF6
:1069880002033360D6E16F4B6F4A1B6811688B4274
:1069980006D00AA9002041F8203D1360FFF7C8FE81
:1069A800019B97F8DA171B8897F8DB070B44013B24
:1069B800B3FBF0F200FB12338B4280F086815A4F12
:1069C8000120FFF73DFEFFF715FD50203E687D686A
:1069D800FFF7BEFDBA683B6810681B687A68034415
:1069E8001068A3EB40000AF019FB6A6873689B1AE9
:1069F8000293AA68B3689B1A0393EA68F36802A82B
:106A08009B1A049305F0FAFE2A6933699B1A0293CC
:106A18006A6973699B1A0393B369AA6902A89B1AE6
:106A280004930AF04FFA06F11C0B05F11C08102418
:106A38003F4901220B68A2401A428A4606D0DBF879
:106A48000000D8F80030C01A0AF0E8FA0134132C14
:106A58000BF1040B08F10408EAD106F1260005F150
:106A68002601002331F9024F30F9022F121B02AC24
:106A780044F823200133042BF4D103214FF00009FB
:106A88004FEA89035FFA83F902AB53F821206AB110
:106A980002F108000F2802D849F0010906E0803207
:106AA800FF2A94BF49F0020949F0030911F1FF31A7
:106AB800E6D24846FFF74CFD00240DF1080BA0462E
:106AC80009F00302022A16D0032A1DD0012A4ED14A
:106AD800B8F1000F05D1DBF800402401E4B290467C
:106AE80045E0DBF8000000F00F002043FFF730FD21
:106AF8004FF000083BE0B8F1000F0CD0DBF80000C5
:106B0800C0F3031020432CE0B8F1000F1ED19BF80E
:106B18000100FFF71DFD9BF80000FFF719FD26E0B7
:106B2800582A0020202C0020C8280020542A0020A1
:106B38004C2A0020482A0020901F0020D42800203A
:106B4800DF7BEFBD602A00205C2A0020DBF8000014
:106B5800C0F303302043FFF7FBFCDBF80000C0F371
:106B68000710FFF7F5FCDBF800402401E4B20BF155
:106B7800040B06AB9B454FEA9909A1D1B8F1010F67
:106B880002D12046FFF7E4FCDAF8003013F4805411
:106B98001FBFB6F86420B5F86410521A029218BFE5
:106BA80001249A040AD50AAA02EB8401B5F8660002
:106BB800B6F86620121A41F8202C0134580513D56E
:106BC80002AA02EB840C06F16A0E05F16A000022A3
:106BD8003EF9021F30F9028FC8EB01014CF8221070
:106BE8000132032AF4D10334190508D50AAA02EBA5
:106BF8008400A96EB26E521A40F8202C01345A044F
:106C080008D50AAA02EB8400696F726F521A40F81D
:106C1800202C013418040BD50AAB03EB8402B5F819
:106C28007810B6F878305B1A42F8203C013400E05E
:106C3800FCB1012C03D102980AF0F0F919E0631EA7
:106C4800002002AA400052F82320C0B20AB140F046
:106C58000100013BF5D5FFF77BFC4FF0000802ABC4
:106C680053F8280008B10AF0D9F908F10108A0453D
:106C7800F5DB30200321FFF749FC36200321FFF71D
:106C880045FC2F4B3C201978FFF740FCDAF8003020
:106C9800990506D5B6F95E00B5F95E30C01A0AF056
:106CA800BDF93A6827487B687A60121A9110264A1B
:106CB800BB604A43531C032293FBF2F202EB4202ED
:106CC8009A1A7C2303FB02033B60204B1B681A06BD
:106CD80030D51F4C1F4D22682B689A420BD1626831
:106CE8006B689A4207D1019B1B88102B11D11A4B54
:106CF8001B885B060DD14820FFF72AFC20680AF0A4
:106D08008DF960680AF08AF923682B6063686B6004
:106D18000EE0124A0F4B11782A7C914208D1104A92
:106D280099681068884203D15268DB689A4201D09A
:106D3800FFF740FC0AF0B4F80BB0BDE8F08F00BFD5
:106D4800901F0020D4280020DF7BEFBDFC27002007
:106D580078100020B42800205A2A0020161100209C
:106D6800181100202DE9F84F0C9E3A4CC2EB030B8A
:106D78000B9BF61A6368002914BF4FF0060A4FF000
:106D8800040A01330546904613D1236853455ED261
:106D9800314A324852F82320032B98BF29460AF07B
:106DA800ABF96368013363602D4B002205469A7185
:106DB80013E0002511E02B4A1278954240DA0B9B2C
:106DC800E3B109FB06F2995C01228A402649096869
:106DD8000A4213D1636801336360D4F804900A9BB4
:106DE8001C4F9945E7DB2BD10A20FFF7B1FB3B6825
:106DF80001333B604FF0FF337B6021E0184A917903
:106E080021B12C20FFF7A4FB013501E0012191718C
:106E1800226809FB0BF308EB030752B958F8030083
:106E28000AF000F997F904104B1C0544D2D00F481A
:106E380002E03A440E4811790AF05EF90544C9E7C0
:106E4800206850452CBF00200120BDE8F88F0020A5
:106E5800BDE8F88F642A0020608A0108EBAB0108BE
:106E6800D81100208C0000204C2A0020FAAB010821
:106E78006DAF010830B585B004AC002524F8025D7B
:106E88000091ADF806002146102006F03FFD9DF860
:106E98000600214606F03AFD9DF80700214606F057
:106EA80035FD9DF80000214606F030FD9DF80100F3
:106EB800214606F02BFD9DF80200214606F026FD2E
:106EC8009DF80300214606F021FD9DF80E00C04301
:106ED800C0B2294606F01AFD05B030BDF8B5044623
:106EE8000E4617460025204620210FF0D8F8044604
:106EF800D0B1013420460FF037F9B0F5617F05DBDA
:106F080040F634039842A8BF184601E04FF4617078
:106F1800A0F56170192390FBF3F00DB9307000E013
:106F280070703B7801333B700DB90125DBE72046D3
:106F3800F8BD30B505460C46134629462246024898
:106F4800BDE8304004F0D6B8F0AC01087FB504784D
:106F58000646E4B9354B1B6803EB8403192193F803
:106F68007B0093F87C6093F8792093F87A304FF49B
:106F7800617511FB005011FB0651009001912C48DE
:106F88002146013404F0B6F8142CE3D14BE00FF09D
:106F9800EBF81328054641DC244B701C1C682021A3
:106FA80000238DF80F300FF07AF81E35064670B1C1
:106FB800013630460FF0D8F819289FBF04EB850337
:106FC80058709DF80F30013398BF8DF80F30304658
:106FD80020210FF064F8064670B1013630460FF0F4
:106FE800C3F80D289FBF04EB850398709DF80F30F8
:106FF800013398BF8DF80F3004EB85043046E11C4F
:107008000DF10F02FFF76AFF9DF80F30042B0AD02D
:10701800601C002104220FF00CF804E00548002150
:107028001322FFF786FF04B070BD00BF4810002090
:107038000FAD010824AD010801480AF09FBD00BF4B
:107048002AAD01082DE9F04304788FB00546002CDD
:1070580059D17B4B0021142209A807AED3F8008030
:107068000EF0E7FF0722304600210EF0E2FF05A8E8
:107078000023A700059308EB070583801A4671498A
:10708800B5F802E031F813C01CEA0E0F0AD00DF172
:10709800380C0E3102F1010E6244595C02F81C1CD6
:1070A8005FFA8EF20133072BE9D100210B46664ABD
:1070B800B5F802E011F802C01CEA0E0F0AD00DF173
:1070C800380C063203F1010E63448A5C03F8242C61
:1070D8005FFA8EF301310629E9D118F807305B49C8
:1070E8008DE841006A78029209A81A0903F00F0393
:1070F80003F0EBFF2146564809AA013403F0FAFFD2
:10710800202CA6D198E00FF02FF81F28044600F392
:10711800868028462021E4B20EF0C1FF1F2C02D938
:10712800FFF78AFF88E0464B1B6803EB8404451C85
:107138000021204604220EF07CFF0027454B09AEB3
:10714800304600210A2217F803905FFA87F80EF0FC
:1071580070FF002315F8012B32B10A2B04D04A45E1
:1071680002D0F2540133F5E74A455ED108F1FF3306
:10717800032B09D8DFE803F01005023F0DF12301C6
:1071880034E00DF123011EE030460EF0EDFF2378C8
:10719800C0B243EA001006E030460EF0E5FF23785F
:1071A80000F00F001843207031E00133062B0AD09D
:1071B800244800F11B069E5D9642F6D103445A7D91
:1071C80063881343638011F8012F02B30023EFE7AC
:1071D8000133072B0AD01B4800F10E069E5D96422C
:1071E800F6D130F8132063881343638011F8012F18
:1071F8006AB10023EFE730460EF0B6FF0F2804DC33
:1072080030460EF0B1FF607001E000236370013773
:10721800052F93D1012408F04DFF6CB980E70E4883
:1072280000211F22FFF785FE06E0204600210422E8
:107238000EF0FFFE0024EEE70FB0BDE8F08300BFBC
:10724800E0110020788A01088D8A010838AD01080C
:1072580047AD0108998A010824AD0108F8B50478FA
:10726800064674B9304DB5F8C621B5F8C8312F486F
:107278002146013403F03EFF042C05F10405F2D148
:10728800F8BD2B490EF0DEFEA8B9274B4FF47A71F2
:107298004FF4FA62A3F8C611A3F8C821A3F8CA11DB
:1072A800A3F8CC21A3F8CE11A3F8D021A3F8D211CA
:1072B800A3F8D421F8BD30460EF056FF0328054642
:1072C8002BD8304620210EF0EAFE044630B10134B6
:1072D80020460EF049FF0126074600E006462046F4
:1072E80020210EF0DCFE10B9BDE8F840A4E601301C
:1072F8000EF03AFF012EF7D1A7F2EE2240F2DC534E
:107308009A42F1D8A0F2EE229A42EDD8064B703597
:1073180003EB8503DF801881F8BD064800210322AE
:10732800BDE8F84005E600BF202C002053AD010859
:1073380066AD010830BB01082DE9FF410478054618
:10734800002C39D17348744D0AF018FCD5ED057A34
:10735800F5EE407AF1EE10FA00F0D88021466F4839
:1073680003F0C8FE95ED050A684603F043FD0146A3
:107378006B4803F0BFFE95ED060A684603F03AFD38
:107388000146674803F0B6FE95ED070A684603F024
:1073980031FD0146624803F0ADFE95ED080A6846E6
:1073A80003F028FD013401465E4803F0A3FE0C2CCF
:1073B80005F11005CAD1A9E05B4905220EF086FE49
:1073C80040B9554B03F1C002002159611033934273
:1073D800FAD19BE02846554904220EF077FE044670
:1073E8002846002C40D120210EF059FE002800F03C
:1073F8008D80451C28460EF060FE07464C4B53F81E
:1074080024601EB94B480AF0B9FB7FE02846314694
:10741800FAB20EF05BFE01340028EFD13E4B03F1C7
:10742800C0029E460021596110339342FAD1424B63
:1074380003EBC4029846D2F804C0BCF1000F04D193
:1074480031463E4803F056FE57E0002718F834301E
:107458009F42F5DA3B010EEB030563440FCB14356D
:1074680085E80F000137F1E70EF07EFE0B2806468F
:1074780047DC284620210EF012FE054650B10135A2
:10748800284603F02DFC244B03EB061383ED050A75
:10749800012400E00446284620210EF000FE05469F
:1074A80048B10135284603F01BFC1B4B03EB0613C0
:1074B80083ED060A0134284620210EF0F0FD05462A
:1074C80048B10135284603F00BFC134B03EB0613B8
:1074D80083ED070A0134284620210EF0E0FD10B99B
:1074E800FFF7AAFD12E0013003F0FAFB0A4B032C68
:1074F80003EB061686ED080AF2D11148FFF71CFFC8
:1075080004E0104801210C22FFF713FD04B0BDE888
:10751800F08100BF6CAD0108202C002087AD010868
:107528008DAD01088CB8010866AD010891AD010860
:107538008094010896AD010820AC0108A5AD0108AA
:10754800ABAA010824AD0108F0B5047887B0064657
:107558001CBB514B1968062303FB0411192091F831
:10756800CA5091F8CB7091F8CE2091F8C9304FF4F9
:10757800617610FB056510FB07600095019091F896
:10758800CC000290C831454849790391214601341D
:1075980003F0B0FD0C2CDCD17CE00EF0E5FD0B28EF
:1075A800044672DC3C4B701C1D68202100238DF8BA
:1075B80017300EF074FD064680B1013630460EF0E5
:1075C800D3FD03289FBF062303FB045383F8CE0093
:1075D8009DF817309CBF01338DF8173030462021B5
:1075E8000EF05DFD074680B1013738460EF0BCFD50
:1075F8000D289FBF062303FB045383F8C9009DF899
:1076080017309CBF01338DF8173006266643A91939
:107618003846CA310DF11702FFF760FC20210EF041
:107628003EFD074670B1013738460EF09DFD14281F
:107638009FBF9DF817307619013386F8CC0098BFA4
:107648008DF81730384620210EF029FD78B1013029
:107658000EF08AFD0D289FBF062303FB045383F811
:10766800CD009DF817309CBF01338DF817309DF879
:107678001730062B0ED0062202FB04500021C93019
:107688000EF0D7FCFFF7D8FC04E0054800210B22D8
:10769800FFF74FFC07B0F0BD48100020B1AD01085E
:1076A80024AD01082DE9F341047880464CB9204601
:1076B80001A90AF057F80134FFF7F4FF122CF6D1AC
:1076C8006BE00EF051FDC6B2112E61D8344C06F1B4
:1076D800D00704EB470308F1010020219D780EF044
:1076E800DEFC18B9AA1E5542554139E04378682B8B
:1076F80006D0732B07D0612B13D14FF0000804E09C
:107708004FF0010801E04FF00208A8F102035D42C2
:1077180000F101004FF020015D410EF0C0FCD8B12E
:1077280015B9FFF789FC38E001300EF01DFD40F275
:10773800ED2380B2984205DD40F6CA039842A8BFFF
:10774800184601E040F2EE2004EB4703A0F2EE20D9
:10775800192290FBF2F0D87004EB470383F80280FB
:1077680004EB47040F4AA378134493F8262055B135
:10777800E3780D4840F2EE241925314605FB034312
:1077880003F0B8FC09E03146084803F0B3FC04E014
:10779800074800211122FFF7CCFB02B0BDE8F081B9
:1077A800202C0020788A0108D1AD0108E3AD01083A
:1077B80030BB010807B50123ADF8041001A98DF805
:1077C80006208DF8073007F037FE03B05DF804FB9C
:1077D8002DE9F843054672B64FF090464FF48061A4
:1077E8004FF40079318530460422A6F82890FFF737
:1077F800E1FF304601224946FFF7DCFF2B4850F8ED
:10780800354000EBC500236842680125570005FA9A
:1078180007F848EA030395402360A561C6F8189065
:107828004FF090431B8A5B05FAD4236848EA0303A8
:1078380023604FF090434FF40072A9B221851A8556
:107848000822C3F8182440F605534FF09040028AE6
:10785800560512D4013BF8D122680323BB4022EA23
:10786800030323604FF400710222FFF7A3FF62B6FF
:107878003220BDE8F84304F0E2B8A56120460422AE
:10788800FFF798FF4FF090431A8A5205CDD5228A08
:1078980092B21542064A4FF400704FF0080115BF26
:1078A8009861188591611185ECE700BF14AE010855
:1078B8000004004810B50446204604F078F918B9C9
:1078C8000A2004F0BCF8F7E710BD002207490C2392
:1078D80003FB02135968814204D10022C2621A7262
:1078E8005A6070470132052AF0D1704718230020EA
:1078F8002DE9F74389469DF8288011461A469DF8D8
:107908002C30064600250C2068431D4FC419C0576B
:10791800B04202D1207A20B12BE00135052DF2D1F9
:1079280027E0022E0FD005DC56B1012E21D100939D
:1079380014480AE01E2E0DD01F2E1AD1012009E08E
:107948000093114801E011480093434601F0D6F82E
:10795800044605E002F044FF4146044604F024F9D9
:107968004CB10C2303FB0575267185F808906C60F3
:1079780001E0002000E0204603B0BDE8F08300BF2E
:10798800182300200044004000380140004800400F
:1079980010B5084B1968002201EBC20393F90240A5
:1079A800844201D1981C10BD0132052AF4D100206F
:1079B80010BD00BF14230020F0B5027887B08AB943
:1079C8004A4C04F1280694F8F221002348495956F4
:1079D80050B281426ED00C333C2BF7D10834B442FC
:1079E800F1D181E0002204920592451C0EF0BCFB07
:1079F800C4B260B2FFF7CCFF074618B18DF810404B
:107A0800012400E00446284620210EF048FB0546E4
:107A180038B1013528460EF0A7FB0134ADF8120045
:107A2800E4B20026284620210EF039FBB0B3451CED
:107A380028460EF099FB00222E4951F82230834245
:107A48005FFA82FE04D00132082AF5D1002300E053
:107A5800734651F82320824220D1022E0FD0032EE4
:107A680012D05A1E012ED2B204D0042A13D88DF88F
:107A780014300EE0042A0ED88DF8153009E0052BD5
:107A880009D88DF8173004E09A1E052A03D88DF816
:107A980016300134E4B20136042EC3D1052C04D8C3
:107AA80007B0BDE8F040FFF7C7BA04AB03CB3860B6
:107AB800796019E094F8F7010E4B94F8F65153F8F1
:107AC8002000B4F8F421009094F8F90153F820004C
:107AD800019094F8F80153F82000029053F82530EB
:107AE800054803F007FB79E707B0F0BD202C00201C
:107AF800182300203C920108F2AD010838B14388F0
:107B080011EA030003D08B420CBF0120022070470A
:107B180030B50A4B0A491C680A79042A0AD8134660
:107B280004EBC303551CEAB29D882842F5D00A71BC
:107B3800981C30BD0A71002030BD00BF14230020FE
:107B4800E0110020014B00221A71E1E7E01100204A
:107B58002DE9F047877890F803C0214DBBB2C7F1F3
:107B6800640E03EB83065C42C3F178005FFA8EFE75
:107B78007600CCF16408A4B280B2A3B20FFA83F9FC
:107B8800B9F1000F05DC002B14BFBA464FF0010A0B
:107B980000E0F24613FB03F303FB0CF21AFB0AF3B3
:107BA80092FBF3F3434403FB09F30A2293FBF2F33A
:107BB80033449BB225F8023FB1F800904A880A3452
:107BC800C9EB020AA4B21AB202FB0AF24FF47A73A2
:107BD800844292FBF3F34B442B80CED1BDE8F0876F
:107BE800E4110020426A806A131A584258417047CB
:107BF8004171704743799B070AD5436A8269D1541A
:107C0800436A01690133B3FBF1F201FB12334362AA
:107C1800704707EE900AF8EEE77ADFED0C6A9FED01
:107C28000C0AF5EEC07AF1EE10FAD4BFB1EE677A1D
:107C3800C7EEA67A08B5D8BFC7EE267A27EE800A1F
:107C480003F0EAFA034B83ED000A08BD8096184B4F
:107C580035FA8E3C7800002038B50D4B0D4D1A8A48
:107C68000D4B1968498811421C4603D003F0C0FE29
:107C7800286007E003F0BCFE2B68984282BFC01A58
:107C8800064B186023685868BDE8384004F0DCBE2D
:107C98000004004800120020A00700200400002073
:107CA80003460A4690F84602D96A9B7902F098BDC5
:107CB800437913F0010310B504460DD002F066F9BC
:107CC80058B1236A6269E168D05C0133B3FBF1F211
:107CD80001FB1233236210BD184610BDF8B59B4B4B
:107CE8001B680446187818B1012800F068819BE2E7
:107CF800242C974D0CD006D80A2C00F0D9800D2CD6
:107D080000F0D68046E12A2C06D02C2C04D041E184
:107D180028716871A8714EE18E4B69792F798C4A68
:107D2800002058542FBB1978D771472921D1597889
:107D380050291ED19978472907D1D978472904D1E4
:107D48001979412901D10121D1719978814A5229A2
:107D580003D1D1784D2900F0918299787D4A47293D
:107D680007D1D178532904D11279562A04BF0322A6
:107D7800EA71EA79764E022A39D0032A4CD0012AD0
:107D880040F08580BA1E072A00F28180DFE802F001
:107D980004080F131A257F2A09F038FCA86076E03A
:107DA8001B78532B73D1AB685B42AB606FE009F073
:107DB8002DFCE8606BE01B78572B68D1EB685B42C1
:107DC800EB6064E01B78302B634B1A788CBF42F071
:107DD800020222F002021A7059E0002009F076FC33
:107DE800287454E0002009F071FC68824FE0072FE6
:107DF80006D0082F4BD1012009F068FCF08246E03C
:107E0800012009F063FC41F2184358434FF47A7398
:107E1800B0FBF3F0B0823AE0022F07D0032F0AD16B
:107E2800002009F053FC4D4B187030E0002009F099
:107E38004DFC30762BE02AD93A1F9210337E01325E
:107E4800D2B2013B02EB8303DBB2102B1FD8F91E21
:107E5800C2F1010201EB8202D2B2012A0BD0042A3C
:107E680011D100205E1E09F031FC3D4B98553D4B69
:107E780000229A5507E05E1E3B4A0020935509F000
:107E880025FC3A4B98553A4A136801331360304B36
:107E98002A2C18BF9A7907F101074FF000000CBF90
:107EA800012254402F7168710CBF5A769C7182E090
:107EB800687E002847D02F4B13F8012D2E495A70A1
:107EC8008B42F9D1234A224C13785278402B85BF34
:107ED800373B1B011B01DBB298BF03F0F003402ABC
:107EE8008CBF373A303AD2B21344AA79DBB29A42FD
:107EF80026D121230B702149E0790B681E4A0133F2
:107F080001280B600AD002281CD1722313701C4B65
:107F1800A28A1A801B4BE28A1A8013E06723137027
:107F28000D4B1B789F070ED5174BA2681A60E268A5
:107F38005A60164B227C1A70154B628A1A8002E02E
:107F48003F230B70002000236B7634E0C407002029
:107F58000012002028280020101100208C1000207A
:107F6800BD100020AD1000208D1000209D100020B5
:107F780060240020D8020020C40200206C240020C5
:107F88001211002074100020181100201611002072
:107F9800141100206B79687E0E2B9FBFA34A591CD1
:107FA8005171A34A98BFD454A04A18B993795C4038
:107FB800947100E00020003018BF0120F8BD9B4BF1
:107FC800997E0022082900F22F81DFE801F0050BD5
:107FD8000F15202B48606A00B52C40F02581DA7611
:107FE80001223AE0622C08BF022236E003229A7688
:107FF8001C775C779C7717E104229A765A7F997FE1
:10800800DC772244D2B25A770A449A770CE10522E7
:108018009A765A7F997F1C842244D2B25A770A44AE
:108028009A7701E106229A765A7F997F2244D2B242
:108038005A770A449A771A8C02EB0424A4B2B4F54E
:10804800AC7F88BF794A1C8484BF0121D176002285
:108058005A84002C40F0E88007229A76E4E05A7FA0
:10806800997F2244D2B25A770A449A775A8CB2F549
:10807800AC7F3CBF6D49891802F1010238BF81F815
:108088002440198C92B291425A84E5D9CCE0082256
:108098009A765B7FA34200F0C780644B0122DA76B0
:1080A8000DE0644D9A7615F8012D6A70624A954282
:1080B800F9D1997F5D4AA14206D03F232B705F4AD0
:1080C800536801335360AFE05D48016801310160D6
:1080D800D07E10B13E232B70A6E021212970D17FDC
:1080E800062941D004D8022907D0032923D0F8BD96
:1080F800122959D0302967D0F8BD5021297051492B
:10810800946A4C60D46A0C60516B4FF47A7491FB9A
:10811800F4F14D4C218092F87C114C4A19B1117838
:1081280041F0020102E0117821F0020111700122F0
:1081380083F87D2169E05321297092F82910CE0730
:1081480005D592F82820D51E6A426A4100E0024609
:1081580002F0010183F87C11002A56D13B490A78C4
:1081680022F002020A7050E04F21297092F82F1075
:10817800CC0705D592F82E20D11E4A424A4100E08C
:10818800024602F0010183F87C1122B92F490A78CE
:1081980022F002020A702E4A93F8531011702D4AE9
:1081A800B3F85010118030E0562129702A49946B99
:1081B8000C8042F21074D16B91FBF4F1274C2180B2
:1081C800012182F87E1120E04921297092F82810B7
:1081D800234A102988BF10211170224914780022DF
:1081E800A2420ED2204D0E7A5655204D4E7A565543
:1081F8001F4DCE7A56551F4D11F80C6F565501324A
:10820800EEE71D490A6801320A6093F87D31074A92
:10821800002B3AD092F87E31BBB3002182F87D1151
:1082280082F87E111846F8BD0020F8BD0012002023
:1082380028280020D8020020C4020020A40700201B
:108248006C240020181100201411002010110020A7
:108258001611002082000020121100207410002046
:108268008C100020241200208D1000209D1000206A
:10827800AD100020BD100020602400201279432A90
:108288007FF46BAD0222EA7167E5F8BD0449054B3E
:108298000968187000225A6199611A77704700BFFF
:1082A80020280020A407002010B5121A07EE902AF3
:1082B8005B1A2DED028BF8EEE78A07EE903A184B21
:1082C800059CB8EEE78AD3ED007A28EE278A28EED7
:1082D800080AA8EEA80A0EF061FBDFED127A049BEB
:1082E80020EE270AF0EE480ABCEEC00A83ED000A29
:1082F800B1EE680A0EF0AEF9DFED0B7A9FED0B7A5E
:10830800E0EE077ABDEC028BFDEEE77A17EE903AC5
:10831800002BBCBF03F50C43A033236010BD00BF86
:10832800780000202C7D8E3F00A00C46A00CB345A1
:1083380044F25063984203DDA0F50C40A038704722
:10834800034B9842BCBF00F50C40A030704700BFFB
:10835800B0B9FFFF73B51A4C036823600B686360FC
:10836800184D0068184EFFF754FC184B009395E819
:10837800030094E80C000196FFF796FF144B32684F
:108388001A606868636813491B1A07EE903A124B23
:10839800286893ED007A23681B1A0B600F4BF8EEE0
:1083A800E77A1A600E4B67EE877A1B68FDEEE77A6C
:1083B800DA880C4BC1ED017A1A8002B070BD00BF9B
:1083C800082700201811002014270020102700205B
:1083D8005027002018270020780000204827002078
:1083E800380F0020442700204279DFED2A5A2A4B13
:1083F8009FED2A5A07EE902AF8EE677AC27BC7EEFD
:10840800A57AB2EE047AC3ED007A07EE902AF8EE68
:10841800677A234ADA60C7EEA57AC3ED017A8179D3
:10842800204B07EE901AF8EE677A017CDA60C7EE07
:10843800877AC3ED007A07EE901A817E06EE101A4D
:10844800F8EE677AB8EE466AC7EEA57A86EE056A50
:10845800C3ED017A83ED026AC179134B06EE901AD7
:10846800417CDA60F8EE666AC6EE876A07EE101A93
:10847800C17EC3ED006A07EE901AB8EE477AF8EEAF
:10848800677A87EE257AC7EE857A83ED017AC3EDA0
:10849800027A70470000C8422027002000007A4472
:1084A8000000FA44302700205427002010B50C4C57
:1084B80023789B0713D50B4B1B78042B0FD90A4A3B
:1084C8000A4B106852685A601860FFF7A2FB084B05
:1084D8001A88084B1A80237843F00103237010BDD3
:1084E800101100201611002018110020781000200B
:1084F800E8100020642700201C4B1B681B0307B5ED
:1085080030D51B4A1B4BD2ED007A1B788DF8003012
:10851800B2EE047A67EE877A174B9FED187A1B78CC
:108528008DF80130FCEEE77A0A2017EE903AD2ED8A
:10853800017A8DF8023067EE877A6946FCEEE77AB1
:1085480017EE903AD2ED027A8DF80330FCEEE77A16
:1085580017EE903A8DF80430094B1B788DF80530EA
:10856800FEF7E6F803B05DF804FB00BFFC27002027
:1085780010280020EE2700200C28002000007A4454
:10858800F2270020054A137883F001031370044A88
:1085980000231360034A1360AEE700BFF2270020F0
:1085A8000828002004280020094A13781844C0B27B
:1085B80010F0800F18BF803810701346054A1978DC
:1085C8001378994201BF00231370014A1370704752
:1085D800692700206827002010B50A4B0A4A1B7833
:1085E80042609C18094A046012789A4225BFD31A3F
:1085F8000B60C3F1800300232EBF4B600B604A6001
:1086080010BD00BF692700206A27002068270020C6
:108618001FB5684602A9FFF7DFFF044B02981B68E5
:1086280003440398184405B05DF804FB28060020AD
:108638002DE9F04F89B082460193002302910392FD
:108648009946039A934205DA029A52F82320013395
:108658009144F6E7019B4D46002B56D102F07AF97A
:10866800002852D101987CE002223F4E8DF81C2050
:108678001A0C4FF480578DF81D2006201A0A8DF821
:108688001E208DF81F3002F089F93785062008F082
:1086980045FD364BB76101221A700020378507A9BE
:1086A800042208F063FD029FD04626464FF0000BD7
:1086B800039B9B451EDABC4657F8042B4FEA8B03F5
:1086C800002A47D0B24235D332465AF80310CDF8C3
:1086D80014C00020049308F049FD049BDDF814C081
:1086E8005AF8032032444AF80320DCF800309E1B75
:1086F800CCF800601C4B4FF480529A611C4A1368F6
:108708002D1B1C44019B14604BB345B3184B1B68CD
:10871800DCB22A19B2F5807F164AD2688CBFC4F53C
:1087280080742C4693429FD3134A00231370134A34
:10873800137014E00020D8F8001008F017FD57F85F
:10874800043CD8F80020F61A1344C8F80030002377
:1087580047F8043C0BF1010B08F10408A8E7C5EB46
:10876800090009B0BDE8F08F000400482506002084
:108778002806002010000020682700206927002014
:1087880030B50B4C0B4D22782B789A4285B00CD023
:10879800684602A9FFF720FF0123684602A90222C2
:1087A800FFF746FF00232B70237005B030BD00BFD4
:1087B800692700206827002030B50E4D0E4C2A7816
:1087C80023789A4285B011D0684602A9FFF704FFC2
:1087D800002302A902226846FFF72AFFFFF7E4FEFA
:1087E80020782B781B1A5842584100E0012005B028
:1087F80030BD00BF692700206827002038B50E4C1F
:108808004FF4805545F2082002F0C8F82585062067
:1088180008F084FC094BA56101221A70C720258540
:1088280008F07CFC064AA56100231370054A137002
:10883800054A136038BD00BF000400482506002023
:10884800682700206927002028060020FFF704BABF
:10885800FFF702BAFFF700BA026BC168034610B50A
:10886800406942B11A6C8C1A013A005D08BF0A4689
:10887800C0B21A6410BD1A6A805C01328A4228BFED
:108888000022C0B21A6210BD436B13B190F84400C5
:108898007047836A406A1B1A584258417047036BF5
:1088A80013B15B68016C01E0C369016A8B423CBF8C
:1088B800C2689B18581AC0B27047836A8169426BB4
:1088C8001944D160416A99429DBF0169CB1A53602E
:1088D800CB1A96BF0023536083624FF0000380F8E1
:1088E8004430136888BF816243F001031360704706
:1088F800436A8269D154436A02690133934228BFAB
:1089080000234362436B1BB11B68DB0705D4D4E724
:10891800026D136843F0800313607047F0B5046D6F
:108928008668236823F0010323608379054613F0E2
:10893800020F40790CBF4FF0000E4FF4005E13F0A9
:10894800040F14BF4FF48067002710F0010F14BF05
:10895800042100218307206820F00100206062685C
:1089680022F440524EEA02026260226822F4B053B6
:1089780023F00C0348BF41F008013B430B4323603D
:10898800A36895B023F44073A360684604F0E4F943
:10899800284B9C4201D10C9B0EE0274B9C4201D1F5
:1089A8000D9B09E0254B9C4201D10E9B04E0244B12
:1089B8009C420CBF0F9B109B2268A879170448BFE4
:1089C8005B00B3FBF6F206FB1233B3EB560F2368DA
:1089D80028BF01321E0441BF4FF6F073C2F34201B3
:1089E800134041EA03026B7992B213F0020FA2819D
:1089F80000F0010114BF4FF400320022DC0748BF29
:108A080042F480322B6D11B159680A4302E059686B
:108A180021EA02025A609A6801074CBF42F0080234
:108A280022F008029A601A6842F001021A6015B032
:108A3800F0BD00BF0038014000440040004800403D
:108A4800004C0040417169E7816067E7026D036B84
:108A580070B50446D5699BB9A90611D5C36A1BB17F
:108A6800908C80B298470BE0E169928C40694E1C6B
:108A7800D2B2E6614254E169E268914228BFE361FB
:108A8800616BA1B92A0612D5636AA26A9A42236D5C
:108A980009D0501CA669A062B25C1A852369984265
:108AA80005D3A16203E01A6822F080021A602B073E
:108AB80042BF236D08221A6270BD0D4B0D484FF45A
:108AC80000525A600C4A11684FF6FE730B4013604F
:108AD800426B11684FF6FE730B401360426A836A5B
:108AE8009A4200D0E9E6012380F84430704700BF7D
:108AF8000000024048260020440002402DE9F047CB
:108B08001E46A64B8CB09842894690469DF8505018
:108B180040F08580A24BA34A1A60A34A5A6102F525
:108B280080729A614FF48072DA601A619F4A1A6300
:108B3800143A5A63A2F54842203ADA6404329A6435
:108B4800C3F8088018659A4B9A6942F480429A6182
:108B58005A6942F001025A6102238DF80830032352
:108B680015F0010A8DF809304FF000038DF80A302E
:108B780014BF022301232C078DF80B3019D54FF0B1
:108B880090444FF4007701978AF001038DF80A307A
:108B9800636A23F0F0036362636A43F070036362FD
:108BA800204601A904F04AFABAF1000F27D1A761BB
:108BB80025E0B00710D50CA94FF4007341F82C3DFF
:108BC8004FF09040436A23F0F0034362436A43F056
:108BD8007003436204F032FAF10710D50CA94FF480
:108BE800806341F82C3D4FF09040436A23F4706352
:108BF8004362436A43F4E063436204F01FFA0E23BE
:108C08008DF800300022012368468DF801308DF878
:108C180002208DF80330624C08F0DEFA0BE1654B58
:108C2800984276D1644B5F4A1A604FF48072DA60DA
:108C38001A61624A5A6102F580729A615C4AC3F805
:108C480008801865D36943F40033D36102238DF893
:108C58000830032315F0010A8DF809304FF000039E
:108C68008DF80A3014BF022301232A078DF80B3030
:108C780019D54FF090444FF4804701978AF00103CB
:108C88008DF80A30636A23F070636362636A43F0A5
:108C9800E0636362204601A904F0D0F9BAF1000F3D
:108CA80027D1A76125E0B30710D50CA94FF480435D
:108CB80041F82C3D4FF09040436A23F070634362C3
:108CC800436A43F0E063436204F0B8F9F70710D54C
:108CD8000CA94FF4004341F82C3D4FF09040436AF3
:108CE80023F070434362436A43F0E043436204F075
:108CF800A5F926238DF800300022012368468DF857
:108D080001308DF802208DF803302B4C08F064FAFE
:108D180091E02B4B984240F00F812A4B214A1A6070
:108D28004FF48072DA601A61274A5A6102F580723C
:108D38009A611F4AC3F808801865D36943F48023F1
:108D4800D36102238DF80830032315F0010A8DF84A
:108D580009304FF000038DF80A3014BF02230123B5
:108D68002C078DF80B3033D5184C4FF480670197DA
:108D78008AF001038DF80A30636A23F47063636232
:108D8800636A43F4E0636362204601A904F056F97C
:108D9800BAF1000F40D1A7613EE000BF00380140A2
:108DA80048260020648F01088013002058000240E4
:108DB8000010024000440040F425002080150020E7
:108DC80000480040A025002080170020000400482B
:108DD800B0070FD50CA94FF4806341F82C3D5848D3
:108DE800436A23F470634362436A43F4E063436273
:108DF80004F024F9F1070FD50CA94FF4006341F8EA
:108E08002C3D4F48436A23F470434362436A43F45A
:108E1800E043436204F012F927238DF80030002262
:108E2800012368468DF801308DF802208DF8033053
:108E380008F0D2F9434CC4F82C900027012384F899
:108E480044302762E761A76267626671C4F80880E8
:108E5800A5712046FFF762FDF20734D5236B002B7E
:108E68002AD001A803F0FCFDE36C01934FF4805372
:108E78000A9380230693E368ADF810302023099302
:108E8800206B636902930B970597079708970397D9
:108E980003F011FE01A9206B03F0EFFD236B216D98
:108EA8001A6842F001021A608A6842F040028A6039
:108EB8005B689BB2236406E0236D20221A621A685D
:108EC80042F020021A60B3072FD5636B43B301A8A1
:108ED80003F0C6FDA36C01934FF480530A938023DB
:108EE80006932369ADF8103000251023606B0393B7
:108EF8000B95059507950895099503F0DCFD606BC2
:108F080001A903F0BAFD636B1A6842F002021A6005
:108F1800226D5D605D60936843F08003936004E0B8
:108F2800226D136843F080031360226D136843F0C9
:108F380001031360204600E000200CB0BDE8F08774
:108F480000040048A02500201FB50123ADF8083013
:108F58000023ADF80C30ADF80A30094BADF8041019
:108F68001B78ADF80620012B08BF032301A908BF11
:108F7800ADF80C3003F02DFE05B05DF804FB00BF22
:108F88002C0100202DE9F04F2DED028B85B007460E
:108F98000293A04B1B889807934636D5109B9E4892
:108FA800DC89B0F900301B1B03F2F31540F2E632FE
:108FB800954203D8002BB8BF5B4201E04FF4FA7327
:108FC800B0F90220121B02F2F31440F2E630844298
:108FD80003D8002AB8BF524201E04FF4FA72934214
:108FE800B8BF1346C3F5FA73052293FBF2F30A22BE
:108FF800643B53433A7FD2105343642293FBF2F30A
:10900800134423EAE373DBB200E064230093CB1C30
:109018000193B8460024019BDFF824A213F8016FDE
:109028000193022C4FEA440905D1BAF904301B36E2
:109038005E43761146E079493AF8142031F9141064
:10904800022012FB0011CBF10002914203DB5945CB
:109058000A46A8BF5A467249029B31F90950551B66
:1090680033F91420154409F03FF988B107EE905AF6
:109078006C4AB8EEE70AB2EE048A105D80EE080A80
:1090880008F036F920EE080AFDEEC07A17EE905A7D
:10909800604A1288D10712D43AF909301B365E4368
:1090A80093074FEA26160DD5BB7C5D439DF900302A
:1090B8005D43642395FBF3F506EB251602E03E7A43
:1090C80075432E11584B042533F9093093FBF5F5F8
:1090D800564BE25C924698F80120751B51466A434C
:1090E8004A43642192FBF1F297F85110D21108EE2D
:1090F800102AA9B1022CB8EEC80A08D14A0803D030
:109108009142A8BF114600E00121494802E0181D1C
:1091180000EBC400D3ED070A01F0B8FDBDEEC08A2C
:10912800DFF808E1434B98F80B6018880EF120032C
:1091380000FB05F253F82410D21206FB0216B6F50E
:10914800001F3D4AA8BF4FF400169642B8BF164606
:109158000EF12C0243F8246052F8243042F82450CF
:10916800EB1A0EF138014FF6FF720009B2FBF0F06E
:1091780043430EF1440051F8245050F8242040F89D
:1091880024509B112A4441F8243097F850101A446F
:109198004FEA840C761300EE102A79B10EF15000D4
:1091A800B8EEC00A00EBC400DEED070ACDF80CC02B
:1091B80001F06CFDDDF80CC0BDEEC00A98F8153062
:1091C80010EE102A18EE101A5A43534653431A4603
:1091D8003144642392FBF3F3184A1B12194422F812
:1091E800091018EE100A02F1080101344CF80100C8
:1091F80002F114012032032C4CF801604CF80230C3
:1092080008F101087FF407AF05B0BDEC028BBDE89B
:10921800F08F00BFD411002038280020223400200D
:10922800F42700207C8F01082C10002080190020D2
:1092380094190020001000200000E0FFE819002029
:10924800F01000202DE9F04F2DED028B85B08046FF
:109258000393BC4B02911C88019204F00204A4B24F
:1092680094B1B94BB3F90240B3F90030002CB8BF40
:109278006442002BB8BF5B429C42B8BF1C46B4F5A1
:10928800007FA8BF4FF40074C2460025AF4AAE4B1A
:1092980032F9152033F81510AD4882EAE27EAEEBBC
:1092A800E27E0BB2BEF5206F4FEA45094FEA430351
:1092B8004FEA850750F8256012DC4FF0040E92FB48
:1092C800FEF29A1A1644B6F57A5FA8BF4FF47A569A
:1092D800A04A9642ACBF40F8256040F8252002E03D
:1092E800002240F82520C6599AF80B20F61156435B
:1092F8009AF801205343934A12884FEAA31B930715
:109308004FEAA61654D0944A019B32F9092002204C
:1093180011FB00215A42914203DB8B42A8BF0B4646
:109328001A468E49039B39F90110511A33F9152051
:109338008B1808EE103A08F0D7FF68B1B8EEC80AE3
:10934800874AB2EE048A80EE080A505D07F0D0FF23
:1093580020EE080ABDEEC08A824883493A5818EEC2
:10936800103A42F2107E1A447245A8BF72468A42E9
:10937800B8BF0A463A5098F8081098F81C005943A4
:1093880000EB8000C911C0F1000E714503DB81427A
:10939800A8BF01468E4698F812104A431213CEEB26
:1093A8000B03B61A6643634302EB66260EEB632B88
:1093B800664A39F90210042291FBF2F16B4A02F174
:1093C8009C00405D4143ABEBA11398F8511008EEA7
:1093D800103A51B1101DB8EEC80A00EBC500D2ED25
:1093E800070A01F053FCBDEEC08ADFF880E1574B55
:1093F8000EF1A00139F8030039F9012029F801001C
:109408000FFA80FC0EF1A4010EF1AC00C2EB0C02C5
:109418003B584FF0040C92FBFCF257F801C07A500D
:10942800634498F8501047F800C0134400EE103A0F
:1094380059B10EF15000B8EEC00A00EBC500DEEDE0
:10944800070A01F023FCBDEEC00A484901F1B40245
:1094580010EE103A525D53435A1118EE103A01F1CA
:10946800680E9819801A01F1700329F80E0018EE99
:10947800100AF85001F17C035242FE5001F18803B2
:109488000AF1010AFA500B460DB90125FEE62E4AEB
:109498009C6AB2F90410029A92790F3252004A4338
:1094A80052112A49002AB1F904104FF0040091FB27
:1094B800F0F0A2EB0000B8BF5242322A98F80D1023
:1094C8000BDC2B4A01FB00418A42A8BF0A46294906
:1094D8008A42ACBF9A62996201E000229A6298F8C7
:1094E800031001FB00F22449097803294FEAA2126C
:1094F8000CD9B8F84E10B1F5FA7F07D2484282422B
:1095080003DB8A42A8BF0A4600E00246996A9A67C6
:1095180041F34F31B1F5807FA8BF4FF480716FF0F0
:10952800FF008142B8BF014650180022A3F86C0022
:10953800C3F88410C3F8902005B0BDEC028BBDE8D9
:10954800F08F00BFD4110020F01000202C10002054
:10955800A019002080C1FFFF22340020F42700203A
:109568007C8F0108141A0020F0D8FFFF8019002012
:10957800FEFFFF0F020000F0901F00202DE9F04FC2
:109588002DED028B87B000260593C54B0491B3F9E6
:109598000280B3F900300392B8F1000FB8BFC8F1E8
:1095A8000008002BB8BF5B429845B8BF9846B8F58D
:1095B800FA7F0746A8BF4FF4FA780090B1460196A3
:1095C800B3463446B74D2B88990758D0B44BB64AA2
:1095D80033F8143032F91420022013FB0022039BC5
:1095E8005B429A424FEA440103DB039B9342A8BFC4
:1095F8001346AE4A31F902A0059A32F91420CAEB93
:10960800030303EB020A08F06FFE88B107EE90AA85
:10961800A74BB8EEE70AB2EE048A185D80EE080A96
:1096280007F066FE20EE080AFDEEC07A17EE90AA53
:109638003B7A642203FB0AF393FBF2F33A7F6FF061
:10964800040101FB02FB5B4505DB02EB820293424E
:10965800A8BF13469B46974A52F824100AEB010309
:1096680042F210718B42A8BF0B4693498B42B8BF98
:109678000B4642F82430BA7C53431B1301932D88C0
:1096880005F00303012B38D0854B8C4933F914902E
:10969800009B51F824E093F801C0894B33F914007A
:1096A80080EAE073A3EBE073B3F5206F4FEA84061A
:1096B80016DC09EB89031A0192FBFCF3042290FBE8
:1096C800F2F0181A8644BEF57A5FA8BF4FF47A5EA6
:1096D8007C4B9E45ACBF41F824E041F8243002E0C1
:1096E800002341F824308B597D2693FBF6F6009B26
:1096F800DB7A7343402693FBF6F6AA0711D5019B44
:10970800C8F5FA7208FB09F008FB06F54FF4FA7180
:1097180002FB0B0002FB035590FBF1F095FBF1F502
:1097280005E0EB074DBF019D354648465846644B5A
:1097380033F91420042392FBF3F3634A02F19C01EA
:109748004FEA440A615C4B436FF04F0193FBF1F31E
:1097580097F85110C31808EE103A51B1101DB8EE21
:10976800C80A00EBC400D2ED070A01F08FFABDEE7B
:10977800C08ADFF854E1524B0EF1B8013AF8030001
:109788003AF901302AF8010002B20EF1BC010EF1DB
:10979800C400D31A042293FBF2F2A30051F824C0A8
:1097A800029350F8243041F82420634497F850106D
:1097B80040F824C0134400EE103A59B10EF150009D
:1097C800B8EEC00A00EBC400DEED070A01F05EFA4D
:1097D800BDEEC00A3C4A02F1B40110EE103A095D30
:1097E80001FB03FE18EE101A02F1680029444FF03D
:1097F800200C9EFBFCF3C91A2AF80010029902F10A
:10980800700E084618EE101A40F80E1002F17C018E
:109818005B42455002F188014350009B013300939D
:109828000CB90124CEE61E4B946AB3F90410049BCC
:109838009B790F335B004B435B112149002BB1F936
:1098480004104FF0040091FBF0F0A3EB0000B8BF48
:109858005B42322B797B0BDC1C4B01FB00418B42BA
:10986800A8BF0B461A498B42ACBF9362916201E0D4
:1098780000239362F97801FB00F31649097803295C
:109888004FEAA31329D9B7F84E10B1F5FA7F24D2BD
:109898004842834220DB8B42A8BF0B461DE000BF35
:1098A800F0100020D411002022340020F4270020DA
:1098B8007C8F0108141A0020F0D8FFFFA01900209F
:1098C8002C10002080C1FFFF80190020FEFFFF0F31
:1098D800020000F0901F00200346916A936741F34D
:1098E8004F31B1F5807FA8BF4FF480716FF0FF0052
:1098F8008142B8BF014658180023A2F86C00C2F88C
:109908008410C2F8903007B0BDEC028BBDE8F08F30
:109918002DE9F04F2DED0A8B85B08346039390F81F
:109928005030029101921BB1322BA8BF322300E0C4
:10993800012307EE903AF8EEE7BADFEDDE7ADE4B68
:109948009FEDDECA1B88C7EEABBA002B08BF012308
:1099580007EE903AB8EEE7AAD94B2AEE0CCA1B8854
:109968007BEE8CBA9807CCEE2BBA27D5D54AB2F93C
:109978000030B2F9022083EAE37182EAE270A1EBD7
:10998800E371A0EBE27088420446B8BF0C46B4F518
:10999800E17F16DA88429FEDCCBA05DD002AD8BFF0
:1099A800524207EE902A04E0002BD8BF5B4207EE34
:1099B800903AF8EEE77A87EE8BBA04E09FEDC3BAE7
:1099C80001E0B7EE00BAC24EDFEDC09ACDF800B0A4
:1099D80006F1080806F1100906F11C050024F0EE4E
:1099E80069AABC49DFF8D8A231F91430B54909EEA3
:1099F800103AB8EEC99AF5EE047A29EE279A31F9A9
:109A08001430BAF80010BDEEC99A08EE103AF8EE14
:109A1800C97A9FEDB19A89074FEA440727EE899AD8
:109A2800B8EEC88A00F08180AC4931F9143007EEED
:109A3800903AF8EEE77AB0EE007AE8EE077A019B02
:109A48005842FDEEE77A17EE901A814203DB8B420B
:109A5800A8BF0B461846A249039B795E401A33F902
:109A68001410084407EE900AF8EEE78A08F03CFC68
:109A780048B19C49F2EE049A88EEA90A085D07F0FD
:109A880037FC60EE298A9BF81C30DFED976A0AEEF6
:109A9800903A9BF8083007EE903AF8EE677AF8EEBD
:109AA8006AAA68EEA77AB1EE047A67EEA67A2AEE79
:109AB800877AFDEEE77A17EE901AF1EE477AFDEE17
:109AC800E7AA1AEE903A994208DBFDEEC7AA1AEE09
:109AD800903A8B42A8BF0B460AEE903AD5ED007A31
:109AE800E8EE8C7ABBEE0E7AF4EEC77AF1EE10FA55
:109AF800F8EEEAAA09D4B3EE0E7AF4EE477AF1EE5C
:109B080010FAC8BFF0EE477A01E0F0EE477AC5EDEB
:109B1800007A9BF8123009EE903AF8EE699A67EEEF
:109B2800A97ADFED729A67EEA99ABAF80010CA0707
:109B380053D46848385E0028B8BF4042B0F5206F5B
:109B480003DD0020C9F8000026E0009B9FED687A3D
:109B58005B7868EE077A07EE103AB8EE477A87EE38
:109B6800877AD9ED007A37EE497AE7EE0C7A9FEDDD
:109B7800617AF4EEC77AF1EE10FA09D49FED5E7AB5
:109B8800F4EE477AF1EE10FAC8BFF0EE477A01E03A
:109B9800F0EE477AC9ED007A009BD9ED007ADB7ABE
:109BA80008EE903AF8EE688A8B0768EEA77ADFED40
:109BB800538A67EEA88A14D538EE6A8AF0EE6A7A74
:109BC800EBEE087A78EEE98AB0EE678AF0EE697A09
:109BD800EBEE287AF0EE678A03E0F0EE698AB0EEE1
:109BE8006A8A474B9FED477A03F19C01625C9BF8B8
:109BF800511007EE902AF8EEE77A67EEC97AA7EED9
:109C0800878A51B1181DB0EE480A00EBC400D3EDA5
:109C1800070A01F03BF8B0EE408A96ED007ADFF8CB
:109C2800E0A0D8ED007AA6EC019A39EE477A0AF15D
:109C3800B40187EE0C7A635C09F10409043509EE76
:109C4800103A37EE677AB8EEC99AEBEE877A38EEB3
:109C5800280AE8EC017A67EE897A9FED2B9A27EEBD
:109C6800899A30EE490A0CF0F3FB0AF16801BDEE5F
:109C7800C88AC85318EE103A0AF17001FDEEE88A56
:109C8800B1EE499A41F82430BDEEC99A0AF17C0137
:109C980018EE903A41F8243019EE103A0AF188018A
:109CA800574641F82430009B0133009374BB0124CC
:109CB80097E600BF83F9223E00100020BD378635A5
:109CC800D4110020F01000200000E1430000000043
:109CD8004C1A00202C100020CDCC4C4022340020FF
:109CE800F42700207C8F01086F12033C0AD7A33D9C
:109CF8000000A043000040C3000040430AD7233CB3
:109D080080190020A69B443BF7CC9238029A584B06
:109D18009479B3F90430640028345C43554BB3F9A3
:109D2800043000EE103ABAEECF0A0CF091FB641141
:109D3800201A002C07EE900AB8BF6442322CF8EEC5
:109D4800E76A03DD0023CAF8283029E0BDEECAAA75
:109D58001AEE103A23F0030307EE903AB8EEE7AA9A
:109D6800DFED457A9BF80D30CAEE277A07EE103AF8
:109D7800B8EE477ADAF8283026EE877A67EE277A3F
:109D8800FDEEE77A17EE902A13443C4A9342A8BFA7
:109D980013463B4A9342ACBFCAF82830CAF8282079
:109DA800BB6A5B13B3F5807FA8BF4FF480736FF075
:109DB800FF029342B8BF134607EE903AF8EEE78ADF
:109DC800FDEEE67A9BF8032017EE903A53439B1179
:109DD80007EE903A2B4B1B78032BB8EEE78A14D981
:109DE800BBF84E20B2F5FA7F0FD2FDEEC87A534287
:109DF80017EE901A994204DB914217EE903AA8BFE9
:109E0800134607EE903AB8EEE78A9BF8511079B1FD
:109E18004B0803D09942A8BF194600E00121B0EED3
:109E2800480A1948D7ED070A00F030FFB0EE408A1B
:109E380038EE280ABDEEC00A8DED000ABDF90030E3
:109E480000EE103AB8EEC00A0CF002FBBDEEC88A6C
:109E5800FDEEE88A0023A7F86C0087ED1E8AC7ED9F
:109E6800218AC7F8903005B0BDEC0A8BBDE8F08FA9
:109E7800F01000202C10002000803B45FEFFFF0F53
:109E8800020000F0901F00209419002038B5294DD9
:109E98002DED048B95ED008AB0EE480A044601F0DA
:109EA800BBF9F0EE408AB0EE480A01F052F995EDA0
:109EB800019AB0EE408AB0EE490A01F0ADF9F0EE31
:109EC800409AB0EE490A01F044F994ED017AD4EDD4
:109ED800027A94ED006A68EE676A27EE088AE7EE70
:109EE800286A68EE000A67EE807AE6EE290AB0EE84
:109EF800660AE7EEA80A0CF0ADFBDFED0F7A0F4B10
:109F080020EE270ADFED0E7A80EE270AD3ED3C7AA1
:109F180030EE270AF2EE047A80EE270A0CF098FA5F
:109F2800BDEC048B83B21A0444BF00F5B47083B24D
:109F380018B238BDF42100200000E1448019002047
:109F4800DB0F494001380A4B042804D8DFE800F049
:109F58000507090B0D00074A08E0074A06E0074A0B
:109F680004E0074A02E0074A00E0074A1A6070471F
:109F780084000020152301088D8F00084126010860
:109F88004D9200088595000819990008437913F047
:109F980001031FBFC36803F1FF32C369006A1DBF15
:109FA800181A1040C0B21846704790F83B3210B5E6
:109FB8007BB990F83A3290F83942A34209D2B0F806
:109FC800401201229A400A430133A0F84022DBB232
:109FD800F3E710BD8379DB07D0F8343144BFB1FA19
:109FE80081F149095A681B8909B193617047138542
:109FF80070476E4B6E4A9FED6F7AD2ED007ADFEDB7
:10A008006E4ADFED6E3A30B51C88B3F90AE01D8A56
:10A0180006EE904AB8EEE76AF8EE666ADFED687A0F
:10A02800B3F9044067EEE67AB7EE004AE6EE077A3F
:10A038009FED647A67EE666A9FED637AE6EE076ADB
:10A0480027EEA77A07EE904AB3F902409FED5F6AC0
:10A05800F8EEE77A67EE277A07EE104AB8EEC77A85
:10A06800DC89E6EE877AB6EE007AFDEEE76A87EEDF
:10A07800866AC3ED066AF8EEE66AD2ED017A9A8935
:10A08800E6EE874A06EE90EAB3F908E09FED507ACB
:10A0980005EE90EAF8EEE66AF8EEE55A66EEA46A8E
:10A0A80065EEA45A66EEA46AB3F806E0E6EE875AAF
:10A0B80065EE875AA5EEA34AF0EE445A04EE10EA7C
:10A0C800B8EE444A25EE844AB5EE404AF1EE10FA5D
:10A0D8005BD02DB205EE905A24B224EEA45A07EEB6
:10A0E800104AF8EEE55A12B265EE255AB8EEC75A8C
:10A0F80065EEA35A64EE854AB0EE007AE4EE875A1C
:10A10800B5EE007A65EE875A07EE102AB8EEC75A00
:10A118009FED307ADFED306AB3F91620E5EE075A85
:10A12800F8EEE77A9FED2D7A76EEE77ADFED2C6A86
:10A13800E5EEC77A05EE902AB0EE677ADFED297A68
:10A14800B3F91420B3F9123067EE277A07EE102A14
:10A15800C7EE847AF8EEE55AB8EEC77A65EEA75AE4
:10A1680027EE877A65EEA75A27EE237AA5EEA67A18
:10A17800F0EE476A07EE103AB8EEC77A36EE877AFD
:10A18800DFED196AE7EE267A01E0DFED187A18B1FB
:10A19800FDEEE77AC0ED007A31B1FDEEC67A6422B1
:10A1A80017EE903A53430B6030BD00BF9802002071
:10A1B800741A00200000003700007AC70000003839
:10A1C800000000390000803A000080380000A045F7
:10A1D80000000036000080470000804900008039F8
:10A1E800000000300050C3450000803D0000000022
:10A1F800704770471FB50123ADF80830ADF804105B
:10A20800002301A9ADF80A30ADF80C30ADF80620EE
:10A2180002F0DFFC05B05DF804FB38B5A0F5137457
:10A228006379A579DB0744D594F8383205F0010540
:10A23800EBB1226B1068C36A5B08436294F83C3246
:10A2480023B1B4F842320133A4F84232917A6A0059
:10A25800FFF7D0FF012384F83B32002384F839321A
:10A2680084F83A3284F83832A4F8403238BD94F889
:10A278003B32012B04BF94F8393284F83A32204635
:10A28800FFF793FE94F83B22236B3AB9012284F836
:10A298003B221868997A05FA02F207E0002284F84E
:10A2A8003B2295421868997A08BF0222BDE83840D7
:10A2B800A0E738BD10B5A0F5127494F83C22BAB9DD
:10A2C800A36A616A994228D0591CA069A162C35C3B
:10A2D8002069DBB25B0043F400738142A4F83E328C
:10A2E8004FF00A0384F83D3228BFA262012312E02E
:10A2F80094F93D327BB1B4F83E124B08A4F83E32D3
:10A30800204601F00101FFF765FE94F83D32013B5C
:10A3180084F83D3201E084F83C3294F83832002B5E
:10A328004ED194F839320133DBB2092B84F8393233
:10A3380003D12046BDE8104037E60A2B40D194F8F7
:10A348003B322BB9B4F8403243F00103A4F8403251
:10A358006379D9071CD5B4F84002820501D4C30734
:10A3680005D4B4F844320133A4F8443210E0E36A67
:10A37800C0F347000BB198470AE0E3696269D0541B
:10A38800E369E1680133B3FBF1F201FB1233E361E6
:10A39800012284F8382294F83B220023012A84F809
:10A3A80039320DD1A27984F83B32236B12F0010FB8
:10A3B8001868997A0CBF02220022BDE8104019E7FC
:10A3C80010BD7620F421312205F0C8B913B5062254
:10A3D80004466B4603211E2005F044F99DF8002031
:10A3E8009DF801309DF8021043EA02231BB21B4A74
:10A3F80007EE903A92ED007AF8EEE77A67EE877A00
:10A4080092ED027AFDEEE77A17EE903A23809DF8F6
:10A41800033043EA01231BB207EE903AF8EEE77ADD
:10A428009DF8041067EE877A92ED017AFDEEE77ADF
:10A4380017EE903AA3809DF8053043EA01231BB23A
:10A4480007EE903AF8EEE77A67EE877AFDEEE77A5C
:10A4580017EE903A638002B010BD00BF24000020C0
:10A4680007B5F7216B460622762005F0FBF89DF824
:10A4780000309DF801100C4A1B0343EA01139DF8B4
:10A48800021043EA111353609DF803309DF804103D
:10A498001B0343EA01139DF8051043EA11131360E7
:10A4A80003B05DF804FB00BF741A00201FB5044612
:10A4B80002210C2001220DF1070305F0D3F8C8B3DF
:10A4C8009DF80730DB0735D50321062202AB0C20A7
:10A4D80005F0C8F80C20092101220DF1070305F049
:10A4E800C1F838B39DF8073013F00C0F22D19DF84E
:10A4F80009209DF8083043EA0223C3EB83339B000D
:10A508009DF80B2023809DF80A3043EA0223C3EB11
:10A5180083339B009DF80D2063809DF80C3043EA3F
:10A528000223C3EB83339B00A3800C200A21012262
:10A5380005F014F904B010BD07B50A2100220C205B
:10A5480005F00CF9142001F07AFA0A210F220C20E8
:10A5580005F004F90A2001F072FA01AB1021032278
:10A568000C2005F07FF80A2001F069FA0A21002280
:10A578000C2005F0F3F80A2001F061FA0DF103034D
:10A58800022101220C2005F06DF80DF103030921C9
:10A5980001220C2005F066F80A2101220C2005F0A2
:10A5A800DDF803B05DF804FB074B1B681869074B1F
:10A5B80020F01F0200F01F01D25801238B401A42DD
:10A5C80001D002F041BA7047B802002014040140DB
:10A5D8002DE9F0437C4A136887B0904693B11A6816
:10A5E8001AB17A49486902434A619A88ADF800204D
:10A5F80002228DF803209868002269468DF802200F
:10A6080004F01AFF322001F01AFA002111221E204C
:10A6180005F0A4F8012160221E2005F09FF86420AF
:10A6280001F00DFA02A8FFF7D1FE00240A272646FA
:10A638002546022101221E2005F090F8322001F063
:10A64800FEF902A8FFF7C2FEBDF90820BDF90A10FD
:10A65800BDF90C308A421444A8BF0A4693421D44EF
:10A66800A8BF134613F5805F0E4404DD013FE0D117
:10A678004FF0010901E04FF000091E2000211222CD
:10A6880005F06CF80A27022101221E2005F066F861
:10A69800322001F0D4F902A8FFF798FEBDF908208E
:10A6A800BDF90A10BDF90C308A42A4EB0204A8BF18
:10A6B8000A469342A5EB0305A8BF134613F5805F2E
:10A6C800A6EB010602DD013FDDD101E04FF00009F4
:10A6D80007EE904A9FED3E7A3E4FF8EEE77A00216A
:10A6E800C7EE277A70221E20F0EEE77AC7ED007ACF
:10A6F80007EE906AF8EEE77AC7EE277A9FED367A8A
:10A70800F0EEE77AC7ED017A07EE905AF8EEE77AAD
:10A71800C7EE277AF0EEE77AC7ED027A05F01EF861
:10A72800012120221E2005F019F81E2002210022F6
:10A7380005F014F8642001F082F9B9F1000F04D192
:10A748004FF07E533B607B60BB60D8F800301E4CF6
:10A758001A7B002A35D01A7D002A32D01B498A6913
:10A7680042F001028A61187B197D02F01DFA236804
:10A778009A689B88128A134223D0184801F004FA79
:10A788002368186902F060F923681B69049300269E
:10A798000C23012504A88DF815308DF814608DF868
:10A7A800165006F037FD23688DF806605B7D8DF83E
:10A7B800043001A803238DF805308DF8075006F002
:10A7C8000BFD07B0BDE8F083B8020020001002407E
:10A7D80000406F462400002001C05E46B1A5000875
:10A7E8002DE9F04F544D1E464FF4147305F108043B
:10A7F800434385B080469146E718A24610B92B44DA
:10A808004E4A03E0012805D14D4A2B449A63103281
:10A81800C3F83C214FF4147303FB08F3EC180AEB5C
:10A82800030203F59C734748A060343253446163C4
:10A83800E261236200224FF0010B4FF48071D4F8DB
:10A848003C3161610320A2626262A1612263E2621B
:10A8580084F8442284F840B284F84122A4F84A22B9
:10A86800A4F84C22C4F810906073A67384F84E8242
:10A8780004F59C7258681B8901924FF0020C03A9D9
:10A88800ADF80C308DF80EB08DF80FC0CDF800C0C3
:10A8980004F0D2FDA36BDDF800C0597B58681B8912
:10A8A8008DF80E1003A9ADF80C308DF80FC004F028
:10A8B800C3FD59463846FFF78DFB322001F0BFF83B
:10A8C800019A214BD2F804B0B3FBF9F1B1F5803FFE
:10A8D80003D3012BF8D95B08F6E74FF4147404FB93
:10A8E80008F805EB0809584689B2482208F5127895
:10A8F80005F0AEFA0AEB0804144BC9F850320022EE
:10A908005846214605F0FAFAD9F8385016F0010FE2
:10A918000CBF022200222868A97AFFF76BFC0C4BB7
:10A92800C9F854322846211D002205F0E7FA3846B6
:10A9380005B0BDE8F08F00BF741A002080A601089A
:10A94800A0A60108808F010800A24A04BDA2000841
:10A9580023A200080F4B73B518781C4698B105233D
:10A968000D4D8DF800304FF4805600238DF80130DE
:10A9780001A82E856946022206F0F8FBAE619DF813
:10A98800050000F0010000F00100207080F00100D7
:10A9980002B070BD2506002000040048064B70B5C3
:10A9A8001D6806461C46FFF7D5FF18B923685B1BD0
:10A9B800B342F8D970BD00BF20280020F7B50323A3
:10A9C8008DF80430030C8DF805308DF80700030A64
:10A9D80006200F4614468DF80630FFF7DFFF78B1E2
:10A9E800084D4FF4805601A904222E85002006F058
:10A9F800BDFB38460021224606F0B8FBAE61204672
:10AA080003B0F0BD00040048024640213C2004F099
:10AA1800A5BE70B500EB8000094CA0F1A1059C38DB
:10AA280025440444074B15F8010F1E787040FFF7C2
:10AA3800EBFFA542F6D13046BDE87040E4E700BF21
:10AA4800988F01082B34002010B5441E14F8010F0C
:10AA580010B1FFF7DEFFF9E710BD024680213C2068
:10AA680004F07CBE10B5D420FFF7F7FF8020FFF775
:10AA7800F4FFA820FFF7F1FF3F20FFF7EEFFD320F8
:10AA8800FFF7EBFF0020FFF7E8FF4020FFF7E5FFA7
:10AA98008D20FFF7E2FF1420FFF7DFFFA120FFF76B
:10AAA800DCFFC820FFF7D9FFDA20FFF7D6FF122016
:10AAB800FFF7D3FF8120FFF7D0FFCF20FFF7CDFFAF
:10AAC800D920FFF7CAFFF120FFF7C7FFDB20FFF708
:10AAD800C4FF4020FFF7C1FFA420FFF7BEFFA62058
:10AAE800FFF7BBFFAF20FFF7B8FFA620FFF7B5FFC2
:10AAF800AE20FFF7B2FF2020FFF7AFFF0020FFF7DF
:10AB0800ACFFB020FFF7A9FF4020FFF7A6FF002009
:10AB1800FFF7A3FF1020FFF7A0FF4FF48064013C6C
:10AB28000020A4B2FFF770FF002CF8D18120FFF7B6
:10AB380094FFC820FFF791FFAF20FFF78EFF012099
:10AB480010BD08B55038C0B2FFF787FF0020FFF7E7
:10AB580084FF1020BDE808407FE7503910B504464F
:10AB6800C8B2FFF77AFF04EB4400400004EB44044A
:10AB780000F00E00FFF771FFC4F3C3001030BDE80A
:10AB880010406AE7F0B50124B0FBF4F58D4201D31B
:10AB98004C43F9E70026D4B1B0FBF4F504FB1500EB
:10ABA800B4FBF1F41EB9002D01DC002CF3D1092D02
:10ABB80003F1010EEFB204DD002A14BF3725572533
:10ABC80000E030253D441D7001367346E3E71C70F4
:10ABD800F0BDF0B50124B0FBF4F58D4201D34C4330
:10ABE800F9E70026D4B1B0FBF4F504FB1500B4FB7B
:10ABF800F1F41EB9002D01DC002CF3D1092D03F16D
:10AC0800010EEFB204DD002A14BF3725572500E0F6
:10AC180030253D441D7001367346E3E71C70F0BDD6
:10AC280003685A1C0260197070472DE9F843089EA2
:10AC3800002B07468846144614BF4FF030094FF0E2
:10AC48002009334613F8012B0AB9254603E0002CE6
:10AC5800FBDD013CF6E7002D04DD38464946C047D8
:10AC6800013DF8E724EAE4743546A01B284415F8AA
:10AC7800011B11B13846C047F7E7BDE8F883024B1E
:10AC8800186800F0A0BF00BFF00F002090ED017A17
:10AC980007EE901AB5EE407AF1EE10FA01BFF8EE21
:10ACA800E77A9FED0E7A67EE877AB7EE007A04BFEF
:10ACB800C7EE277AC0ED017A90ED017AD0ED007ADF
:10ACC80030EE877A30EE670AC0EE870AE0EE807AC7
:10ACD800B0EE670AC0ED007A704700BFDB0FC940CD
:10ACE80010B50278202A034600F10100F9D0092A9C
:10ACF800F7D02D2A03D10346BFEE000A04E02B2A21
:10AD080008BF0346B7EE000ADFED387A1A46134645
:10AD180012F8010BA0F13001CCB2092C0AD807EEC9
:10AD2800101AB8EEC77AF2EE046AA7EEA67AF0EE29
:10AD3800477AECE72E2816D1F2EE046A1146B0EEF7
:10AD4800666A0B4611F8012B303AD0B209280AD8A6
:10AD580007EE102AB8EEC77A87EE267A66EE866A7C
:10AD680077EE877AEDE71A7802F0DF02452A35D1C7
:10AD78005A782D2A02D10233012004E02B2A14BF6D
:10AD8800013302330020013B002213F8011F303940
:10AD9800CCB2092C03D80A2404FB0212F5E7B2F559
:10ADA8009A7F28BF4FF49A721346B7EE007A072BA2
:10ADB80005D9DFED0F6A083B27EE267AF7E702F0A0
:10ADC80007032BB1F2EE046A27EE267A013BF8E777
:10ADD800F0EE476A20B1C7EE877A03E0F7EE006A23
:10ADE80067EEA67A20EE270A10BD00BF000000001B
:10ADF80020BCBE4C30B52DED028B87B0B0EE408A3A
:10AE08000C220021054603A80BF013F9B5EEC08A01
:10AE1800DFED2A7AF1EE10FACCBF38EE278A38EE49
:10AE2800678ADFED277A28EE278A6946FDEEC87A19
:10AE380017EE904A84EAE470A0EBE47006F092FC06
:10AE4800002CACBF20232D2368468DF80C300BF066
:10AE580034F9012807D130238DF80D308DF80E30E4
:10AE68008DF80F300CE0022805D130238DF80D3015
:10AE78008DF80E3004E0032804BF30238DF80D3020
:10AE8800694603A80BF0FCF803A80BF016F9033881
:10AE9800C4B2224603A928460BF03CF900232B55DF
:10AEA800284608490BF0ECF803AB284619190BF0B3
:10AEB800E7F8284607B0BDEC028B30BD6F12033AA5
:10AEC80000007A4454AE010870B506461546084697
:10AED800B6FBF2F414B12046FFF7F6FF05FB146445
:10AEE800024B1B5D00F8013B70BD00BF56AE010868
:10AEF8002DE9F04F814689B08A4616461C46002542
:10AF08003178002900F0DD80252902D00136484635
:10AF180075E07278302A08BFB278A2F1300319BF01
:10AF2800B71C4FF0000BF71C4FF0010B092B4FF02B
:10AF3800000819D8A2F13003D9B2092905D80A2284
:10AF480002FB083817F8012BF4E7A2F16103052B7F
:10AF580002D8A2F1570305E0A2F14103052B03D85B
:10AF6800A2F137030A2BEADD6C2A31D13A78642A38
:10AF780007F1010600F083800BD8252A3DD003D8BD
:10AF8800002A00F09E80BBE7582A0CD0632A19D00B
:10AF9800B6E7732A22D002D86E2A37D0B0E7752ACE
:10AFA8005CD0782AACD1271D2068A2F158046242EF
:10AFB8004FF01001624155E02CD9582A32D0632A4B
:10AFC8002AD13E4648462178271DD04701350FE053
:10AFD800642A64D00ED9732A14D13E46236800939C
:10AFE8004846514642460023FFF71FFE271D0544E9
:10AFF8003C4685E7252ADFD13E4648462521D047ED
:10B0080001357DE70AD86E2A06D13E462368043406
:10B018001D6075E7002A54D03E4671E7752A26D090
:10B02800782AF9D1A2F1580304F1040C5A42206895
:10B03800CDF80CC04FF010015A4105ABFFF7A2FD47
:10B04800DDF80CC03E46644605AB009348465146C1
:10B0580042465B46FFF7E9FD054451E72068271D96
:10B068000A21002205ABFFF7B4FD3C46ECE704F1EA
:10B07800040CCDF80CC020680A210022DDE7206806
:10B08800002804F1040708DA2D238DF81430404213
:10B098000DF115030A210022E5E705ABFAE7206860
:10B0A800002804F1040C0ADA2D238DF814304042EC
:10B0B8000DF11503CDF80CC00A210022BEE705AB3F
:10B0C800F8E7284609B0BDE8F08F0EB40FB505AB18
:10B0D800019053F8042B0649039301A8FFF708FFD2
:10B0E800019B00221A7004B05DF804EB03B07047AE
:10B0F80029AC00080FB413B50B4904AB08680B4919
:10B1080053F8042B09680193FFF7F2FE0446084B35
:10B11800186800F04CFD0028F9D0204602B0BDE8C0
:10B12800104004B0704700BF040100200001002057
:10B13800F00F002080EAE073A3EBE0738B4206DB9C
:10B14800002801DD401A704702D0084470470020EB
:10B158007047FDEEC07A17EE903A2033402B43D863
:10B16800DFED237AB4EEE70AF1EE10FA04DDDFED45
:10B17800217A30EE670AF3E7DFED1F7AB4EEE70ACB
:10B18800F1EE10FA04D5DFED1B7A30EE270AF3E76B
:10B19800DFED1A7AB4EEE70AF1EE10FA04DD30EECC
:10B1A800670A37EEC00A0AE09FED157AB4EEC70ABF
:10B1B800F1EE10FA44BF30EE270A37EE400A60EE8F
:10B1C800007ADFED106A9FED107AA7EEA67ADFED20
:10B1D8000F6AE7EE876A9FED0E7AA7EEA67A20EE51
:10B1E800276AA6EE070A70479FED0A0A704700BF54
:10B1F800DB0F4940DB0FC940DB0F49C0DB0FC93FFC
:10B20800DB0FC9BF9A7C2E36FAAF4FB93587083C99
:10B21800A4AA2ABE00000000DFED027A30EE270A59
:10B2280097E700BFDB0FC93F38B52DED068B90EDD2
:10B23800008AB0EE480A0C460546FFF7EDFFB0EE6F
:10B2480040AAB0EE480AFFF784FFD5ED018AB0EEB8
:10B25800409AB0EE680AFFF7DFFFB0EE408AB0EE22
:10B26800680AFFF776FFD5ED02AAF0EE408AB0EE45
:10B278006A0AFFF7D1FFF0EE409AB0EE6A0AFFF7CC
:10B2880068FF60EE0A6A69EE297AF0EE665AE7EE20
:10B29800A85A29EE8A6A29EE007A69EE889A29EE78
:10B2A800489A28EE400A28EE0A8AC4ED035AF0EEBE
:10B2B800465AE7EE685AE6EEA87AA6EE687AC4ED32
:10B2C800009AC4ED028A84ED059A84ED088ABDECE3
:10B2D800068B84ED010AC4ED045A84ED067AC4EDA8
:10B2E800077A38BD10B52DED048B8AB090ED009A21
:10B2F800D0ED028A90ED018A0446084601A9FFF7BD
:10B3080093FFDDED047A9DED017A68EE277AE9EE88
:10B31800077A9DED077AE8EE877A9DED027AC4ED0B
:10B32800007ADDED057A68EE277AE9EE077A9DED79
:10B33800087AE8EE877AC4ED017ADDED067A28EE20
:10B34800278ADDED037AA9EE278ADDED097AA8EED2
:10B35800A78A84ED028A0AB0BDEC048B10BD074BA6
:10B368001A8822EA0000904210B518801C4602D0C4
:10B37800012000F0BFFB208810BD00BFD4110020C1
:10B38800064B1A881043904210B518801C4602D00C
:10B39800012000F0AFFB208810BD00BFD4110020B1
:10B3A800024A936823EA000090607047202C00202E
:10B3B800024A936818439060704700BF202C002011
:10B3C80008B5104B1A780023D9B2914207D20E491A
:10B3D80051F823100968002008600133F4E732208F
:10B3E80000F02DFB094B1B685A0309D5084B9B68D5
:10B3F8005B0305D440F2DC50BDE8084000F01FBBF9
:10B4080008BD00BF901F0020601F0020FC270020FF
:10B41800202C0020454A69232DE9F34113704FF48D
:10B42800FC635380BE231371EF2382F8DD370023BA
:10B4380082F8DE3719461646F25C0133B3F5FC6F25
:10B4480081EA0201F8D1394B83F8DE17384B1A69C3
:10B45800120604D5374A5A6002F188325A60042726
:10B468000020013F17F0FF074FD0314B3422DA603C
:10B47800002444B1002356F80480019301F038FAFF
:10B488000428EED117E001F033FA0428E9D1284D59
:10B498002B6943F002032B61274B6B612B6943F047
:10B4A80040032B6101F024FA2B69042823F00203DE
:10B4B8002B61DFD0D5E71E4D2B6943F001032B61CB
:10B4C80004F1006303F57E331FFA88F21A8001F055
:10B4D8000FFA042810D1194B23440193019B4FEA1A
:10B4E8001848A3F8008001F003FA2B69042823F018
:10B4F80001032B6105D0B4E72B6923F001032B610D
:10B50800AFE70434B4F5FC6FB3D1094A13690428D2
:10B5180043F08003136102D105F0A3F910B90A20A2
:10B5280000F000FB02B0BDE8F08100BF202C002035
:10B53800002002402301674500F8030802F80308C9
:10B5480010B50E4C206800F0D9F92068047A002262
:10B5580002FB02F3193B634303F6C4135343192157
:10B5680093FBF1F3064921F812300132072AEFD193
:10B578000449BDE81040FCF7EBBA00BF701000208A
:10B58800C00F0020642D00202DE9F04105F069F975
:10B5980010B90A2000F0C6FAA44CA549A54D4FF4ED
:10B5A800FC6220460AF03AFD94F8B437022B84BFB7
:10B5B800002384F8B43794F8B4274FF4CC7101FB16
:10B5C80002F3E018234400F53B70286093F8400329
:10B5D80003F54E73022801FB024284BF0020187253
:10B5E80092F84033944A13700C2202FB0343934AA7
:10B5F80003F2B6731360A26846F2090313401BB93D
:10B608004FF40050FFF7D4FEA368D80703D54FF4D2
:10B618000050FFF7C5FEA368590409D50820FFF7B5
:10B62800BFFE4FF40050FFF7BBFE0120FFF7B8FE46
:10B63800A3681A0706D54FF40050FFF7B1FE0120A2
:10B64800FFF7AEFEA3689B0402D54020FFF7A8FED3
:10B6580094F8DC21754B2AB193F8E02112B100224D
:10B6680083F8E021764B774E1E604FF0000C67465A
:10B6780004EB0C03B3F8F4E14FEA5E0101F0773113
:10B688004FEA9E0303F03333C1EB0E00C11A4FEAB1
:10B69800DE0303F01133CB1A03EB23131EF001086A
:10B6A80003F00F324FF0FF0392FBF3F3C3EB0323D6
:10B6B80018BF0137A2EB030318BFFFB2012B0ADD45
:10B6C800022B40F0B080B8F1000F00F0AC801EF003
:10B6D800BC0F00F0A8800CF1080CBCF1280FC7D1F2
:10B6E800013F012F00F29F80FFF72AFF302200213F
:10B6F8005548564F0AF09DFC554BD5F800801F6001
:10B70800544B002108F17900C3F8008000F036F9A5
:10B71800514B80F001001870504B07F126021A6057
:10B728004F4B07F1D8021A6098F80000FEF70AFCA0
:10B7380028684C4B00F5C5721A60FCF755FE4A4B59
:10B74800DFED4A6A07F194021A60494B00221A8019
:10B758009A71484B07F12C021A602B68464A93ED00
:10B76800187A03F219111160444A03F28911116021
:10B77800434A07F108011160424A1760424A07F13B
:10B788009C011160414A07F1A601116040495361CB
:10B7980067EE266A0E60B6EE007AB4F8661187EE98
:10B7A800267A101D07EE901AB4F86811F8EE677A39
:10B7B800C2ED027A07EE901A93F85C10117193F8B3
:10B7C8007810517194F8DF111174F8EE677AB3F8B4
:10B7D8001611C2ED037A07EE901A2E492E4A086018
:10B7E80003F1640111602D4A2D4982ED007AF8EECB
:10B7F800E77A9FED2C7A2C4A0B60C7EE277A2B4903
:10B808009FED2B7A67EE877AC2ED007A03F1680222
:10B818000A60284903F211130B60274B1F60274B5E
:10B828001A60BDE8F08101F037F85DE7202C0020B0
:10B8380000F803084810002060280020701000203D
:10B84800142C0020AA2D0020F40E0020642D0020C6
:10B85800280F00202C0F00200C000020442100207D
:10B8680004060020380F0020E80E0020DB0F4940B6
:10B87800340E0020A0210020BC24002064090020F0
:10B88800AC200020B0200020780800201C1F0020D9
:10B898003C090020D421002014220020102200207E
:10B8A8009807002000006144740800208C070020DD
:10B8B8004C3D0F44640800206C08002094060020CA
:10B8C80008B5FFF7A7FDFFF75FFE0120BDE80840B8
:10B8D80000F010B9034B4FF4004208B19A61704769
:10B8E8001A85704700080048034B4FF4004208B11E
:10B8F8001A8570479A6170470008004810B5447867
:10B908000078002202FB02F3193B634303F6C413D9
:10B91800534340F6C411434393FBF1F3034921F821
:10B9280012300132072AEDD110BD00BF341F0020AC
:10B938000430114B33F91000B0F5617F10B506DB08
:10B9480040F6330398420246A8BF1A4601E04FF476
:10B9580061720C78192340F2833013FB040494427B
:10B9680007DA497813FB01039342B4BF0020012092
:10B9780010BD002010BD00BF3828002010B500F110
:10B98800500302788A4203D18478C278944204D35F
:10B9980004309842F5D1002010BD012010BD1FB51C
:10B9A800084B1B681B030AD58DF8040001230D20E2
:10B9B80001A98DED030A8DF80530FAF7B9FE05B037
:10B9C8005DF804FBFC2700201FB5084B1B681B0310
:10B9D80009D58DF80400029100230D2001A98DF8E6
:10B9E8000530FAF7A5FE05B05DF804FBFC2700203A
:10B9F80010B50A4A0A4B11689B6800BF1268914249
:10BA0800F7D1084A14694FF47A7000FB04F2D31A8C
:10BA1800B3FBF4F300FB013010BD00BF2028002069
:10BA280010E000E0341F002038B50446FFF7E0FFBF
:10BA38000546FFF7DDFF401BA042FAD338BD10B51D
:10BA480004462CB14FF47A70FFF7EEFF013CF8E79B
:10BA580010BD024A13680133136070472028002084
:10BA6800054B5A6910B51C4602B19047A36913B13A
:10BA7800BDE81040184710BD341F0020014B1B685B
:10BA8800184700BF1034002010B50020FFF7F6FF5C
:10BA9800054B00241C7007F087F9044B1C771C62C7
:10BAA8009C849C6210BD00BF182C0020341F00200D
:10BAB80010B510B9BDE81040E6E700230C225A4340
:10BAC8000A4C1119125D824203D00133102BF5D1B3
:10BAD80010BD074B986A18B14A784078824203D261
:10BAE800002299629A841A6210BD00BFAC970108BF
:10BAF800341F002010B540001428A8BF14200023CC
:10BB0800074A022199540B4499181424834201F8D6
:10BB1800014CF5DBFF21D1540F20BDE81040C7E7E9
:10BB28008C28002038B540F2DB15124B08226843F8
:10BB38009A61851E0B24013C14F0FF0412D00D4AB3
:10BB4800938A9BB283F0080393822846FFF777FF16
:10BB58000120FFF793FF1920FFF771FF0020FFF77F
:10BB68008DFFE8E7044B054A1A60054B054ADA6081
:10BB780038BD00BF00040048FC9F0020EFBEADDECA
:10BB880000ED00E00400FA0506494B690A4623B1B6
:10BB98008B690BB10F20C5E7012302EB83035861C2
:10BBA800704700BF341F002003685B6918470368AB
:10BBB8001B6918470368DB68184703689B681847C0
:10BBC80003685B68184703681B6818472DE9F84F36
:10BBD800B0F90230934218BF00232DED028B18BF35
:10BBE8000370057804460E469146002D40F08B8080
:10BBF80007EE902A9FED770AF8EEE77AB6EE008A0C
:10BC080027EE800ADFED747A20EE270AA04620EEA0
:10BC1800080A0AF093FCDFED716A60EE266AB7EE57
:10BC2800006AB0EE667AA0EE007A40F2DC536365F3
:10BC3800D0EE006A1023A4F8523037EE067A76EE7A
:10BC4800866AC6EE077A1823A4F85030274684ED92
:10BC5800046A27EE807A27EE007A77EE075A84ED99
:10BC6800017AC4ED025A70EE005A84ED037AB8EEF8
:10BC7800007AA5EE807A27EE877A67EEA67A84EDB9
:10BC8800057AC4ED067ADFED567A98ED047A27EE48
:10BC9800277AF0EE678AB5EEC07AF1EE10FA4CBF5B
:10BCA80077EE487A77EE087A013517EE900A07F0B2
:10BCB800F7F8D8ED017A67EEA87AC7E90E01F5EE34
:10BCC800C07AF1EE10FA4CBF77EEC87A77EE887A30
:10BCD80008F1040817EE900A07F0E2F8032DC7E907
:10BCE800080107F10807CED1A6F2DC531B0423672D
:10BCF800E3676367C4F88030A367C4F8843001231E
:10BD0800A4F802902370D4F85490B4F95280636A6E
:10BD1800276A206FE26FD4F840C0D4F88010C4F8C6
:10BD28008020C9EB060606FA08F64FEAE67B73435D
:10BD380007FB0B332667A7FB06671F44636C656F19
:10BD480060674FEAE27B53430CFB0B3EACFB0223DC
:10BD58007344B61A67EB0307E36AA26AC4F884104F
:10BD68004FEAE07B434302FB0B3EA2FB00237344F4
:10BD7800B6185F41E36CA06CB4F95020A5674FEA90
:10BD8800E17B4B4300FB0B33A0FB01011944636BC0
:10BD9800361A206B4FEAE57B05FB03F300FB0B33F8
:10BDA80067EB0107A0FB050119448019794107F0E9
:10BDB8004DF808F1FF3201239340E067C01841EBCA
:10BDC800E371424607F042F8BDEC028B4844BDE8F7
:10BDD800F88F00BF6F12833ADB0F4940F404B53F78
:10BDE8000000804B2DE9F8430024234B93F85C6056
:10BDF800E0B2B0420CD203EB8003204ADB6A32F88F
:10BE080010101BB10B2801D8DB6898470134ECE708
:10BE18001B4B1B685B032DD500242346E2B2B242BC
:10BE280028D2DFF8549009F12C074FEA840857F814
:10BE3800242055689D4215D0284604F033F8EFF3C6
:10BE48001283502282F3128828216A6A01FB00902B
:10BE58000132C0F884206A6942F001026A61DBB2EB
:10BE680083F3118857F808301B6800221A600134E0
:10BE78002B46D3E7BDE8F883341F00204C10002080
:10BE8800FC27002008B50E4B1B6813F4805F0D4B90
:10BE980014BFD3F87821D3F87C2193F85C109288EA
:10BEA8000023D8B2884204D2074820F8132001336F
:10BEB800F7E7FFF797FF3220BDE80840BFE500BF6E
:10BEC800FC270020341F00204C1000200A4B1A6861
:10BED8000A4B30B502F48052D3F87841D3F87C513C
:10BEE80000230AB1A18800E0A988054820F81310AA
:10BEF80001330C2BF5D130BDFC270020341F002066
:10BF08006228002070B5124D0024214605F28110E8
:10BF1800702285F880410AF08CF82146D5F8F43172
:10BF28000B4A0B4493F9020080B102F281141E6897
:10BF38000E5108199C8884809B79837192F880310E
:10BF480007310133702982F88031E7D170BD00BF15
:10BF5800341F0020094B1A680E2303FB0020437A84
:10BF6800FF2B07D0064A12789A4203D9054A32F8BD
:10BF7800130000E0808800B2704700BFBC24002096
:10BF88000C230020382800202DE9F04F2DED048BDC
:10BF9800944C954FD4F8FC31DFF850828DB00646AA
:10BFA80092489847914894F80C22014601F082F88B
:10BFB8003B8804F51772002B73D0D4F810321B7825
:10BFC80008EE103A04F5057904F508754FF0000AF3
:10BFD800B7F800B038F91A00BBF57A7F02BF002322
:10BFE800C9F800302B61D9F800300344C9F8003093
:10BFF8002B6907EE900A0133012B4FEA4A01F8EE4C
:10C00800E77A2B6106D10023C5ED017AC5ED007AE8
:10C01800AB601BE0D5ED006A07EE103A37EEE66A32
:10C02800B8EEC77A86EE077A36EE877AD5ED026AD9
:10C0380085ED017A77EEC77A85ED007AE6EE276A14
:10C04800F0EE667AC5ED036AC5ED026A0023BBF11E
:10C05800010F28F8013053522ED12B69012BC3BF91
:10C0680003F1FF3300EE103AD5ED037A9FED600A35
:10C07800C8BFB8EEC00A8DE80600C8BF87EE800AC0
:10C088000AF08CFC9DE8060018EE103A5BB1F8EE59
:10C09800C87AB4EEE70AF1EE10FA04DD4FF47A73C9
:10C0A8003B8000231CE0D9F800304FF47A7003F588
:10C0B800FA7393FBF0F353520AF1010ABAF1030F32
:10C0C80009F1040905F1140582D1BBF1010F04D16E
:10C0D80058460092FFF7ECFC009A3B88013BDFE7EB
:10C0E80038F8131032F813003E4D091A28F81310C7
:10C0F8000133032BF4D13F4F3B6813F0020300F0E8
:10C10800C9823D4B05F262205B6898473B4B05F2BC
:10C1180062201A78014600F0CDFFB5F8683205F2C2
:10C128006229002B41D0D5F86C020023B4F86822AC
:10C13800334939F913E02B4DB2F5C87F04BF00220B
:10C1480041F823204FEA830C51F80C20724441F83F
:10C158000C20002129F8131020F813100133032BA9
:10C16800E4D1B5F86832012B1AD1D5F870324FF402
:10C17800C87EC83393FBFEF30380D5F87422C83217
:10C1880092FBFEF242801F4AD5F878321288C833F3
:10C1980093FBFEF39B1A838031807180FFF790FB3D
:10C1A800B4F86832013BA4F86832174B1B6859078A
:10C1B80040F18D80B4F87C220A4B322A26D1D3F87C
:10C1C8006C221188A3F87E1251889288A3F88222E3
:10C1D8003288A3F884227288A3F88012A3F88622F2
:10C1E80016E000BF341F0020263400202C10002049
:10C1F800000000000C110020802800202C340020B2
:10C20800A421002020000020FC270020002A3DD087
:10C21800D4F86CC20023B4F87C22AA4939F9130077
:10C22800A94D322A04BF002241F823204FEA830E89
:10C2380051F80E20024441F80E20002229F813205C
:10C248002CF813200133032BE5D1B5F87C32012BF0
:10C2580017D10C2085F8942285F89532FFF728FC31
:10C26800D5F86C32B5F87E221A80B5F880225A804B
:10C27800B5F882229A80B5F884323380B5F88632D0
:10C288007380B4F87C32013BA4F87C3294F896327F
:10C298008D4AE3B1D2F86C52D2F88802002182F8B4
:10C2A80096124FF0320E90FBFEF02880D2F88C02E6
:10C2B80090FBFEF06880D2F89032844A93FBFEF33C
:10C2C80012889B1AAB8031807180FFF7F9FAD4F895
:10C2D8006C22B4F8623211885B1AA4F86232518871
:10C2E800B4F864325B1AA4F864329288B4F86632FF
:10C2F8009B1AA4F86632FFF77BFBD4F8983294EDCA
:10C30800A76AD4F8A062C4F89802C3EB000A07EE43
:10C3180090AAB8EE678A002528EE066A96F800C04B
:10C328006B486C490DF10C0E2A4638F9123007EEAD
:10C33800903AF8EEE77A67EE867AEEEC017ABCF18D
:10C34800000F1CD007EE90CAF8EEE76AB7EE007A45
:10C35800C7EE266A39F9123007EE903AF8EEE77A16
:10C3680037EE667A67EEA67AD1ED006AE6EE877A4E
:10C37800C1ED007AFDEEE77A17EE903A01E039F860
:10C388001230438030F8023F0132032A13FB035571
:10C3980001F10401C9D1DFF834814F4864236B43AC
:10C3A800B8F800506D4393FBF5F5493D03A9ADB2CC
:10C3B800FEF798FF3B2DD6ED016A11D9B4F9BC32CE
:10C3C800D4EDAE0A07EE903AF8EEE77A434BF4EE76
:10C3D800E70AF1EE10FA1EDD1A7842F008021DE0B5
:10C3E800F7EE007A36EEA77A3B4A87EE877A002383
:10C3F8003B4931F913100133032B07EE901A92EDE4
:10C40800006AF8EEE77AE6EE267A67EE877AE2ECDB
:10C41800017AEDD1D2E71A7822F0080294EDAD0A3C
:10C428001A700AF017F9B0EE409A84EDB00A94ED4C
:10C43800AE0AD4EDAD7AD4EDAC8ADFED2A9A2A4D56
:10C4480020EE000AF1EE688AA7EEA70A0AF0A6FA1B
:10C45800F0EE400AB0EE680A0AF0FCF8F0EE408A06
:10C4680084EDB10A29EE290A09F0F2FF28EEA90A9B
:10C47800288009F0EDFF3B6868801A073AD51B4809
:10C4880003A9FEF72FFFD6ED026A184AF7EE007AE5
:10C4980036EEA77A002387EE877A154931F913100B
:10C4A8000133032B07EE901A92ED006AF8EEE77A53
:10C4B800E6EE267A67EE877AE2EC017AEDD10B4850
:10C4C80043E000BFBC210020341F002020000020D2
:10C4D800D8100020D8210020E421002010110020CD
:10C4E800DA1000204C3D0F44F4270020FC210020E6
:10C4F800321000206D4D03A92846FEF7F3FE95ED96
:10C50800010A95ED007AD5ED027A20EE000AA7EE31
:10C51800070AA7EEA70A0AF041FAB5EE400AF1EEBB
:10C5280010FA11D0D5ED007AC7EE807AC5ED007A01
:10C53800D5ED017AC7EE807AC5ED017AD5ED027A9C
:10C5480087EE800A85ED020A5848FDF79FFC584B94
:10C55800DFED587A1880564B9FED577AB3F90030C3
:10C5680028EE278A07EE903A544BF8EEE77AB3F9AB
:10C57800002067EEC77AB1EE499ACDED087A07EE4A
:10C58800902AB3F90220B3F904308DED069AF8EE3B
:10C59800E77AF1EE688ACDED097A07EE902AF8EE8F
:10C5A800E77A09A8CDED0A7A07EE903AF8EEE77A2D
:10C5B80006A9CDED078ACDED0B7AFEF793FE7378C9
:10C5C8009DED0B7A012B19D13D4B1B785B070FD4DE
:10C5D800D4F8D432402293FBF2F29B1A07EE903A39
:10C5E800F8EEE77A77EE877AFDEEE77AC4EDB57A6A
:10C5F800D4F8D432402293FBF2F301E0B8F80030CB
:10C608009DED090A07EE903AF8EEE77A37EE677A79
:10C61800D4EDB67A8DED0B7A94EDB77A38EE077AC9
:10C6280088EE078A9DED0B7A37EE677AE8EE077A8F
:10C63800B0EE678AC4EDB67A09F00AFFD4F8E05282
:10C648002978FEF777FDD4F8E4329DED0A0A1844FC
:10C65800C4F8E40209F0FCFE2978FEF76BFDD4F873
:10C66800E832B0EE480A1844C4F8E80209F0F0FECF
:10C678006978FEF75FFDD4F8EC32124A1844136863
:10C68800C4F8EC0253441360D4F8F0320133C4F810
:10C69800F03205E0A5F86232A5F86432A5F86632F2
:10C6A8000DB0BDEC048BBDE8F08F00BF300000205A
:10C6B800E8100020BD37863535FA8E3CDA100020A8
:10C6C8002A3400200C340020084BDA68D10709D43A
:10C6D800DA68D20608D4DB6813F0040F14BF03200D
:10C6E8000420704701207047022070470020024054
:10C6F80003788B4286BF024B33F811000020704745
:10C708002822002070B5344C0546FFF771F9A3695B
:10C71800A061C31AB3F5FA5FE36182BF002384F80E
:10C72800203084F8213094F820302BB9A12D02BF95
:10C73800294A012182F8211094F82110264A31B1A2
:10C74800D118EDB2013381F8225082F8203094F8E4
:10C75800205094F84330AB423CD11F4B93F84430FF
:10C76800052B02D0062B03D02FE0002006F09AFA02
:10C7780094F823301E2B28D100200246C1B26B1E2C
:10C7880099421ADA214491F822300821DBB283EA6F
:10C798000206F60744BF83F01803C3F3460301F10A
:10C7A800FF3154BF5B0843F0800311F0FF01C2F36F
:10C7B8004702ECD101301A46E0E7234493F82230CF
:10C7C8009A4202D1032006F06DFA002384F8213042
:10C7D80084F8203070BD00BF2822002010B5044620
:10C7E800B0F9000004F01AFCB4F9020004F016FCD9
:10C7F800B4F90400BDE8104004F010BC10B50446BC
:10C80800006804F00BFC606804F008FCA068BDE850
:10C81800104004F003BC2DE9F74F0120FBF792F913
:10C82800002488B3012C2FD8194E4FF04C0909FB6E
:10C8380004FA06EB0A0808F19007BD7815B101342F
:10C84800E4B2EEE790F9003090F804E01846114B96
:10C8580003228DE8240001212A4653F82E30FBF7E5
:10C8680047F8834660B106F14800504429464A46D5
:10C8780009F0DFFB01231C44C8F848B0BB70E4B2E0
:10C888000120FBF745F9CCE703B0BDE8F08F00BF06
:10C89800282200203C92010800212A2210B51148C4
:10C8A80009F0C7FB104B002219461048105C83F8AA
:10C8B800F20104240520013283F8F74182424FF047
:10C8C800000483F8F60183F8F94183F8F80103F1CD
:10C8D8000803EAD10123A1F8F431522381F8F03199
:10C8E80010BD00BF102E0020202C00207BAE0108B8
:10C8F80010B5FFF7E9FE4FF43024012806D11CB12A
:10C90800FFF7E2FE013CF8E7052010BD002C08BF48
:10C91800052010BD70B50646441E14F8011F89B1E4
:10C92800094D284609F0BBFB0028F6D005F108039D
:10C9380098423FBF054B401BC018A31B38BF80F867
:10C948008A31EAE770BD00BF06B80108202C002034
:10C9580007B51C4B03F1E402C3F8E0201A4A92F829
:10C9680092215AB1012A14D1032183F8E610072134
:10C9780083F8E82083F8E7100C2208E0022183F806
:10C98800E610032183F8E82083F8E710072283F8EC
:10C99800E4200E4B0E4A1A604020FBF7D3F870B122
:10C9A8000122002390F9000040218DE80C00094A7B
:10C9B8004FF4E133FAF79CFF003018BF012003B0B1
:10C9C8005DF804FB28220020202C00203C000020D9
:10C9D800652A0108192B01080120002105F028B853
:10C9E800F0B5184A92F8E930D2F8EC701546042BE5
:10C9F80011D807EBC3025E1C941CF6B209D013468B
:10CA08009288D10705D5104203D008E001310529E5
:10CA180008D13346EBE785F8E9300020F0BD93F8FC
:10CA280002E00021074C0C2204F1F00C02FB01F398
:10CA38001CF803209645E9D1234484F8E960D3F82B
:10CA4800F400F0BD2822002020F01F01012300F08F
:10CA58001F00024A83408B50704700BF14040140F6
:10CA680000230360436083608381036143618361C2
:10CA7800C36103624362836270478A68036810B5C2
:10CA88000C6A14430A6914434A6914438A691443B3
:10CA9800CA6914434A6A14438A6A23F4FF4323F099
:10CAA80070032243134303608B8943600B688360E0
:10CAB8004B68C36010BD02684FF6FE7313400360F5
:10CAC8000023036043608360C360294B984201D10F
:10CAD800284A27E0284B984201D1264A2AE0274BCA
:10CAE800984201D1234A2DE0254B984201D1214A91
:10CAF80030E0244B984201D11E4A33E0224B984241
:10CB080004D11C4A536843F470032EE01F4B98422B
:10CB180004D1184A536843F0706326E01C4B9842CE
:10CB280004D11C4A536843F00F031EE01A4B984285
:10CB380004D1184A536843F0F00316E0174B9842A3
:10CB480004D1144A536843F470630EE0144B9842BE
:10CB580004D1104A536843F4704306E0114B9842DD
:10CB680004D10C4A536843F470235360704700BFE4
:10CB780008000240000002401C0002403000024051
:10CB880044000240580002406C000240800002400D
:10CB980008040240000402401C0402403004024021
:10CBA800440402405804024001F0030301F0FC0170
:10CBB80001F1804101F5803110B59B008C680F228E
:10CBC8009A4024EA02028A608A68984002438A608E
:10CBD80010BD0A888B88F0B54C880E89CD88C2B9FB
:10CBE800026A22F0010202628269016A22F0F302FB
:10CBF8001A4342EA061344F0010421F00A021443DE
:10CC080083610462836923F00C03836183691D4394
:10CC18001FE0042A016A1ED14FF6EF720A40026231
:10CC28008269016A1B0222F4734243EA0633240133
:10CC3800134344F010044FF65F720A40A4B2224333
:10CC480083610262836923F440638361836943EAF1
:10CC580005258561F0BD082A1DD14FF6FF620A40FF
:10CC68000262C269076A4FF60C7111404FF2FF5217
:10CC78003A4042EA042443EA06130B4344F480741E
:10CC88009BB2A4B2C3610462C2694FF6F373134046
:10CC9800C361C3691FE04EF6FF720A400262C169B0
:10CCA800026A40F6FF470F4045F6FF7111401A022D
:10CCB80042EA063341EA04343B4344F480549BB2CD
:10CCC800A4B2C3610462C2694FF2FF331340C36167
:10CCD8002D02C369ADB21D43C561F0BD036A23F0DF
:10CCE80001030362036A70B5446882690D6822F41F
:10CCF800803222F0730215438A8923F0020313431A
:10CD08008A881343134A90420FD002F5006290427A
:10CD18000BD002F54062904207D002F58062904243
:10CD280003D002F5806290420DD1CA89CE8823F0E3
:10CD3800080313430A8A24F4407414434A8A23F0EC
:10CD48000403334314438A68446085614263036281
:10CD580070BD00BF002C01409B4A536803F00C03D0
:10CD6800042B2DE9F04105D0082B06D09749016026
:10CD7800B3B916E0954B036012E053685468C3F3E7
:10CD88008343991CE30349BFD36A914B8F4C03F04B
:10CD98000F0344BF0133B4FBF3F34B43036000E0DC
:10CDA800002351688B4FC1F3031139440D79016891
:10CDB800EDB221FA05F444605668C6F302263E44F3
:10CDC800367924FA06FEC0F808E05668C6F3C2268B
:10CDD8003E443679F6B2F440C460D2F82C80C8F3E9
:10CDE800041808F00F0C07EB4C0C18F0100FBCF8E7
:10CDF80014C01FFA8CFC07D0BCF1000F04D0B3FBA1
:10CE0800FCFCC0F810C000E00161D2F82CC0CCF3E3
:10CE1800442C0CF00F0807EB48071CF0100FBF8AD2
:10CE2800BFB204D01FB1B3FBF7F7476100E041611F
:10CE3800176BFF065ABF654F87618161176BBF0685
:10CE48005ABF624FC761C161176B7F065ABF5F4FF8
:10CE580007620162176BFF0506D5994204D1AE42FD
:10CE680002D14F00476200E04462176BFF0406D509
:10CE7800994204D1AE4202D14F00876200E0846239
:10CE8800176BBF0506D5994204D1AE4202D14F00B7
:10CE9800C76200E0C462176B7F0506D5994204D1CA
:10CEA800AE4202D14F00476400E04464176B3F056F
:10CEB80006D5994204D1AE4202D14F00876400E002
:10CEC8008464176BBF0406D5994204D1AE4202D1DF
:10CED8004B00C36400E08464156B3B4BAD0701D184
:10CEE800046315E01C6B04F00304012C01D10163F9
:10CEF8000EE01C6B04F00304022C02D14FF4004333
:10CF080005E01B6B03F00303032B01D12F4B0363D5
:10CF1800146B2D4B14F4403F02D1C0F834E018E0F4
:10CF28001C6B04F44034B4F5803F01D1416310E038
:10CF38001C6B04F44034B4F5003F02D14FF40043B5
:10CF480006E01B6B03F44033B3F5403F01D11F4BA0
:10CF58004363146B1C4B14F4402F02D1C0F838E023
:10CF680018E01C6B04F44024B4F5802F01D18163D0
:10CF780010E01C6B04F44024B4F5002F02D14FF4E8
:10CF8800004306E01B6B03F44023B3F5402F01D1A7
:10CF98000E4B8363146B0C4B14F4401F02D1C0F882
:10CFA8003CE021E01C6B04F44014B4F5801F01D16F
:10CFB800C16319E01C6B04F44014B4F5001F0BD1D5
:10CFC8004FF400430FE000BF0010024000127A0047
:10CFD80000093D003C0000201B6B03F44013B3F52F
:10CFE800401F01D1134BC363126B134B12F4400F54
:10CFF80003D1C0F840E0BDE8F0811A6B02F44002AA
:10D00800B2F5800F02D10164BDE8F0811A6B02F419
:10D018004002B2F5000F02D14FF4004306E01B6B4B
:10D0280003F44003B3F5400F01D1024B0364BDE89C
:10D03800F08100BF00127A0000100240F0B5002312
:10D048000E681C460125A54005EA060EAE452BD103
:10D058000F797A1E012A15D8856803229A4025EA95
:10D06800020282604D7982689D40154385608288FE
:10D0780092B222EA0E0282808A798588A2402A43E7
:10D0880092B28280032205689A40D2431540056017
:10D0980005689F402F430760C7681740CA7902FA9E
:10D0A80003F547EA0502C2600134102C03F10203BC
:10D0B800C8D1F0BD38B52DED048B4A4C0368C4F8CF
:10D0C8002C318388A4F83031013A0D46072A42D81A
:10D0D800DFE802F0040A101822292F35B4F82C31A1
:10D0E8000B80B4F82E3113E0B4F82E310B80B4F86D
:10D0F8002C3105E0B4F82C315B420B80B4F82E31AA
:10D108005B4205E0B4F82E315B420B80B4F82C3159
:10D118006B80B4F830311DE0B4F82C315B420B80E1
:10D12800B4F82E3112E0B4F82E310B80B4F82C315B
:10D138000CE0B4F82C310B80B4F82E3105E0B4F8CB
:10D148002E315B420B80B4F82C315B426B80B4F813
:10D1580030315B42AB80244B93F83430002B3ED106
:10D16800B5F9003094ED500AD4ED4D7A09EE103A35
:10D17800B5F9023008EE103AB8EEC88AB5F90430AD
:10D18800B8EEC99A28EE000A08EE903AA7EE890A86
:10D19800F8EEE88AD4ED537AA7EEA80A09F058F910
:10D1A80094ED510AD4ED4E7A288028EE000AA7EEB5
:10D1B800890AD4ED547AA7EEA80A09F049F994ED42
:10D1C800520AD4ED4F7A688028EE000AA7EE890A41
:10D1D800D4ED557AA7EEA80A09F03AF9A880BDEC73
:10D1E800048B38BD282200203C000020104BDFEDC6
:10D1F800117A1B689A89104B1B6883F31003D31AA2
:10D2080007EE103AB8EEC77A27EE277A07EE902A8B
:10D21800F8EEE77AC7EE277AFDEEE77A17EE900A7E
:10D228006428A8BF642020EAE070C0B2704700BF3D
:10D23800F81000200000C84208110020094B1A68A5
:10D24800137844F6FB7103EB431300FB0313507888
:10D25800C0EB0030B3FBF0F39078B3FBF0F080B292
:10D26800704700BFF810002008B50A4890F85931F7
:10D2780000EB43030A22B3F8681189B2A0F87011D1
:10D2880000F5BC70FEF7A2FC80B2FFF7D7FF024B97
:10D29800188008BD28220020FC10002008B5084886
:10D2A80008F00BFFC0B209280246054B04DC013028
:10D2B8002021C0B29954F6E700221A5408BD00BFD5
:10D2C8004924002008B5074808F0F7FEC0B2142822
:10D2D800044B04D8421C20211954D0B2F7E700228D
:10D2E8001A5408BD492400202DE9F74FA74CFEF732
:10D2F8007FFB26686568A768861BF643451BC71B26
:10D30800ED43FF43F60F8046ED0FFF0F2EB93FB9EF
:10D31800002D00F08682B9462CE04FF0000929E084
:10D32800B14627E003EB8A0BBBF802301A050ED48E
:10D3380013F4805F1DBF964A9BF801101268954A46
:10D34800954B14BF52F82120126843F82A20BBF8E5
:10D358000230D80516D499050AD5904B1B7813F0DE
:10D36800040F0CBF8E4A8F4A8B4B126843F82A2051
:10D3780009F10109207B8C495FFA89FA82450B681B
:10D38800D0D326E0894A5046594602F023FE884BFE
:10D398001B885A0603D550465946864A16E0580750
:10D3A80003D550465946844A10E0190703D550461C
:10D3B8005946824A0AE09A0703D550465946804A98
:10D3C80004E0DB07D4D57F4A5046594602F002FEF6
:10D3D800CEE7DFF808E20093BEF906307822A3F51D
:10D3E8007A7353434FF47A7293FBF2F303F22B13DD
:10D3F80001930022F3465FFA82FE864517D2009B0E
:10D4080003EB820EBEF802E01EF4806F0DD0DFF849
:10D418008891019B39F822E040F2671A9E449EFBEE
:10D42800FAFC0AFB1CEE29F822E00132E3E74DB3CF
:10D4380008F5C333A0336360637B544A13BB93730B
:10D44800614B1B6813F0020F0AD0DFF894E19EF8D5
:10D4580000E0BEF1000F03D04FF0010E82F80EE09D
:10D46800DA0506D5594B5B791BB1A37B43F0020360
:10D47800A3734A4B1B7813F0050F02BFA37B43F03D
:10D488000403A37394F80EE0BEF1000F03D13F4BE1
:10D498005B7B002B4FD094F80DC01CF0010FACF152
:10D4A8000C031DD1BCF1030F07D8DFF8E8903C4A04
:10D4B8001EF0040F08BF4A4600E0364AACF1040CDF
:10D4C800BCF1070F05D8DFF81CC11EF0010F18BF0B
:10D4D8006246DBB2032B0ED81EF0020F3C4B06E06F
:10D4E800DBB2032B06D82F4B2A4A1EF0020F18BFB7
:10D4F8001A4600E0274A4FF0000C5FFA8CF383428B
:10D508000DD20B6803EB8C035B881B0642BF224BD2
:10D51800D2F8009043F82C900CF1010CEDE785B19E
:10D52800BEF1000F08D0637B184A0133DBB2142B1D
:10D5380006D1002304E025B1637B002BF3D100E082
:10D548005373002E52D0234AB2F90250B2F9002088
:10D55800002DB8BF6D42002A4FF03203B8BF5242C7
:10D5680095FBF3F592FBF3F2EDB2D3B2AB4238BFC1
:10D578002B46194A13B192FBF3F300E013464344D8
:10D588002360E37B014A7BBB01232EE02824002093
:10D59800B824002050A70108AA0D00202A34002032
:10D5A8009497010884970108E01100205C92010813
:10D5B800D411002062920108689201086E92010855
:10D5C800749201087A920108FC270020340E00208A
:10D5D8009C970108F0100020400D03003828002017
:10D5E8005C110020A49701080023D3738E4D8F4B44
:10D5F8002D78E27BADB9002F00F00E818C4B267B95
:10D608001A788C4B8C4D93F800C08C4BD3F800E003
:10D618000B6802F004020021D2B203EB86060F4623
:10D62800B5E01AB9864A1A61002508E0854AFAE782
:10D638000A68AB00D6187688760604D40135EBB2B2
:10D648008342F5D3D7E7804EB6F90060192E25DD61
:10D6580012F803E094F814C026690EF00F09E145AA
:10D668000CDCDFF8C8C19CF815C0BCEB1E1FDEBF80
:10D67800DFF8D8E1D6F800C043F80EC012F803E08E
:10D6880094F816C00EF00F09E14533DBDFF89CC1B2
:10D698009CF815C0BCEB1E1F2CDC26E0193629DAD5
:10D6A80012F803E094F814C026690EF00F09E1455A
:10D6B8000CDCDFF878C19CF817C0BCEB1E1FA2BFBA
:10D6C800DFF888E1D6F800C043F80EC012F803E08E
:10D6D80094F816C00EF00F09E1450BDBDFF84CC1DA
:10D6E8009CF817C0BCEB1E1F04DBD6F800E0574EB1
:10D6F80043F806E0544EB6F90260192E1BDD12F805
:10D7080003C094F814E026690CF00F09F1450CDC0D
:10D71800DFF8189199F81590B9EB1C1FDEBFDFF8F8
:10D728002CC1D6F8009043F80C90D25C02F00F0C94
:10D73800F4451EDD82E7193680DA12F803C094F842
:10D7480016E026690CF00F09F1450CDBDFF8DC90D8
:10D7580099F81590B9EB1C1FDEBFDFF8F0C0D6F8BA
:10D76800009043F80C90D25C02F00F0CF445FFF6E1
:10D7780065AF94F817E0BEEB121FA2BF334A3668B4
:10D788009E505BE75888000504D404330435B3423F
:10D79800F8D122E04AB101EB0C0A06209AFBF0F915
:10D7A80000FB19A001280DDC01E057B9012793F807
:10D7B80001900EEB89003EF829A090F80290C078FD
:10D7C80003E01746002081468246013125F802AC65
:10D7D80085F800906870C9B2D7E7164A1378013BFC
:10D7E80013F0FF0308BF06231370114B1B785B0768
:10D7F80041BFBBF90630A3F57A7303EBC3034FF4BB
:10D808007A7243BF93FBF2F30133DBB20123104A70
:10D8180092FBF3F34344A36003B0BDE8F04F01F07B
:10D828002DBD03B0BDE8F08F630E00202824002032
:10D838002A34002074000020AC0D0020B8240020F9
:10D84800A097010850A70108F0100020AA0D002099
:10D85800400D030030B50028104C114AB8BF4042B3
:10D868003C2590FBF2F304FB030068430D4D90FB4D
:10D87800F2F22D682D7B25B903EB830303EB8303B9
:10D8880001E0C3EB031302EB83030B8004FB0202EA
:10D898004FF47A7392FBF3F24A8030BD806967FFD8
:10D8A8008096980000110020022803D0431E584299
:10D8B80058417047064B1B681B7823B1054B186805
:10D8C800C0F3C0407047044B1878C0F3800070471D
:10D8D800040600200C1000202A34002010B50A4C41
:10D8E8005E280146206805D15D21FEF76CF92068A5
:10D8F8003E2105E05D2903D1FEF765F920683D2149
:10D90800BDE81040FEF75FB940240020A0F17D0378
:10D91800012B70B504460D460A4E05D830687D21A6
:10D92800FEF751F984F0200430682146FEF74BF9E0
:10D9380035B12B881C4404EB142404F0FF042C801C
:10D9480070BD00BFC411002010B5054C2068FEF75B
:10D9580037F918B12068FEF730F9F6E710BD00BFB7
:10D968009411002010B50446C0B2FFF7B7FFC4F306
:10D978000720BDE81040B1E7024B5E211868FEF7AA
:10D9880022B900BF4024002038B5064C05465E2168
:10D998002068FEF718F920682946BDE83840FEF7E8
:10D9A80012B900BF4024002013B5044601A900683D
:10D9B800FFF750FF1320FFF7E7FFBDF90400FFF75B
:10D9C800D1FF1B20FFF7E0FFBDF90600FFF7CAFFF4
:10D9D8002320FFF7D9FF2368002BB4BF53204E2024
:10D9E800FFF7C0FF01A96068FFF734FF1220FFF7B7
:10D9F800CBFFBDF90400FFF7B5FF1A20FFF7C4FFFE
:10DA0800BDF90600FFF7AEFF2220FFF7BDFF6368F0
:10DA1800002BB4BF57204520FFF7A4FF02B010BD6C
:10DA2800674B73B51878674DFFF73EFF2B78834235
:10DA3800044620D0C8B1644B1B68E3B193F90000D9
:10DA480002230093614B1B685B78003318BF0123E6
:10DA5800019304214FF416530022F9F749FF5C4B58
:10DA6800186040B101232B7005E0594E3068F9F772
:10DA78002CFF34602C70574B574D1878FFF714FF64
:10DA88002B788342044618D088B1544B1B68A3B145
:10DA98000022012493F9000000944FF49643019268
:10DAA8000821F9F725FF4E4B186028B905E04C4EC0
:10DAB8003068F9F70AFF34602C704A4B4A4D1878E1
:10DAC800FFF7F2FE2B78834204462E4642D0002808
:10DAD80037D0464B1A68002A3CD0D37992F9000017
:10DAE800434C002B08BF022302220092002254F864
:10DAF800233001921021F9F7FBFE3E4B05461860D2
:10DB080040B33D4C94F84A30022B0BD094F8962041
:10DB1800022A01D14C3405E023B1002A04F14C0457
:10DB280018BF0024354B1C6044B1204600214C220C
:10DB380008F07FFA0223256084F84A300123337005
:10DB480008E02C4E306803F01FFF3068F9F7BDFE7F
:10DB580034602C702A4B2B4D1878FFF7A5FE2B78D4
:10DB68008342044629D000B3274B1B682BB3274AAE
:10DB780093F9000012685278002A0CBF0822092283
:10DB88000323009301924FF4614320210022F9F707
:10DB9800AFFE1F4B186080B11E4A012313702B7013
:10DBA8001D4B1A681D4B1A6007E0194E3068F9F7CB
:10DBB8008CFE184B34601C702C7002B070BD00BF16
:10DBC8000C060020D01000200806002000110020BC
:10DBD800402400200D06002020110020A411002060
:10DBE8009411002018060020AA1100201406002015
:10DBF8003C920108AC11002070220020B0110020D6
:10DC080024060020C0110020200600201C06002049
:10DC1800C4110020C811002020280020CC110020A9
:10DC2800642928BF6421F8B510FB01F56424064671
:10DC380095FBF4F40027E4B2FBB2A34204D29F2080
:10DC4800FCF7E7FE0137F7E7B4420BD2C4EB8410C8
:10DC58001421C4EB800095FBF1F5663D2844C0B261
:10DC6800FCF7D7FE0134E4B2B44201D29A20F7E7B8
:10DC7800F8BD2DE9F743934CFDF7BAFE6368C31A64
:10DC8800002BC0F2678300F5433303F5A07363608C
:10DC98008D4B1D78237AC5F38005EB1A18BF012335
:10DCA80025724DB1002B00F05583884B5A789A7035
:10DCB80001225A701A702BE0844A2BB1D37843F0B2
:10DCC8000203D37093785370D67806F0020101F0FE
:10DCD800FF0339B97D498968411A002903DB06F039
:10DCE800010300E0012303F00107784917707BB1B5
:10DCF800F2070DD50A790132D2B20523B2FBF3F34C
:10DD080003EB8303D31ADBB2714A0B71D35C4B70FC
:10DD18006E4EDFF8088233787BB3F37823F0020382
:10DD2800F3706C4B0344AE20B360FCF796FE08B169
:10DD3800FCF798FE88F80000002800F00B83B0205C
:10DD4800FCF78BFE4020FCF788FE0020FCF785FEE0
:10DD58001020FCF782FE4FF48067013F0020BFB21D
:10DD6800FCF752FE002FF8D13846FCF7EAFE72782D
:10DD7800594B53F82200FCF767FE98F80030002B47
:10DD880000F0E8827378062B00F2B382DFE813F024
:10DD98000700B102180078006C018901EE014F49B3
:10DDA8004F4A504B5048FDF790F90120FCF7C9FE47
:10DDB8004D48FCF749FE0220FCF7C3FE4B48AEE194
:10DDC8004B4F3B689B0735D5DFF85481DFF85491FA
:10DDD800B8F8001044480A23B1FBF3F203FB12130E
:10DDE80099F80010009192B242499BB2FDF76DF983
:10DDF800FFF768FA0120FCF7A4FE3B48FCF724FE75
:10DE08003D4B99F800201868B8F80030067906FBF1
:10DE1800123164234B43C1788E1B56430220B3FB57
:10DE2800F6F6F6B2FCF78DFE31461520FFF7F8FE40
:10DE3800032600E001263B681F0540F15A822F4B5C
:10DE48002F491F680968009164232E4997FBF3F254
:10DE5800254803FB1273FDF738F9FFF733FA30460C
:10DE6800FCF76FFE2048FCF7EFFDFFF7BFF9074608
:10DE7800701CFCF766FE15203946FFF7D1FE38E224
:10DE88000120214FFCF75DFE2048FCF7DDFD3B68D3
:10DE9800980749D51E4A1448B2F90210B2F9003061
:10DEA8000091B2F904201B4901921B4AFDF70DF9B4
:10DEB800FFF708FA0220FCF744FE0B48FCF7C4FD04
:10DEC800032632E0402400202A3400207824002051
:10DED80080AE0108404B4C008092010885AE0108D5
:10DEE8008EAE010889A701084924002095AE0108D3
:10DEF800FC270020A0AE0108F81000200411002023
:10DF080008110020B8AE01080C110020CDAE0108A0
:10DF1800DA100020E3AE0108F2AE01087902002011
:10DF2800FC1000208000002002263B68D9071AD583
:10DF38007C4A7D48B2F90210B2F900300091B2F97A
:10DF480004207A4901927A4AFDF7BFF8FFF7BAF937
:10DF58003046FCF7F6FD744806F10108FCF774FD3D
:10DF68005FFA88F846463B681A0718D5714A6E4822
:10DF7800B2F90210B2F900300091B2F904206B49ED
:10DF880001926D4AFDF7A1F8FFF79CF93046FCF7BE
:10DF9800D8FD6548771CFCF757FDFFB23E46674A37
:10DFA8006249B2F90030B2F902200092644A5E4830
:10DFB800B2F900200192634A634FFDF786F8FFF734
:10DFC80081F93046FCF7BDFD5748FCF73DFD97ED5C
:10DFD800000A5548FCF70EFF534808F06EF806F1A2
:10DFE80001085FFA88F8C0B2B946092809D8431C65
:10DFF8002044DBB220224272E218002191721846B6
:10E00800F3E7494F99ED010A3844FCF7F3FEFFF7AF
:10E0180059F94046FCF795FD3846FCF715FD99ED92
:10E02800020A3846FCF7E6FE384608F046F802369B
:10E03800F6B2C0B2092809D82318421CD2B220214E
:10E048005972A318002199721046F3E73F4AB2F9B2
:10E05800003000EE103A3844B8EEC00AFCF7CAFEA9
:10E06800FFF730F9304657E00026394F3B78B34286
:10E0780040F23F810E2E00F03C8170080130FCF721
:10E0880060FD304603F048FB3B78B34206D92020B8
:10E09800FCF7BFFC701CC0B203F03EFB0236F6B2C0
:10E0A800E3E72C4E2C4996F8B4271F48FDF70DF8E6
:10E0B8000120FCF746FD1C48FCF7C6FC274B284905
:10E0C8001F7819483A46FDF700F80220FCF739FD99
:10E0D8001548FCF7B9FC0C2303FB0766214996F8A1
:10E0E800B72796F8B6371048FCF7EFFFFFF7EAF8BE
:10E0F8000320FCF726FD0C48FCF7A6FC96F8BC1795
:10E1080096F8BA2796F8BB37074800911649FCF7E6
:10E11800DCFFFFF7D7F80420FCF713FD0248FCF7F3
:10E1280093FCE6E02C10002049240020E3AE01080F
:10E13800F6AE0108321000201EC40108F4270020A2
:10E14800E8100020FAAE0108E4210020F0210020A8
:10E158000C230020202C0020FEAE0108602800209F
:10E168000AAF01081BAF01082CAF01087B4B1B68E5
:10E178001B0640F1BA80236A616A794A8B421FBF45
:10E18800536292F82830013303F003034FF0010182
:10E198004FF0000018BF82F82830FCF7DEFC94F836
:10E1A8002830704AD05CFCF734FC02200121FCF7CF
:10E1B800D4FC00266C4B9B5D3620C3EBC30393FB5A
:10E1C800F0F0C0B2062828BF06206038C0B2013679
:10E1D800FCF71FFC102EEDD1644B65491B78654890
:10E1E80013F0020F644B1A7814BF59234E23FCF71F
:10E1F8006CFFFFF767F80220FCF7A3FC5D48FCF70B
:10E2080023FC5E495E4B4E680A685A4892FBF3F25B
:10E218005C4996FBF3F3FCF758FFFFF753F803202C
:10E22800FCF78FFC5348584EFCF70EFC574B5849E7
:10E238001A885048FCF749FFFFF730F80420FCF72C
:10E2480080FC4C48FCF700FC524B53491A8849485B
:10E25800FCF73BFFFFF722F804210A20FCF77DFCBE
:10E268004448FCF7F1FB4D49E26A4248FCF72DFFB0
:10E27800FFF714F80520FCF764FC3E48FCF7E4FBC4
:10E288007268B36846493B48FCF71FFFFFF706F87A
:10E2980005210A20FCF761FC3648FCF7D5FB3369F9
:10E2A800F26840493348D21AFCF70FFFFEF7F6FF31
:10E2B8000620FCF746FC2F48FCF7C6FBB2683A4933
:10E2C8002C48FCF702FFFEF7E9FF06210A20FCF7BD
:10E2D80044FC2848FCF7B8FB34492648152207F0C7
:10E2E80019FFFEF7DBFF072016E7F37843F0020378
:10E2F800F370002D2ED12E4B9B79032B9BBF2D4AFB
:10E308009B183F251D7F00211220FCF726FC28467C
:10E31800FCF77FFB13200021FCF71FFC264B1B7822
:10E32800002B264B1B7814BF72202120002B18BF0E
:10E338005220FCF76EFB14200021FCF70EFC94F829
:10E348003050084B585D013505F00305FCF761FBBB
:10E3580084F8305003B0BDE8F08300BFFC270020EC
:10E36800402400203EAF0108BD10002010110020FD
:10E3780043AF01084924002016110020181100207D
:10E388008096980054AF0108A407002012110020BD
:10E3980061AF01087410002069AF010870AF01086F
:10E3A80077AF010880AF010887AF0108C4020020D9
:10E3B800340E002080920108630E0020C80E002051
:10E3C80038B500240B4D6059254403F0D7FB696824
:10E3D80011B10948FCF78EFEA96811B10748FCF78E
:10E3E80089FE0748103403F0C9FBB4F5F07FE9D182
:10E3F80038BD00BFA0920108C0AF0108C6AF010830
:10E40800E8B9010870B50546284607F056FE0646E5
:10E4180058B91A4B1A485A791A4B03EB8203BDE8CC
:10E428007040D3F8DC11FCF765BE28461649324621
:10E4380007F04CFE60B91548154C03F09FFB54F8E3
:10E44800041F19B11348FCF755FEF8E7124805E018
:10E458000024124B53F8241021B91148BDE870402C
:10E4680003F08CBB2846324607F030FE0134002802
:10E47800EFD1024B0B4D5C71C6E700BF202C00208A
:10E48800CCAF0108A0920108D8AF0108DDAF0108A0
:10E498007C940108F0AF0108E8B9010880940108EC
:10E4A80096AD0108ABAA0108F0B585B0044607F09F
:10E4B80004FE082826D1621EE01D1F4912F8013FFC
:10E4C80009681944497801F00301022908BF203B73
:10E4D80082421370F1D1254604F1080715F8016B43
:10E4E8001648314607F0DBFD20B12846314607F0D3
:10E4F800D6FD10B1F8F7A0FD1CE0BD42EED12046D4
:10E50800FEF708FA0E4803F039FB00230D4A1A44B7
:10E5180004A992F88A210A440849595C02F80C1C9B
:10E528000133082BF2D1002307488DF80C3001A9DC
:10E53800FCF7E0FD05B0F0BD9000002006B801082A
:10E54800F4AF0108202C00208CB80108264B274C7A
:10E558001D68206880B5F9F7ADF92846F9F7AAF9DA
:10E56800206841798A0703D441F00201FDF71CFBBA
:10E578001F4B08229A611F4B1A6812F4003F1F466E
:10E588001FBF06236371E37923F001031CBF43F027
:10E598000203E3712068FDF713FB90B1144E0823C2
:10E5A8003385124B1868FDF708FB8046F9F796FB90
:10E5B80008B101F0D9FD28464146FDF704FB0823C0
:10E5C800B3612846FDF7FCFA38B128462668FDF7FE
:10E5D800F4FA01463046FDF7F6FA3B689B03D9D5B5
:10E5E800FFF747FBD6E700BF7C28002074240020F3
:10E5F80000040048FC2700202DE9F041054607F0FB
:10E608005CFD2C4B04469E6888B92B4803F0B6FA8B
:10E618002A4B53F8241041B10123A340334202D0BE
:10E628002748FCF767FD0134F2E7264821E0284631
:10E638002549224607F04AFD58B92448244C03F0DE
:10E648009DFA54F8041F0029EFD01D48FCF752FD2D
:10E65800F7E72B782D2B03BF013504F1FF344FF07A
:10E6680001084FF000080026144B53F8267027B90C
:10E678001848BDE8F04103F081BA284639462246D9
:10E6880007F024FD98B90120B040B8F1000F03D07D
:10E69800FCF786FE104802E0FCF78AFE0F4803F0FC
:10E6A8006DFA39460E48BDE8F041FCF723BD013646
:10E6B800DAE700BF202C0020FAAF0108E89401082F
:10E6C800F0AF0108E8B90108D8AF010804B00108A3
:10E6D800E494010896AD010810B0010819B00108CA
:10E6E8008BB8010810B5084803F048FA074B002416
:10E6F8001C741C64064B1C70FDF7E8FB03F0F0FB70
:10E70800044B1C6010BD00BF21B001087424002018
:10E718002D3400207C28002070B5064600240B4BC1
:10E72800E518AA8816420AD0E1580948FCF7E2FC25
:10E738002846002103F0AFF9064803F01FFA143405
:10E7480040F694439C42EAD170BD00BF4C99010841
:10E758004DB00108E8B9010808B50848FCF7CAFC3B
:10E76800FAF74CF8FCF7F6F818B96420FDF767F9E2
:10E77800F8E70348BDE80840FCF7BCBC57B00108FF
:10E7880064B001082DE9FF410A4806888568448875
:10E79800B0F80480C768F9F73BFFCDF80080029015
:10E7A800019731462A4623460348FCF7A3FC04B0E8
:10E7B800BDE8F081100000206CB00108F0B50478C5
:10E7C8008BB005460CB1002436E04A4B19680E237D
:10E7D80003FB041101F58C70B1F91D51B1F9192130
:10E7E800B1F91B31009591F82051019591F821510B
:10E7F800029590F90700039001F590713E4891F950
:10E808000210049121460134FCF774FC082CDCD179
:10E818006DE02D2B14D1072C1BDC284607F0A4FC37
:10E828000AAB661C03EB440424F8100C15F8013FEE
:10E83800303B092BFAD934462B78002BE9D104E078
:10E84800A3F13002092A09D8E5E7082CBDF81820F9
:10E8580009D00BB0BDE8F040F8F7EEBB202BF8D19B
:10E8680001352646E7E7072AF3D8BDF81A00214BF9
:10E87800A0F2EE2189B240F2DC55A9421B68E8D823
:10E88800BDF81C10A1F2EE24A4B2AC42E1D8BDF848
:10E898001E7004B23EB2A642DBDB0DB2AE42D8DC3B
:10E8A800A542D6DBBDF92440642CD2D1BDF8266040
:10E8B80034B2112CCDDCBDF82050B42DC9D8BDF828
:10E8C8002240B42CC5D812B24FF00E0E0EFB023304
:10E8D800A3F81B116421A3F81901A3F81D7183F88B
:10E8E800205183F8214183F81F1183F822610BB06E
:10E8F800F0BD00BF48100020C9B00108F0B50446BB
:10E908008FB0204607F0D9FBC5B225BBAC48AD4C4B
:10E9180003F034F994F8D61009B9AB4854E049B279
:10E9280094F8D42094F8D530009194F8D710019138
:10E9380094F9D810029194F9D910039194F8DA1047
:10E948000491A24829460135FCF7D4FB102D04F1A7
:10E958000704DFD1E1E720469D49052207F0B6FB11
:10E968000546B8B929469B48702207F062FB9A4BC6
:10E97800196828460E2303FB0013013000220828DB
:10E9880083F8232183F8242183F8252183F826217D
:10E99800F0D113E120469149042207F097FB054680
:10E9A8002046002D4AD1202107F079FB002800F0ED
:10E9B8000581461C304607F080FB2C460746884BED
:10E9C80053F824502DB987480FB0BDE8F040FCF744
:10E9D80091BB30462946FAB207F078FB013400288B
:10E9E800EDD1784A02F170011646002382F8DA3038
:10E9F80082F8D63082F8D53082F8D43007328A428D
:10EA0800F3D1794901EBC40191F8A022934210DABD
:10EA1800D1F8A472C3EBC302B0183A4400F1D40190
:10EA28001768C0F8D4709088888092798A71013309
:10EA3800E7E729466D48FCF75DFB90E06C49072243
:10EA480007F044FB05462046002D4AD1202107F057
:10EA580026FB064607F031FBC4B274BB6548FCF7D9
:10EA680049FB214664480134FCF744FB0E2CF8D1DD
:10EA78005548FCF73FFB002460482146FCF73AFB69
:10EA88000025554A5E4811680E2202FB0412012334
:10EA9800D2F823215B49AB4013425B4B05F10105DA
:10EAA80008BF1946FCF726FB0E2DEAD1464801346B
:10EAB800FCF720FB082CDFD180E03046534907F0F3
:10EAC80057FB2C4600284CD0022C4FD007F04CFBAB
:10EAD80006AB4E4943F82400002007F049FB0134F7
:10EAE800F0E74A4907F044FB002460B1082C38D00D
:10EAF80007F03AFB06AB454943F82400002007F02D
:10EB080037FB0134F1E7082C2BD1069B0F2B28D8B3
:10EB1800DDF81CE0BEF1070F23D8089F0D2F20D881
:10EB2800099E06F16402C82A1BD80A9DFF2D18D831
:10EB38000B98642815D80C99642912D8884210DAE1
:10EB48000D9C032C0DD8324AC3EBC303134483F83E
:10EB580004E05F719E71DD71187259729C722D4CC0
:10EB6800CFE60FB0BDE8F040F8F766BA069B072B72
:10EB780020D807990D291DD80278722A0DD06E2A3F
:10EB880018D1154A12680E2000FB032301228A407F
:10EB9800D3F8231121EA020209E00F4A12680E2075
:10EBA80000FB032301228A40D3F823110A43C3F848
:10EBB800232101E0F8F740FA0D4CA2E60FB0F0BDB2
:10EBC800F1B00108202C0020E8B901081CB10108A7
:10EBD80066AD0108F42C00204810002091AD010812
:10EBE8008094010896AD0108A0920108A5AD01081E
:10EBF800E9B00108CAAF010838B101086DAF0108D2
:10EC08003DB1010863BC01081DBD010841B10108FF
:10EC1800F02C0020ABAA01082DE9F743047805463B
:10EC28008CB9324D95F8AF12B5F8AC2295F8AE32E2
:10EC38002F48009121460134FCF75CFA102C05F1AD
:10EC48000405EFD14EE007F08FFA0F28044636DCB2
:10EC58002846202107F023FA264EE4B2D6F844804D
:10EC6800451CA4000027284607F07EFA5FFA87F9BA
:10EC7800B9F1010F83B208D0B9F1020F0BD0B3F587
:10EC8800B47F24D2726C13530AE0FF2B1FD8736C25
:10EC98002344987004E0FF2B19D8736C2344D87070
:10ECA80028462C2107F0FBF9054608B1013502E09A
:10ECB800B9F1020F0BD10137032FD4D112E00E485E
:10ECC80000210F2203B0BDE8F043F8F732B908EB92
:10ECD80004000021042207F0ACF903B0BDE8F043BA
:10ECE800F8F7AAB903B0BDE8F08300BF202C0020D4
:10ECF80043B101087424002024AD01082DE9F04136
:10ED08002DED048BB3498AB0044607F09BF9B2494C
:10ED1800002820460CBF0126072607F093F9AF49C3
:10ED28000028204608BF022607F08CF9002808BFF3
:10ED38000426F10740F10681A948AA4C02F01EFFFB
:10ED4800002002F021FDA84802F018FFA74802F0B1
:10ED580015FF6279A64BA74803EB82032546D3F833
:10ED6800DC11FCF7C7F9A448FCF7C4F94FF0000818
:10ED7800274695ED058AB5EE408AF1EE10FA04D1E2
:10ED88009E48FCF7B7F9002570E09D48D5ED069A36
:10ED980095ED079AD5ED088A4146FCF7ABF9B5EE33
:10EDA800C08AF1EE10FA02D5202002F0DFFEB0EEA4
:10EDB800480A06A8FCF71EF801469248FCF79AF99B
:10EDC800F5EEC09AF1EE10FA02D5202002F0CEFE40
:10EDD800B0EE690A06A8FCF70DF801468948FCF769
:10EDE80089F9B5EEC09AF1EE10FA02D5202002F0AA
:10EDF800BDFEB0EE490A06A8FBF7FCFF01468148B4
:10EE0800FCF778F9F5EEC08AF1EE10FA02D5202069
:10EE180002F0ACFEB0EE680A06A8FBF7EBFF08F1BB
:10EE2800010801467848FCF765F9B8F10C0F05F1BF
:10EE380010059ED1A4E749B294F8D42094F8D530AF
:10EE4800009194F8D710019194F9D810029194F98F
:10EE5800D910039194F8DA1004916C4829460135C9
:10EE6800FCF748F9102D04F1070403D094F8D610E4
:10EE78000029E0D100254FF00E0808FB05F8002412
:10EE8800634A926C42440123D2F80A20A3401342F9
:10EE980040F0948001340E2CF2D10135082DEAD1CE
:10EEA8005C485D4C02F06AFED7F8088054F8041FED
:10EEB80019B15A48FCF71EF9F8E70D46584B53F8B4
:10EEC800254054B10123AB4013EA080F03D055483D
:10EED8002146FCF70FF90135F0E7534802F04EFEE2
:10EEE80021467B180AAA93F88A3113444F4A8A5C50
:10EEF80003F8102C01310829F3D1002306A94C4846
:10EF08008DF82030FCF7F6F84A4802F037FE4A48F8
:10EF1800F8F752FD494802F031FE4748F8F792F8F1
:10EF2800474802F02BFE4448FFF776FE4548FCF7B9
:10EF3800E1F84020FFF7F0FB434802F01FFE3E488F
:10EF4800F8F7B0FBB20726D5404802F017FE404854
:10EF580002F014FE384802F057FC3E4802F00EFE5C
:10EF68003548F7F7F3FF3C4802F008FE3248F8F757
:10EF7800EBFA3A48FCF7BEF82F48F8F76FF938482B
:10EF880002F0FCFD2C48FFF719FC2E48FCF7B2F8FC
:10EF98008020FFF7C1FB730716D5324802F0EEFD5B
:10EFA800314802F0EBFD244802F008FC2548FCF744
:10EFB800A1F84FF48070FFF7AFFB05E02946224621
:10EFC8002A48FCF797F865E70AB0BDEC048BBDE862
:10EFD800F08100BF57B10108CBB501085EB1010847
:10EFE80064B10108202C002072B1010884B1010825
:10EFF800A092010890B101089BB10108A8B10108CD
:10F00800B5B10108C9AF01088CB80108BDB1010844
:10F0180074240020DCB10108E4940108ECB1010873
:10F02800E8940108FAB1010807B2010806B8010816
:10F0380013B201081CB20108ABAA01082BB20108DF
:10F0480037B20108E8B9010845B2010852B201080F
:10F0580065B2010873B201087DB201088CB20108DB
:10F068009AB20108A6B20108B7B20108C9B20108EC
:10F0780010F80A3C0133DBB20A2B84BF10F8131CCA
:10F08800044A00F80A3C82BF002322F8113000F835
:10F098000A3C70476C2B0020334A136C9068194463
:10F0A800081A40F68C23984270B513469160D060D8
:10F0B80051603BD9127893F945108A4210460BD11A
:10F0C800111F082908D893F84610182901D80131CA
:10F0D80003E083F8442002E0002183F8461093F906
:10F0E80044402149A24219D191F84740B4B10C31AA
:10F0F8000024944206DA1D4D51F8046F25F8146077
:10F108000134F6E70C2805D01849002421F81040EE
:10F118000130F7E7164801780131017083F845207E
:10F12800002201211A7083F8471070BD92F8471029
:10F13800C9B1A0F2EF2440F2DA518C4208D8117814
:10F148000B2905D80B1D0131117042F8230070BD41
:10F15800002283F84720074B03F13002002143F8CF
:10F16800041F9342FAD170BD300100206C2B00209F
:10F17800340600203C010020024A136C0133194474
:10F188001164704730010020024B53F820301B688F
:10F1980019607047601F0020064B53F820301A682A
:10F1A8001B89A1F57A7159434FF47A7391FBF3F1F6
:10F1B80011607047601F0020054B98420CBF054A3C
:10F1C800054A138801339BB213800020704700BFA3
:10F1D80000540040081000200A10002038B510F82C
:10F1E8000E2C50F8043C04465AB9012200F80E2CA3
:10F1F80020F80C1C997A18680222BDE83840F9F703
:10F20800A3BE30F80C2C20F80A1C891A89B220F801
:10F21800081C084A10F80F0C002522F8101004F8F2
:10F228000E5C1868997A2A46F9F78EFE04F8065C8F
:10F2380038BD00BF6C2B0020044B53F820301BB1A5
:10F2480007289CBF1B681960704700BF5802002040
:10F25800074A13689B060AD5064B00211970064910
:10F2680008684FF6FE7303400B6020235360704715
:10F2780000000240293400201C0002402DE9F0471C
:10F28800664D2B6866490A78581C02F0FF068E46C0
:10F298000AB10346F6E72B60687BAB6895F80C80EB
:10F2A800AA7B374639B2202900F09B80DFF880C15D
:10F2B8000CEB81033CF82110DC789B78C3F1FF0349
:10F2C8009BB2002B65D0C3F1FF0363434FF03C0CA6
:10F2D8001B12B1FBFCF9B9F1050F5DD8DFE809F0A5
:10F2E800030B1A293A4AE01ADAB24143B1FBFCF09F
:10F2F8001044C0B251E0B1FBFCF00CFB101189B214
:10F30800DAB2C1F13C01E31A4B432046B3FBFCFCE3
:10F3180094442CE0B1FBFCF00CFB10115FFA83F86D
:10F32800E21A89B24A43B2FBFCF24244D2B2204606
:10F3380032E0B1FBFCF90CFB191189B25FFA83F8D2
:10F34800E01AC1F13C014843B0FBFCF04044C0B2B4
:10F35800224621E0B1FBFCF80CFB1811D8B289B2A7
:10F36800E31A01FB03F2B2FBFCFC224684445FFA79
:10F378008CF412E0B1FBFCF80CFB181189B2D8B27E
:10F38800C1F13C01E31A4B43B3FBFCF20244D2B295
:10F3980003E02246204600E044464FEA042C4CEAAB
:10F3A800004C4CEA020C172306F117014FF0010834
:10F3B80008FA03F8C91A18EA0C0F89B2DFF8748042
:10F3C80014BF4FF011094FF0090913F1FF3308F882
:10F3D8000190E9D218360137B6B2BFB2114BA04638
:10F3E80060E7AA73AB60104AE98001238EF8003009
:10F3F8000E4985F80C8040F22A336873AE8053605A
:10F4080000234B620B889BB243F001030B80136807
:10F4180043F001031360BDE8F08700BFC02400205B
:10F4280029340020CC2400201C000240002C01407C
:10F43800AA0D0020D902002073B506460D46002407
:10F4480001232A88A34013421AD0AA78009302F015
:10F4580003038DF80430EB78022B03D0032B0CBF89
:10F46800032301238DF805303046C2F301136946A2
:10F47800C2F381028DF806308DF80720FDF7DEFD16
:10F488000134102CDCD102B070BD2DE9F04F734E61
:10F49800F57B07460C4687B011469A4600686B1CF8
:10F4A800914622464FF0020BF37300F083FC3B8930
:10F4B8007868ADF8043001A98DF806B08DF807B06A
:10F4C800FFF7BAFF0023ADF80A30ADF81230ADF8F7
:10F4D800163070230193BA7A3C68CDF80CA001234A
:10F4E80006F110082D01ADF808304FF48073A844D8
:10F4F800ADF810B0ADF814300C2A7ED8DFE802F071
:10F50800077D7D7D0F7D7D7D387D7D7D5E0020467C
:10F5180001A9FDF7E3FBA36943F0080326E0236A8A
:10F528004F4823F010032362236A6168A26922F01E
:10F53800807222F4E642844242F4E04206D000F5AA
:10F548000060844202D043F0300307E023F0E00378
:10F5580021F4406143F0300341F480616160A261AD
:10F56800C4F838A02362A36943F40063A36144E0AC
:10F57800236A3B4823F480732362226A6168E36943
:10F58800844223F0730343F0700306D000F5006053
:10F59800844202D042F4407207E022F4606221F40F
:10F5A800405142F4407241F480516160E361C4F813
:10F5B8003CA02262E36943F008031DE0236A28485F
:10F5C80023F480532362226A6168E369844223F446
:10F5D800E64343F4E04342F4405203D000F50060B0
:10F5E800844201D141F480416160E361C4F840A0E4
:10F5F8002262E36943F40063E3613A7B3B681AB132
:10F608005A6C42F400425A641A8892B242F00102DB
:10F618001A80BA7A0C2A18D8DFE802F007171717E9
:10F628000B1717170F1717171300721903F1340167
:10F638000AE0721903F1380106E0721903F13C017E
:10F6480002E0721903F14001116135444046A5F802
:10F6580018906B6107B0BDE8F08F00BFC024002090
:10F66800002C0140F8B53A4E3A4C4000C7B24FF46E
:10F6780020453068C4F8D050D0F818E01EF4004F88
:10F6880005D0AE46013DBEF1000FF5D116E0D0F829
:10F6980004E0314D0EEA050545F490353D434560DB
:10F6A8004FF42045C4F8D050D0F818E01EF0020FEF
:10F6B8002DD1AE46013DBEF1000FF5D1C4F8D050B2
:10F6C8001FE02946013D0029F8D081694906F8D58F
:10F6D800C4F8D05020494568294041F0007141F4F0
:10F6E800105141EA0241394341604FF42041A2B12F
:10F6F800306885696D071ED411F1FF31F9D2C4F85D
:10F70800D010FFF759FD003018BF0120F8BD4FF4A5
:10F7180020458162C4F8D050D7E73068C4F8D010CB
:10F728000B46826992060CD41A46013B002AF8D18E
:10F73800C4F8D030E5E7416A03F8011B013AD2B2B8
:10F74800D3E7C4F8D0302023C3610120F8BD00BF3F
:10F7580004100020C0240020009800FC400070B570
:10F76800C5B23248324B00684FF42044C3F8D04049
:10F778008669360404D52646013C002EF8D113E0EC
:10F7880046682C4C344044F0807444F490342C4344
:10F7980044604FF42044C3F8D0408669B60729D4A2
:10F7A8002646013C002EF8D1C3F8D0401CE0214683
:10F7B800013C0029F8D081690E06F8D544681D4936
:10F7C800214041F0007141F48031294341604FF4F8
:10F7D8002041C3F8D0108469A40711D40C4601391C
:10F7E800002CF8D1C3F8D010FFF7E6FC003018BFA2
:10F7F800012070BD4FF420448162C3F8D040DAE79D
:10F8080082624FF42042C3F8D0208169890606D469
:10F818001146013A0029F8D1C3F8D020E4E7C3F82B
:10F82800D0202023C361012070BD00BF0410002038
:10F83800C0240020009800FC6C4B6D4A2DE9F04F65
:10F848005E8914684FEA062AB4EB0A0A9C884FEAD4
:10F8580004481C894FF000054FF0000B65EB0B0BBB
:10F86800A4FB0A6704FB0B77F40944EA476418EB26
:10F8780004065C884FF000094FEAE7154FEAC438E0
:10F88800DC8849EB050787B0CDE90467A4FB0A6764
:10F8980004FB0B77340A44EA076418EB04064FEAC2
:10F8A80027259C894FF0000949EB0507CDE900673A
:10F8B800AAFB046704FB0B77F40D44EA472414F50C
:10F8C800FA664FEAE75545F10007B6F5FA6F77F1A2
:10F8D8000003CDE90267964667DAA4FB046704FBD8
:10F8E80005F34FF0050C07EB4307DDE90489A6FB98
:10F8F8000C230CFB07335F104FEA3206B8EB0608FF
:10F908004FEA920669EB070946EA83769F10DDE91C
:10F918000023921B63EB0703DDE90267CDE90023AF
:10F92800344A4FF0FF33964277EB0303CDE904895D
:10F9380028DA40F6AC52A4184FF000035D4104FBEE
:10F9480005F3A4FB044505EB43056FF00602664288
:10F9580002FB0566A4FB0223334418EB020649EBBD
:10F968000307CDE904670B26A4FB062306FB053332
:10F97800DDE900455B104FEA3202A41A65EB030586
:10F98800CDE900450AFB0BF3DDE90245AAFB0AAB0A
:10F998000BEB430B4FEADA7242EA4B02A41A4FEA26
:10F9A800EB7365EB0305CDE90245DEF80440009BE7
:10F9B800019DA4FB032304FB05334FEA52584FEA89
:10F9C800635948EAC328DDE90423B8EB020269EB6E
:10F9D80003039946D30B43EA494300B1036009B1D5
:10F9E800029B0B6007B0BDE8F08F00BF86020020C5
:10F9F8009425002024FAFFFF772048210122FFF7F1
:10FA0800ADBE772058210122FFF7A8BE07B5002117
:10FA180001AB03227720FFF725FE9DF805309DF8FE
:10FA280004001B0243EA00439DF80600184303B094
:10FA38005DF804FB08B5FFF7E9FF014B586008BD06
:10FA48009425002008B5FFF7E1FF014B186008BDB9
:10FA58009425002013B506220446432168206B46EE
:10FA6800FFF700FEA0B19DF800209DF8013043EAA1
:10FA7800022323809DF802209DF8033043EA0223E5
:10FA880063809DF804209DF8053043EA0223A38093
:10FA980002B010BD13B5062204463B2168206B4610
:10FAA800FFF7E0FDA0B19DF800209DF8013043EA82
:10FAB800022323809DF802209DF8033043EA0223A5
:10FAC80063809DF804209DF8053043EA0223A38053
:10FAD80002B010BD13B501220DF107033A21044607
:10FAE8006820FFF7BFFD0520FBF79EFF9DF8073054
:10FAF80003B10123237002B010BD084B1B681869BD
:10FB0800074B20F01F0200F01F01D25801238B4041
:10FB18001A4201D0FCF798BF704700BF800200204E
:10FB280014040140F0B52B4D2B7A85B0002B4ED133
:10FB3800294C2368002B4AD01A68284E12B17169E3
:10FB48000A4372619A88ADF80020022298688DF8FD
:10FB58000320694600228DF80220FFF76DFCB36987
:10FB68001D4F43F00103B3612368187B197DFDF72E
:10FB78001BF82268936894881B8A1C4002D00123D2
:10FB88002B7224E01648FBF7FFFF3B681869FCF767
:10FB98005BFF3B688DF80C401B69029308230DEB53
:10FBA800030001268DF80D308DF80E6001F032FB50
:10FBB8003B688DF806405B7D8DF8043001A803236F
:10FBC8008DF805308DF8076001F006FBD7E705B022
:10FBD800F0BD00BF942500208002002000100240E4
:10FBE80003FB000808B5FFF79DFF6B218022682002
:10FBF800FFF7B4FD6420FBF722FF6B210322682086
:10FC0800FFF7ACFD0F20FBF71AFF124B19211A78EA
:10FC18006820FFF7A3FD0F20FBF711FF0E4B1A21F9
:10FC28001A786820FFF79AFD1B2118226820FFF731
:10FC380095FD1C2110226820FFF790FD3721022234
:10FC48006820FFF78BFD682038210122BDE80840B5
:10FC5800FFF784BDB40200200000002008B5FFF7BC
:10FC680061FF074B1B7813B1012B03D008BD4FF47C
:10FC7800006201E04FF48052024B1A8008BD00BFB9
:10FC880084020020200000202DE9F0410369C768A4
:10FC980005460E461F40002F35D0B7FA87F24FF0C1
:10FCA8000043D340DB432B611F40A2F11B03042B0D
:10FCB800F1D8DFE803F0221F1C190300746A24B18D
:10FCC800013C0023A4B2736201E0EC6AA4B2D6F846
:10FCD8002080B8F1000FDED0D8F800304046214629
:10FCE8009847D8F80480F4E73068696B07E07068D3
:10FCF800A96B04E0B068E96B01E0F068296C03685F
:10FD080089B29847C7E7BDE8F08107B52320FBF71C
:10FD180096FE6820752101220DF10703FFF7A2FC6A
:10FD280028B19DF80700A0F168035842584103B074
:10FD38005DF804FB01480249A6E700BF00480140FE
:10FD480084200020014802499EE700BF004001408E
:10FD5800342000200148024996E700BF000800400F
:10FD68000C200020014802498EE700BF0004004033
:10FD7800E41F00204FF08040004985E7BC1F0020A9
:10FD880010B5054C05482146FFF77EFF04F1C80170
:10FD98000348BDE8104077E7941F0020002C01407D
:10FDA80000440140014802496EE700BF002C0140B1
:10FDB800941F0020224B10B5224C5A43224BB3FB10
:10FDC800F2F203880139013AA04289B292B29BB299
:10FDD8000ED004F50064A0420AD0B0F1804F07D0DD
:10FDE800A4F59834A04203D004F58064A04202D15F
:10FDF80023F070039BB2154CA04206D004F5806432
:10FE0800A0421CBF23F440739BB203800D4BC16218
:10FE1800984202850FD003F5006398420BD003F592
:10FE28004063984207D003F58063984203D003F5F6
:10FE38008063984201D1002303860123436110BDEA
:10FE480040420F00002C014000A24A04001000406C
:10FE580073B505460068FFF7ADFF2A6813889BB2A3
:10FE680043F001031380EB7A8DF804300124002657
:10FE780001A88DF805408DF806608DF8074001F05F
:10FE8800ABF9EB7A1B2B0BD1192301A88DF80430A1
:10FE98008DF805408DF806608DF8074001F09CF953
:10FEA80002B070BD134B800A984220D00AD84A3B52
:10FEB800984212D00133984211D0B0F5801F14D166
:10FEC800012070470C4B98420BD0013398420AD05E
:10FED800023B984209D10420704702207047032052
:10FEE80070470520704706207047FE2070470020A5
:10FEF800704700BF4B00100051001000F8B50468AF
:10FF0800064620460F461546FFF7CCFF06284BD875
:10FF1800B27A910847B902238B40D4F80CE0DB434E
:10FF28009BB203EA0E03E3600A23204A03FB001393
:10FF380042F82370043342F8235015463FB1B17A92
:10FF4800E268890802238B409BB21343E3602822AE
:10FF580002FB00522032EFF31286502383F31288FB
:10FF680003B203EB8303DB0003F10C011C332944C8
:10FF78002B4451F8047F17B117600A68043299427C
:10FF8800F7D100231360F3B283F31188282303FB0E
:10FF98000050036A1BB1E36843F0010303E0E26821
:10FFA8004FF6FE731340E360F8BD00BF941F0020B6
:10FFB8000148F8F74BBD00BFA02500200148F8F71D
:10FFC80045BD00BFF42500200148F8F73FBD00BF3C
:10FFD8004826002010B54B88DC0641BF2F4B14790A
:10FFE8001B6853F8244044BF2D4B43F820404B88EE
:08FFF8009B0641BF294B54791F
:020000040801F1
:100000001B6853F8244044BF274B43F820404B88DB
:100010001C070ED5254B0C781B78B3EB141FA1BF22
:10002000204BD4781B6853F82440A4BF1E4B43F8E0
:1000300020404B889B070ED51D4B0C781B78B3EBEB
:10004000141FDFBF174B54781B6853F82440DCBFE4
:10005000154B43F820404B88DC070FD5154C0B7827
:10006000247803F00F03A342DFBF0E4B14781B6804
:1000700053F82440DCBF0C4B43F820404B885B070F
:100080000FD50B780C49097803F00F038B42A1BF01
:10009000044B92781B6853F82220A4BF024B43F80C
:1000A000202010BDB8240020AA0D00203F240020ED
:1000B0003D2400203C2400203E240020254A2648E0
:1000C00026490023F0B5156803700B701C461A46CC
:1000D0002E1976884EB92F5D3FB9037000230A7040
:1000E0004B7007781C461A460CE0360548BF0132B3
:1000F00004F1040403F1010348BFD2B2802CDBB247
:10010000E6D1EAE7E0B2B8420CD215F824000609BD
:100110009E4200F00F00A8BF731C9042A8BF421C73
:100120000134EFE78A704B70C2F3470102F001021D
:100130000A444C1E0A490B480A70C3F3470203F0F5
:100140000103134404700849501E084A08701370D4
:10015000F0BD00BFE0110020342400209C260020C8
:100160003E2400203C2400203F2400203D24002089
:100170002DE9F04FC24BDA682DED028B1A61C14AAE
:100180001168D960C0490B6843F020030B60BF4B76
:100190001978012990460CBF002201221A70BC4B2D
:1001A0001A78910789B040F13D83BA49097804294A
:1001B00040F23883B849097801F0040101F0FF00EA
:1001C00011B922F001021A701B78DB0702D408B1C2
:1001D000F8F770F9B149CA78531C052293FBF2F283
:1001E00002EB82029A1AAE4BCA701B7803939200FC
:1001F0000023AC4CDFF8CCC2DFF8D8925CF82310B7
:1002000091FBF9F504F1080004F1100640F82350C1
:10021000A54844F8231000FB051142F2107091FB31
:10022000F0F080B226F813004FF0140E04F114061B
:1002300004F13C0A0EFB036E5AF823605EF802706C
:100240004EF80210F61B314444344AF823100526B8
:1002500091FBF6F109FB051144F82310039C012CD6
:100260004FEA830BE24605D10238B0F5797F98BF9B
:100270004BF80C100BB90123BBE7884CD8F80030C1
:10028000226D9FED8A7A8A4E8A4D9B1A07EE903A2C
:10029000F8EE677AD8F800302365C7EE877A7C4B92
:1002A0001B78B7EE008AF4EEC87AF1EE10FA58BF68
:1002B000F0EE487A13F00103C4ED157A12D005AAC6
:1002C00000927D4B06AA01920CCB9AE80300F7F747
:1002D000EFFF6421059A069BB2FBF1F293FBF1F369
:1002E000328000E033802B8094F858306B48002B2C
:1002F0003BD0D0ED157AC26DDAF80030C8EE276A2F
:100300009B1A026E022507EE103AB8EEC77ADAF8A9
:10031000043027EE267A9B1AFDEEC77AB0F96620E4
:1003200017EE901A07EE903A644BB8EEE77AD3EDE9
:10033000007A67EE277A67EEA67AFDEEE77A17EE87
:10034000903A02FA83F3B0F9642093FBF5F302FAD2
:1003500081F29BB292FBF5F292B2A0F86A30A0F85B
:100360006820A0F86630A0F86420012384F8583093
:10037000534BDAF804101B88DAF80000474D514E51
:10038000216603F03003E065002B00F04B8205F19D
:100390007403009305F178030193EA6E2B6FF7F76E
:1003A00087FF72682B6F9B1A07EE903A434B3268B7
:1003B00093ED007AEB6EF8EEE77A9B1AEB67384B19
:1003C00067EE877A1B78FDEEE77A012BC5ED207A80
:1003D00003D0022B00F0DF8024E2D5ED287A3A4BDF
:1003E000D5ED215A95ED255A95ED156A95ED264ADC
:1003F000D5ED274A35491D68B1EE677ABDEEC77A5B
:10040000FDEEE77A17EE10EA17EE90CA0020304AA8
:1004100091ED007A52F8207007EE907AF8EEE77AC4
:10042000A2F1140367EEA57A33F81060FDEEE77AC7
:10043000283217EE903A9B1B9BB222F810301BB269
:1004400007EE903AF8EEE77A3B4467EE857A44008F
:10045000FDEEE77ACDED037A07EE903AF8EEE77A13
:10046000BDF80C8067EE847AA7EE867AFDEEC77A37
:1004700017EE902A724531DB6245A8BF62462EE036
:10048000A4070020202800200C1100207610002056
:1004900010110020161100202A3400209C26002074
:1004A000340F0020A0260020806967FF00007A44F6
:1004B0008A1100208C110020781000207800002084
:1004C000D411002018110020380F0020680F0020E0
:1004D0001827002080969800DB0FC940724607EE6F
:1004E000902AF8EEE77A5FED046AC1ED007AFDEE3E
:1004F000E77A313617EE903A43449AB2AB78D1EDB1
:10050000027A07EE103AB8EE477A4B684F6027EE52
:10051000267AFB1A88EE077AB6B2622E06EE903A79
:10052000F8EEE66A37EE067AC6EE866A86EE077A57
:1005300076EEE76AE7EE267AC1ED047AC1ED027A3B
:100540000FD964EEA77ABA4EFDEEE77A17EE903A2D
:10055000B3F5FA6FA8BF4FF4FA63B342B8BF33469E
:1005600000E0002313441BB240F6B8329342A8BF08
:100570001346B04A9342B8BF1346AF4AA352AF4A9C
:10058000142303FB002351F8142B1A60002840F0B9
:10059000498101203BE7AA4BD5F874801F68D4F845
:1005A00078903E89DFEDA78A4FEA58039E4228BF24
:1005B0001E46B5F8A8301AB29642C3BFD5ED157ADB
:1005C0009FEDA17A67EE877AB6B2C1BFFDEEE77AFA
:1005D00017EE906AF618B6B2C8BFA5F8A860D4F8AE
:1005E000AC50C5EB09052846F7F7A6FE0028D8BF92
:1005F000404241F293129042CCBF0020012088B3C8
:1006000007EE905AB8EEE70A20EE280AFAF7A5FDA1
:1006100007EE908AF8EE677A40F6B83320EE270AA4
:10062000FDEEC07ACDED037ABDF80C20A4F8B02021
:1006300012B29A42A8BF1A467E4B9A42ACBF09EB4F
:1006400002034B4448F6A042934203DDA3F50C435A
:10065000A03B04E0002BBCBF03F50C43A033C4F85F
:10066000B43001E0C4F8B490D4F8B450C5F50C53DC
:10067000283307EE903AF8EEE77A67EEA88AB0EEF4
:10068000680AFAF7CDFD8DED070AB0EE680AFAF7B1
:1006900064FDD4ED317AD4ED2E4AD4ED155A94EDA3
:1006A0002F4A94ED305A65498DED060AB1EE677A0E
:1006B000BDEEC77AFDEEE77A0DF1180E17EE10AA1F
:1006C00017EE90BA0020614AFEEC016A32F9103050
:1006D000DFF88C9107EE903A07EE106AF8EEE77AB1
:1006E000B8EEC77A3C32D6EE877A4FEA400CFDEE80
:1006F000E77ACDED037ABDF90C30B3F57A7FA8BF68
:100700004FF47A734B45B8BF4B461FFA83F922F872
:1007100010900FFA89F207EE902AF8EEE77A27EEAA
:10072000A47ABDEEC77A8DED037A27EE847AD1EDF7
:10073000007ABDF80C90E7EE257AFDEEE77A17EE29
:10074000902A524503DB5A45A8BF5A4600E052465C
:1007500007EE902AF8EEE77A9FED3D6AC1ED007A48
:10076000BA7891ED027A06EE902AF8EE666A4A6847
:100770004B6066EE866A9A1AC8EE266A143106EE57
:10078000102AB8EEC66A76EEA56A86EE256AC5EE30
:10079000A66A36EE476AA6EE867A01ED017A01ED89
:1007A000037A25EE077ABDEEC77A17EE103ABDEE52
:1007B000E77A4B4417EE102A13441BB240F6B832C6
:1007C0009342A8BF13461B4A9342B8BF13461A4A26
:1007D0002CF802301F4A142303FB0023C3ED007AD8
:1007E00008B901206FE73B7923B1642395FBF3F54A
:1007F000194B1D803B8898450DD9D4F8AC30A06FBB
:10080000C01AF7F799FD80EAE072A2EBE07242F2BB
:1008100010739A4206DD114B01221A700E4BB4F888
:10082000C8201A8009B0BDEC028BBDE8F08F00BF74
:1008300030F8FFFF48F4FFFFBC0F0020900F0020AE
:10084000380F0020D30237390000C84204270020A7
:10085000DB0FC940680F0020300F0020340F00204C
:1008600018FCFFFF0846F5F777BE0F4B1A78692A88
:1008700016D15A88B2F5FC6F12D11A79BE2A0FD15F
:1008800093F8DD27EF2A4FF000000BD113F8012B6E
:100890005040064A9342F9D1B0FA80F040097047BF
:1008A00000207047704700BF00F80308E0FF03080E
:1008B0002DE9F04FEB4C85B000214FF4FC6220464F
:1008C00005F0BBFBE84B04F53B721A60E74B0025D3
:1008D0001D70E74B04F2B6721A6069232370022080
:1008E00003236371FAF768FD4FF48070FAF764FD33
:1008F0004FF416732022A4F8663184F86A21FA2393
:100900006E22A4F8683184F87C21BC230A22A4F862
:10091000643184F87D214FF4FA732B22A4F86E31F0
:1009200084F87F210123212284F8623184F87E310A
:1009300084F8802184F886312322002384F88121E1
:10094000C4F820324FF4C872C4F824320523A4F846
:10095000822184F8B457A4F87251A4F87051A4F815
:10096000745184F8585184F8595184F85A51A4F8B4
:100970005C51A4F85E51A4F8605184F8635184F886
:100980006B5184F86C51A4F88451A4F8885184F810
:100990001D5284F81C5284F8285284F82B3240F2FD
:1009A000DC53A4F8983140F24C43A4F89A3140F259
:1009B0006C73A4F89C3140F27533A4F89E3140F674
:1009C0004303A4F8A03184F8295284F82A5284F809
:1009D000925184F893512A462346991802320025F1
:1009E0004FF01E09242A9F4C81F8A25181F8A3914F
:1009F000F3D14FF4FA6340F27E4040F27E57DFF8C5
:100A000068B2A4F8C831A4F8CC31A4F8D031A4F865
:100A1000D431A4F84401052340F23A70A4F84C7193
:100A200040F2EA5701264FF47A78C82219214FF094
:100A3000320A84F8DE31A4F846014FF4C87340F25C
:100A4000DC50A4F84E7140F2B457A4F8E2210392AE
:100A500084F8DF110191A4F8E631A4F84A0102906C
:100A600084F8959184F8DD6184F8E06184F8E161AF
:100A700084F8E46184F8EA61A4F8507184F8945130
:100A800084F89651A4F8C681A4F8CA81A4F8CE814E
:100A9000A4F8D28184F8D65184F8DC5184F8E85166
:100AA000A4F84881A4F852A1A4F8543184F8ED6167
:100AB000A4F856A184F8EB5184F8EC5184F8EE5177
:100AC000FBF7EEFEDBF8003026744FF0170E83F8CC
:100AD00015E083F816E04FF0550EE673A573A58177
:100AE00083F803E04FF00F0E83F805E00199D97108
:100AF0004FF0220E83F806E021214FF00E0E83F80E
:100B00000B9083F80C9083F810E059744FF0350E79
:100B100053214FF0640928274FF02D0C83F81AE079
:100B2000D9764FF05A0E0A2183F81C904FF07809BD
:100B300083F80DC083F808E0997483F80A901D705B
:100B40005F709F70DD7583F804A09D731D76DD7363
:100B50005D765F7283F814C04FF4FA7CA3F84EC040
:100B6000DFF820C1C3F838C0C3F83CC0DFF818C1B3
:100B7000C3F828C04FF07E5CC3F834C0F7EE087AA3
:100B8000DFF80891DFF808C1C3ED087AC3F82C90AC
:100B9000C3ED097AC3F83090C3F848C0F1EE047A87
:100BA00002989E774FF04B0C4FF0000983F85010DD
:100BB00083F8525083F85170C3F84090C3ED117A16
:100BC00083F84CC084F8B6E7A4F8C0074FF0410E94
:100BD000042084F8B7E784F8B8A784F8B95784F8F4
:100BE000BD5784F8BE5784F8BA5784F8BB5784F8C9
:100BF000BC5783F85C0015200191A3F85850A3F866
:100C00005A50A3F85650C3ED187A83F86800194873
:100C1000D866194818671948586783F878601848E3
:100C200083F8647083F86570FBF778FEDBF80030BA
:100C30000199039A83F814614FF4487083F81151B5
:100C400083F8125183F8137183F81851A3F8160131
:100C50005E4684F8D81184F8D921A4F8DA811946BF
:100C600018E000BF202C0020481000206028002041
:100C7000701000209A99193FF6287C3F3D0A773F73
:100C8000FDB701088FC2F53C00002040CDCCCC3E22
:100C9000000040400E2202FB05326FF0170082F880
:100CA0001901032082F81A016FF02F0082F81B014E
:100CB000072082F81C016FF0230082F81D01052037
:100CC00082F81E0101355A2081F8200181F82101A6
:100CD0006422FF20082D81F81F2181F8220101F1F3
:100CE0000E01D7D1002183F88911C821A3F88A11F8
:100CF000142183F88C11A3F890211E214FF49672D1
:100D000083F88D11A3F8922101212822A3F89421C0
:100D100083F88E112E4B03F1C0021F46C3F81490C6
:100D200010339342FAD12B480021402205F085F977
:100D30000023294D264C5959FA1804330868C2F883
:100D4000AC02382BF5D104F50B700021802205F0A0
:100D500074F905F13801702204F50B7005F062F9A1
:100D6000FFF7ACF94FF40020FAF726FB36680125AF
:100D7000314604F284404FF4CC7284F8DC5784F896
:100D8000DA5784F8DB5705F04DF904F21C60314660
:100D90004FF4CC7205F046F9104B1B681A68C4F882
:100DA000C2275A68C4F8C6279A68C4F8CA271A68BE
:100DB000C4F8CE275A68C4F8D2279A68C4F8D62750
:100DC000022384F8D85484F8703605B0BDE8F08F5B
:100DD000202C0020CC2E0020D0960108701000207E
:100DE0001549D1F8883043F47003C1F88830134BAB
:100DF0001A6842F001021A605868114A02405A60AB
:100E00001A6822F0847222F480321A601A6822F47E
:100E100080221A605A6822F4FE025A60DA6A22F0CE
:100E20000F02DA62186B074A02401A6300229A60C6
:100E30004FF000638B60704700ED00E0001002404F
:100E40000CC07FF8CCFC00FF074B93F8DC37012B7C
:100E500008D1064A064BD0681B68834234BF002085
:100E60000120704700207047202C00201000002037
:100E70002806002038B5094B93F8DC5765B9084CB3
:100E80002068F6F726FD074B25601B78022B03D15F
:100E9000BDE83840FBF7C3BC38BD00BF202C0020A4
:100EA000B0280020AC280020064B93F8DC371BB19B
:100EB000012B05D1F7F784BC034B1868FAF77BBE0A
:100EC00000207047202C0020B0280020F8B5011F1A
:100ED00006460023083051F8042F02F120043F2C6D
:100EE0003BD802F108040F2C06D80232032A04D999
:100EF000002B08BF012300E002238142EBD1012B2C
:100F000030680ED0022B1AD0736803F003039B00E5
:100F100000F0030043EA0010B36803F00303184332
:100F200017E000F00F0040F04000F5F715FBB06847
:100F3000736800F00F0040EA0310C0B209E000F04F
:100F40003F0040F08000F5F707FB3079F5F704FB30
:100F5000307ABDE8F840F5F7FFBA06F10C073446E1
:100F60003A46002552F8043D03F18001FF294FEA7B
:100F7000850510D903F50041B1F5803F02D245F057
:100F8000010508E003F50003B3F1807F34BF45F0AD
:100F9000020545F00305B242E4D165F03F00C0B25E
:100FA000F5F7DAFA05F00303022B207807D0032BBC
:100FB0000CD0012B13D1F5F7CFFA60780FE0F5F7DD
:100FC000CBFA6078F5F7C8FAA07808E0F5F7C4FA2C
:100FD0006078F5F7C1FAA078F5F7BEFAE078043446
:100FE000F5F7BAFABC424FEAA505DBD1F8BD10B55A
:100FF0000446C0B2F5F7B0FAC4F30720BDE81040CC
:10100000F5F7AABA10B504467F2C06D964F07F0024
:10101000C0B2F5F7A1FAE409F6E7E0B2BDE8104086
:10102000F5F79ABA430083EAE070EBE72DE9F04761
:10103000304B93F8DC37012B86B0074601D00446CD
:101040004AE005F03EF803A9054606466846F7F76C
:10105000C7FA039B049A029713442B443F2B059530
:1010600019D90023684603A90322F7F7E5FA039B81
:101070003BB9049B2BB9204A13705370059BABB34B
:1010800001E0F7F795FA039B049A059E1344334455
:101090007F2B2BD8029FDFF86090CA4639461AF89A
:1010A000024BC4F18008B04528BFB0460AEB0400EB
:1010B0004444E4B2424604F0B5FF802C89F8004075
:1010C00014D1C8EB0606504607EB0801324604F07F
:1010D000A9FF89F8006009E0254614F8011B21B139
:1010E000064B1868FAF773FDF6E7ED1B284606B0C5
:1010F000BDE8F087202C002068270020B0280020C1
:101100000FB407B504AB064953F8042B0193002034
:10111000F9F7F2FE03B05DF804EB04B0704700BFCE
:101120006508010840F2E9330F4A1289920704D496
:10113000013B9BB2002BF7D10BE00C4A40F2E933A4
:10114000107009490989C9070AD4013B9BB2002BD9
:10115000F7D1074A138801339BB21380FF207047F1
:101160001078C0B2704700BF003800400C38004013
:10117000EC27002030B5174B9B894FF47A733AB3B4
:1011800011B10D78013107E0FF2505E0013B9BB26D
:101190004FF6FF74A3420FD00E4C2489A407F5D557
:1011A0000D4C25700B4D2D89ED070BD4013B9BB2E7
:1011B0004FF6FF75AB42F5D1084A138801339BB255
:1011C000138005E0247808B104700130013AD6E7B5
:1011D000012030BD003800400C380040EC270020D2
:1011E0000C4B0D49DA684378D243C2F30222C2F1B4
:1011F0000402934002781B010A44DBB282F80033F8
:1012000003780122580903F01F0302FA03F341F89F
:101210002030704700ED00E000E100E0036823F0BB
:101220001F0202F1804202F5823270B503F01F0105
:101230001468012303FA01F124EA01011160026834
:101240002A4C22F01F0502F01F02295903FA02F26C
:1012500021EA02022A510279016802F1804221F05A
:101260001F0402F5823201F01F01155903FA01F142
:101270002943115102681E4D22F01F0402F01F0283
:10128000615903FA02F221EA020262510268194C22
:1012900022F01F0602F01F02315903FA02F221EA7E
:1012A0000202417932511029026812D122F01F0145
:1012B00002F01F024E5903FA02F232434A51026809
:1012C00022F01F0102F01F020859934003430B5103
:1012D00070BD01F1804122F01F0001F5823102F062
:1012E0001F020C58934023430B5070BD040401406F
:1012F000080401400C040140F0B5BE4CA3782DED6C
:10130000028B013B012B85B000F26F81E5788542AD
:1013100040F06B812379022B00F06781B64B5B5D57
:101320006371A3796D00F2EE048A1BB16319B3F9FE
:10133000083009E06319D4ED037AB3F90830F1EE0F
:10134000677AC4ED037A5B4208EE103A2369A94E2E
:10135000B8EEC88A1A0388EE288A35D5D6ED037A06
:10136000FDEEE77A28EE280A17EE903AD6ED057AD8
:101370008DF80A30FDEEE77A17EE903A8DF80B30D3
:1013800005F0B0F8FCEEC07A96ED060A17EE903A3A
:1013900020EE280AADF8083005F0A4F8FCEEC07A7B
:1013A00096ED070A17EE903A20EE280AADF80C30B9
:1013B00005F098F8FCEEC07A0C2017EE903A02A9DE
:1013C000ADF80E30F5F7B8F9D4ED077A894BF5EEA4
:1013D000407AF1EE10FA60D1D3ED067AB4EEE78AE6
:1013E000F1EE10FA04DDDA6883ED068A5A61E8E06E
:1013F000F5EEC07AF1EE10FA40F3E38093F8202086
:1014000042B1022A00F2DD805A6B83ED078AFA327C
:101410009A63D6E0D3ED037A38EE678AF7EE007A66
:10142000B4EEE78AF1EE10FAACBF01210021D3ED52
:101430000A7A69B19FED717A27EE877ADFED707ACB
:10144000B4EEE77AF1EE10FA58BFF0EE477A03E017
:101450009FED6C7A67EE877AC3ED0A7A2369654A55
:101460001B0311D58DF808105379116B0B440B2019
:101470005A788DF80920DA7A8DF80A205B7D8DF88C
:101480000B3002A9F5F758F90123226B84F82030BC
:10149000637913440022DA7291E0B4EEE78AF1EE48
:1014A00010FA48BF83ED078AA16B636B94ED067A4F
:1014B000D4ED076A591AC943C90F77EE667A59B94C
:1014C000B7EE006AF4EEC67AF1EE10FA79DDB4EE0A
:1014D000E68AF1EE10FA74DDD4ED056A454BB4EE00
:1014E000E67AF1EE10FACCBF0126002666B1D3ED04
:1014F000097A9FED427A67EE877A9FED427AC3EDD3
:10150000097AD3ED0B7A0AE0B0EE007AF4EEC77AEE
:10151000F1EE10FA08DDD3ED0B7A9FED387A67EE25
:10152000877AC3ED0B7A07E0D3ED097A9FED357A20
:1015300067EE877AC3ED097AD4ED097A206B627978
:1015400067EEA87A1044FCEEE77ACDED017A9DF8BB
:1015500004304370D4ED0B7A2769FCEEE77A3F0341
:10156000CDED017A9DF8042042750ED546EA410181
:101570008DF808108DF80930C37A8DF80A300B20E9
:1015800002A98DF80B20F5F7D7F894F82020194B15
:10159000022A11D1D3ED0A7A9FED1B7A196B67EEFF
:1015A000877A002283F82020FCEEE77A5A7917EE3A
:1015B000903A0A44D37202E0022283F82020F6F720
:1015C000E5FFA2790B4B0AB1104A00E0104ADA603D
:1015D0002544D4ED037AB5F9083000EE103AB8EEA0
:1015E000C00A80EE280A37EEC00A05B0BDEC028BB7
:1015F000F0BD00BFEC270020A8970108EC51783F10
:101600006F12833A0AD7833F00007A440000A0415A
:101610000000A0C12B4BF0B52B4D1E6805F110004A
:101620002F78F3192C46597801F00401013501F0A7
:10163000FF0219B18542F3D10020F0BD224D631B9A
:10164000022B0ADD1AB102EB82025200D2B215F867
:10165000013B303B1A44D2B2F1E70021AC420AD937
:1016600019B101EB81014900C9B215F8013B303BCA
:101670001944C9B2F2E72E2F16D1013404200023F9
:101680002578771903EB83037F785B007F079BB294
:1016900044BF303D5B1900F1FF3044BF01349BB2C1
:1016A00010F0FF00ECD100E0002308484143642023
:1016B00000FB03130620B3FBF0F3054800FB0230E8
:1016C000F0BD00BF900000202828002040420F00FD
:1016D0008096980030B500231A4610498C1894F86B
:1016E0003C40BCB12E2C06D1013298B18C18044478
:1016F000002584F83C5011440A2491F83C106343BF
:10170000A1F13004092C9CBF303B5B180E2A03D892
:101710000132E2E7184630BD002030BDEC27002042
:10172000104B10B50446185CF9F777F90E4800EB3A
:101730004400B0F94C10B1F57A7F05DBB1F5FA6FD2
:10174000A8BF4FF4FA6101E04FF47A71A1F57A7104
:101750000A23092091FBF3F1BDE81040C9B2FCF760
:1017600063BA00BF06B80108EC270020031EB8BF0B
:101770002D2210B5B8BF58420C46B8BF01F8012B56
:101780000A22F9F7A5FB00230370204610BD00BF15
:1017900007B5064B0093064B01930649064A074BD3
:1017A0000748F9F7ABFC03B05DF804FBB4A70108E8
:1017B00089A7010895AE01088EAE0108A8A7010807
:1017C0001BB8010808B5037833B90C4B0C481978DD
:1017D000BDE80840F9F792BC04F0CAFC02280CD816
:1017E000064B1870074B0C2202FB0030064B0630EC
:1017F0001860F9F7A9FE0548E5E708BD6028002054
:101800003BB80108D033002070100020ABAA0108BB
:1018100008B503783BB90B4B0B4893F8B417BDE8F8
:101820000840F9F76BBC04F0A3FC022808D8054B6C
:1018300083F8B407F9F7F2FDF9F7AAFE0348E8E7E1
:1018400008BD00BF202C00203FB80108ABAA01084A
:1018500038B5037803BB214B1B6801330F2B07D826
:101860001F490C2202FB03121C4695682DBB00E0A9
:101870001C4601340F2C01DD002400E005D8184976
:101880000C2202FB04129568BDB99C42F1D11548A7
:10189000BDE83840F9F732BC04F06AFC0F28044672
:1018A00005D80F4A0C2303FB00239D682DB9214660
:1018B0000D48BDE83840F9F721BC084B1C60FAF729
:1018C000E7F821462A460948F9F718FC0C235C433F
:1018D000034B185DBDE83840FAF7EEB87C000020F5
:1018E000AC9701084CB8010862B801087AB8010841
:1018F00073B5037813B9F5F7A3FB3DE01F4901AABF
:1019000004F097FC002401462646254699B134B1DF
:10191000012C08D1084604F02BFC064603E00846DB
:1019200004F026FC05461549002001AA04F081FCBC
:1019300001340146EAE70B2D02D911480C220BE0D5
:10194000022C10D1A6F57A73B3F57A7F07D90D482A
:101950004FF47A714FF4FA62F5F7EFFA0CE00A4BA4
:1019600003EB45035E80084B084803EB450329461B
:10197000B3F90220F9F7C2FB02B070BD41B1010812
:1019800024AD0108EDB401086028002091B80108D9
:1019900038B50D4C23688342054606D1F5F799FF0B
:1019A000204600214C2204F048FBE36CAB4209D1F5
:1019B0002846F5F78EFF054800214C22BDE8384047
:1019C00004F03BBB38BD00BF70220020BC220020C9
:1019D000034B1A68D379591C1344D171187A704794
:1019E000B411002010B5FFF7F3FF84B2FFF7F0FF4A
:1019F00004EB002080B210BD10B5FFF7F3FF0446E2
:101A0000FFF7F0FF04EB004010BD064B10B5044695
:101A100021461868FAF7DBF8034B1B689879604099
:101A2000987110BDB8110020B4110020014B1B6843
:101A30009879EAE7B411002038B5044624200D4611
:101A4000FFF7E3FF4D20FFF7E0FF002C084C14BF29
:101A500021203E20FFF7D9FF2368002228469A71F3
:101A6000FFF7D3FF236893F84900BDE83840CCE77F
:101A7000B411002001460020DEE710B50446C0B2D4
:101A8000FFF7C3FF200ABDE81040BEE710B50446CB
:101A900080B2FFF7F2FF200CBDE81040EDE737B54C
:101AA00082888368044610060D4641BF2B4991F891
:101AB000B4174FF4CC7000FB0133D10544BF284963
:101AC000097802F03F0244BF01EB410103EB8103BF
:101AD000042A12D006D8012A0DD0022A32D193F955
:101AE000001030E0102A0AD0202A0AD0082A29D172
:101AF000B3F9001027E0197825E0198823E0196868
:101B000021E093ED000A6846F9F778F90146154897
:101B1000F9F7F4FA05B3D4ED037A6846B8EEE70AAC
:101B2000F9F76CF901461048F9F7E8FA94ED040A60
:101B30006846B8EEC00AF9F761F901460A48F9F7B4
:101B4000DDFA09E000210948F9F7D8FA25B108487B
:101B5000E1682269F9F7D2FA03B030BD202C0020E9
:101B600060280020C9AF0108C2AF01086DAF0108AD
:101B7000A0B80108024B0146D869FAF728B800BF9F
:101B80006028002010B5441E14F8011F21B1034B3A
:101B9000D869FAF71CF8F7E710BD00BF60280020ED
:101BA00010B503781BB90A48BDE81040EAE704F015
:101BB000DFFA0446082899BF21460648064808214E
:101BC000F9F79CFA601E40B2BDE81040F5F704BE7C
:101BD000A7B80108EEB801081AB90108F7B52B49F2
:101BE0002B4B08782B4D1C682B4B05EB80001A887B
:101BF0002A4BD0F8C0101B78294800914FF47A7115
